:1000000070060020C5000000C1000000C100000013
:1000100000000000000000000000000000000000E0
:10002000000000000000000000000000C10000000F
:100030000000000000000000C1000000C10000003E
:10004000C1000000C1000000C1000000C1000000AC
:10005000C1000000C1000000C1000000C10000009C
:10006000157C0000818600004D7C0000C10000006E
:10007000C1000000C1000000899C0000C100000018
:10008000C1000000C1000000C1000000C10000006C
:10009000C1000000C1000000C1000000C10000005C
:1000A000C1000000C1000000C1000000C10000004C
:1000B000C1000000C1000000C1000000C10000003C
:1000C000FEE7C04610B5154B154A9A420ED2154BA5
:1000D000124A0332D21A92080132920000231048C9
:1000E0001149CC58C45004339342FAD10F4B104AF3
:1000F0009A420ED20F4B0D490331C91A89080131BA
:1001000089000023140000201A19106004338B4268
:10011000FAD109F0D3FE02F0C9FA10BD0C0000209C
:10012000000000200400002074D500006C020020B4
:100130000C00002010000020F8B5CA4B1B78DBB281
:10014000FF2B00D0FCE0C84B1B78DBB2FF2B00D0AC
:10015000C6E0C54B5B78DBB2412B1FD002D8402BE9
:1001600005D0BDE0422B41D0432B75D0B8E0BF4B4A
:100170001B68BD4A9278D2B25B0DDBB2934200D0CD
:10018000AEE00023B848BA49C25CD2B2CA540133C7
:10019000092BF9D10122B74B1A70A1E0B34B1B68B0
:1001A000B14A9278D2B25B0DDBB2934200D097E0B5
:1001B000AE4B1B689B0BDBB2AF4A137011787F23E9
:1001C0000B401370A84BDB781278DBB2934200D05F
:1001D00086E00023A448A649C25CD2B2CA540133C7
:1001E000092BF9D10122A34B1A7079E09F4B1B68B0
:1001F0009D4A9278D2B25B0DDBB2934270D19B4B99
:100200001B689B0BDBB29C4A137011787F230B4059
:100210001370954BDB781278DBB2934260D1934B2D
:100220001B68DB09DBB2944A137011787F230B4003
:1002300013708D4B1B791278DBB2934250D100239F
:1002400089488B49C25CD2B2CA540133092BF9D117
:100250000122884B1A7043E0844B1B68824A9278D3
:10026000D2B25B0DDBB293423AD1804B1B689B0B41
:10027000DBB2814A137011787F230B4013707A4BE5
:10028000DB781278DBB293422AD1784B1B68DB090A
:10029000DBB2794A137011787F230B401370724BD5
:1002A0001B791278DBB293421AD1704B1A68D2B222
:1002B000714B1A7019787F220A401A706A4A527973
:1002C0001978D3B28B420BD1002367486849C25CCE
:1002D000D2B2CA540133092BF9D10122654B1A70ED
:1002E000614B5B78042B01D002F0BEF95E498B783C
:1002F000CA780C7949790320184040057F231A40B9
:100300009203024319400A432340DB0113435B4A33
:1003100013601268554B1B689A4201D002F0A4F991
:100320000022574B1A70C832564B1A704E4B1B782E
:10033000DBB24C4A13700122534B1A7002F094F94D
:10034000494B1B78DBB2FF2B00D034E2FF22484B35
:100350001A704C4B1B78002B0CD04C4A1278002A98
:1003600008D1013BDBB2474A1370002B02D1FF22B8
:100370003C4B1A703C4B5B78033BDAB2402A00D905
:1003800014E29300424AD3589F460522414B1A700B
:1003900002F06AF90123404A1370404A1360394A57
:1003A00013780133137002F05FF93D4A1378DBB222
:1003B0003C490B702C4B9B78DBB213700B78127896
:1003C000DBB2934201D102F04FF9374B1B78002B7F
:1003D0002AD0FF22234B1A700023344A1370344A68
:1003E0001370344B1B889BB2002B04D0314B1B88FD
:1003F0009BB2314A138007F013FE07F07DF800220C
:10040000294B1A70A022D20580235B0059241620A4
:100410008821D450D050D150D558002DF9D0012288
:10042000A023DB059A60FEE70122174B1A701C4BD4
:100430001B78DBB2062B00D913E19B001F4AD3586F
:100440009F461F4B01241C61DC619C620021062039
:1004500007F058F81B4807F07DF8134B1C7002F0AA
:1004600003F9C046E40000201C02002054020020D2
:10047000E8000020F601002047020020A80100202B
:10048000210100200C000020440200202F02002047
:10049000B4A10000AC0100208800002038420050C8
:1004A000B2010020430100203F020020DA010020B9
:1004B000310100208C0000203C010020B8A2000087
:1004C00000000440ECCA0000C74B01221A61DA6147
:1004D0009A62FE32C54B1A700023C54A1370C54A92
:1004E0001370C54B1B889BB2002B04D0C24B1B88DA
:1004F0009BB2C24A138007F093FD06F0FDFF012274
:10050000BF4B1A70A022D20580235B00592416200D
:100510008821D450D050D150D558002DF9D0012287
:10052000A023DB059A60FEE7AF4B01221A61DA6176
:100530009A6202F099F8B34B1B78002B17D0B24B9C
:100540001A780132A84B1A61B04A12780132DA6186
:10055000AF4A127801329A629A68802149000A43B0
:100560009A609A68802149020A439A6004E0A64B87
:100570001B7801339C4A93629B4A916801230B4389
:100580009360A44B1B889BB2002B01D002F06CF847
:1005900000229B4B1A7002F067F89A4B1B78002BD5
:1005A00017D09D4B1A7801328F4B1A619B4A1278F3
:1005B0000132DA619A4A127801329A629A6880218D
:1005C00049000A439A609A68802149020A439A6066
:1005D00004E08D4B1B780133834A9362824A916811
:1005E00001230B4393608B4B1B889BB2002B01D0E4
:1005F00002F03AF80022824B1A7002F035F8814B73
:100600001B78002B17D0874B1A780132764B1A6172
:10061000854A12780132DA61844A127801329A628C
:100620009A68802149000A439A609A6880214902A9
:100630000A439A6004E0744B1B7801336A4A936260
:10064000694A916801230B439360724B1B889BB2EC
:10065000002B01D002F008F80022694B1A7002F05A
:1006600003F8684B1B78002B11D05F4B06221A61F0
:10067000033ADA6102329A629A68802149000A4399
:100680009A609A68802149020A439A6004E05E4BAE
:100690001B780133544A9362534A916801230B43F8
:1006A00093605C4B1B889BB2002B01D001F0DCFFF8
:1006B0000022534B1A7001F0D7FF504B1B889BB29E
:1006C000002B01D001F0D0FF4B4B9B7EDB0701D507
:1006D00001F0CAFF484B9B7E9B0701D501F0C4FF88
:1006E000534B1B889BB2002B01D001F0BDFF514B37
:1006F000DA789978404B1B88D2018A185B045B0C2E
:100700009A4201D001F0B0FF07F08AFC0023394A79
:100710001370374A13700122474B1A7001F0A4FF7F
:10072000464B1B78022B01D001F09EFF0522444B63
:100730001A7001F099FF3F4882787F231A40110018
:10074000C2782D4B1B88D20152185B045B0C9A4275
:1007500001D001F089FF01797F230B402649CB703E
:1007600043795B0606D50A00098880231B020B43E8
:10077000138004E0204A13885B045B0C13802D482F
:100780008279D2001C4B9A6042799C683F210A40D2
:10079000920212199A60C27999685206520F0A435E
:1007A0009A600122244B1A7001F05EFFC822254B8B
:1007B0001A7001F059FF1F4B1B780C4A1278DBB2FC
:1007C000934201D001F050FF09F0EEF9C8221D4B11
:1007D0001A70184B5B78DBB2252B01D901F042FF70
:1007E0009B00194AD3589F4600000440E4000020B3
:1007F000DA010020310100208C0000203C010020A3
:100800003F0200202F010020F10100209C01002068
:1008100064000020C0010020FF01002078010020BA
:100820004202002062010020420100209A010020C3
:100830007C0100201C02002044020020460200200F
:10084000FE0100200C000020D4A20000D54B1B8824
:100850009BB2002B40D0D44B1B78002B3CD1D34B08
:100860001B78002B38D1D24B1B78002B34D1D14BC5
:100870001B88D14A1340934202D10022CD4B1A80EB
:10088000CE4C01236370C74B1A887F210A40A270A7
:100890001B88DB090B40E370002323716371A37194
:1008A000E371200009F070F92072C5490B889BB2F2
:1008B0005A1E92B20A80002B05D10122C14B1A7038
:1008C0000022B84B1A800023BF490022CA540133CA
:1008D000202BFBD101F0C8FEBC4B1B78002B14D0A1
:1008E000BA4E3378DBB2B54C63707378DBB2A37069
:1008F0000025E57025716571A571E571200009F08D
:1009000043F92072357001F0AFFEB14B1B78002B1C
:1009100046D00022AE4B1A70A84904234B70AD4A52
:1009200010887F24204088701388DB092340CB7017
:1009300053792E3BDAB2092A12D89300A64AD3582B
:100940009F4600229D4B1A710AE001229B4B1A71AF
:1009500006E00222994B1A7102E00322974B1A71AA
:100960009C4B5B792E3BDAB2072A09D893009B4A4D
:10097000D3589F46914A117904230B43137104E025
:100980008E4A117908230B4313718C4C0023637139
:10099000A371E371200009F0F7F8207201F064FE02
:1009A0008F4B1B78002B1ED000238D4A1370834C75
:1009B00013226270874D298B7F200140A1702A8B02
:1009C000D2090240E27023716371A371E3712000C8
:1009D00009F0DAF820722B889BB2724A138007F074
:1009E0001FFB01F041FE7F4B1B78002B00D183E001
:1009F00000227B4B1A70774B1B8B9BB2002B27D1AD
:100A00006E4B14325A7000229A70DA70714908885D
:100A10007F24204018710A88D20922405A714B79EC
:100A20002E3BDAB2092A5ED893006F4AD3589F460C
:100A30000022624B9A7156E00122604B9A7152E09B
:100A400002225E4B9A714EE003225C4B9A714AE09F
:100A500064490B78013BDBB20B701822D31ADBB26E
:100A6000564A53705B4B188B7F24204090701B8B31
:100A7000DB092340D3700B78DBB2012B1DD0002B98
:100A800027D0022B0DD0032B2DD1524A117BC9B296
:100A90004A4B1971517BC9B25971927BD2B29A718A
:100AA00021E04C4AD17BC9B2444B1971117CC9B2C7
:100AB0005971527CD2B29A7115E0464A917CC9B202
:100AC0003E4B1971D17CC9B25971127DD2B29A7163
:100AD00009E040494A7DD2B2384B1A718A7DD2B2C0
:100AE0005A7100229A71354C0023E371200009F0FD
:100AF0004BF8207201F0B8FD3C4B1B78002B20D046
:100B00002E4C0D23637033490B887F200340A37064
:100B10000A88D2090240E2708A68120C02402271EF
:100B20008B68DB0D034063718B689B0FA3710025FD
:100B3000E571200009F028F820722C4B1D7001F09F
:100B400093FD2B4B1B78002B56D01C491B234B705D
:100B5000204A13887F2003408B701288D2090240FC
:100B6000CA70244A138803400B711388DB090340C1
:100B70004B7113885B04DB0F8B7113881BB2002B46
:100B800004DA0A00897940230B4393710B4C00254A
:100B9000E571200008F0F8FF2072154B1D7001F080
:100BA00063FDC0463C0100203F02002019020020E6
:100BB00040000020680000200F070000E80000202F
:100BC000B401002044020020FC0000203801002075
:100BD000320100208C0000206CA3000094A30000D0
:100BE0007000002050020020B4A300006500002027
:100BF000C20100206C010020CB4B1B78002B11D0D0
:100C0000CA4C242363700025A570E57025716571B9
:100C1000A571E571200008F0B7FF2072C24B1D706E
:100C200001F022FDC24B1B78002B48D02422BF4B81
:100C30005A70BF4B1B78012B27D1233ABB4B9A70BC
:100C4000BC4B1B78002B04D0BB4A117808230B4304
:100C50001370BA4B1B78002B04D0B74A11780123CC
:100C60000B431370B64B1B78002B04D1B24A11789A
:100C700004330B431370B04B1B78DBB2AB4AD37019
:100C8000B04B1B78DBB2137109E0A84B02229A70BB
:100C90000B32DA70063A1A710022A74B1A70A34C75
:100CA00000236371A371E371200008F06DFF2072CF
:100CB0009F4A1378013BDBB2137001F0D5FCA24BC5
:100CC0001B78002B35D0994B24225A70213A9A7008
:100CD0009D4B1B78012B05D1944B0022DA701A71C1
:100CE0005A7117E0994C208880B2052109F032F939
:100CF00080B220808D4A0123D37021887F2001405B
:100D000011712388DB09034053718F4A1378013B2B
:100D1000DBB21370854C0023A371E371200008F04F
:100D200033FF2072884A1378013BDBB2137001F065
:100D30009BFC874B1B78002B13D07C4C24236370C7
:100D40000025A570E57025716571A571E57120001C
:100D500008F01AFF2072744B1D707D4B1D7001F05E
:100D600083FC7C4B1B78002B3DD0704B24225A70A7
:100D70001D3A9A70774B1B78012B0CD1764B198852
:100D80007F200140694AD1701B88DB090340137141
:100D90007F23537118E0704B1A887F20024063490B
:100DA000CA701B88DB0903400B716C4B1B78002B4E
:100DB00002D003224A7102E001225C4B5A71654A5B
:100DC0001378013BDBB21370584C0023A371E3711D
:100DD000200008F0D9FE20725E4A1378013BDBB296
:100DE000137001F041FC5E4B1B78002B43D05C4B31
:100DF0001B78DBB2022B13D0032B21D0012B2ED179
:100E00004A4A10335370574B598A7F2001409170E2
:100E10005B8ADB090340D3700022514B1A701EE03D
:100E2000424A102353704F4B598A7F2001409170E2
:100E30005B8ADB090340D3700022494B1A700EE035
:100E40003A4A12235370474B598A7F2001409170D0
:100E50005B8ADB090340D3700022414B1A70334C8C
:100E6000002323716371A371E371200008F08CFEED
:100E7000207201F0F9FB3C4B1B78002B00D17DE088
:100E8000394B1B78032B1FD1284C03336370374B2E
:100E90001A887F210A40A2701A88D2090A40E2709B
:100EA0001B889B0B0B402371012363710023A371EB
:100EB000E371200008F068FE20722B4A1378013B92
:100EC000DBB2137001F0D0FB274B1B78012B27D12D
:100ED000164D05336B70254C23887F210B40AB707A
:100EE0002288D2090A40EA7023889B0B0B402B71A1
:100EF00000266E71AE71EE71280008F045FE287272
:100F00001B4B1E70184A1378013BDBB21370012291
:100F1000184B1A70184B1B889BB2238001F0A4FB5E
:100F200008F042FE01F0A0FB70010020E800002064
:100F30003C02002030010020B80100203D020020CA
:100F4000230100204101002043020020A4010020D1
:100F5000B7010020DD000020980100202D020020B4
:100F600042000020740000204602002030020020D1
:100F70003B01002044020020D6010020CE4B1B780C
:100F8000002B00D105E10022CB4B1A702432CB4B51
:100F90005A70CB4B1B78002B00D1A2E00022C74B2C
:100FA0009A71C84B1B78DBB2082B08D002D8012BF2
:100FB00008D04CE0092B0FD00A2B29D047E00122A2
:100FC000BE4B9A71BD4B0F229A700D32DA7000221F
:100FD0001A7105325A717AE0B8490D238B70BA4AFA
:100FE00013887F2003404B711288D20902408A7116
:100FF000B64C2288013A92B222800240CA702288FE
:1010000093B25A1C92B22280DB0903400B715EE05E
:10101000AD4B1A88120AC0231A43AD4B5A80A74918
:101020000D238B707F2422404A710C3B8B71A748A3
:101030000288013A92B202802240CA70028893B2BA
:101040005A1C92B20280DB0923400B713FE0A14B96
:101050001B78002B08D0994A112393709A4B1B8858
:101060009B045B0E937113E09B4B1B78012B07D104
:10107000924A0E339370994B1B78DBB2937107E061
:101080008E4A0D239370904B1B889B045B0E9371CB
:101090008D4B1A887F231340884A53718B4B1B88D2
:1010A0009BB2002B02D10122884B1A8087490A8803
:1010B000013A92B20A807F2422408048C2700A8896
:1010C00093B25A1C92B20A80DB09234003717D4B14
:1010D0001B78002B54D07B4A1378013BDBB2137092
:1010E0004EE0784B1B78102B05D1764A1378013BE4
:1010F000DBB213700DE0734B1B780F2B09D1714AD3
:101100001378013BDBB21370704A138801339BB232
:101110001380704B1B78002B05D0684B10229A70FF
:1011200000225A7110E06C4B1B78012B07D1634AE7
:101130000D339370644B1B88DBB2537104E05F4B3B
:101140000C229A7000225A7100225C4B9A715F4BFC
:101150001B889BB2002B02D101325C4B1A805B4989
:101160000A88013A92B20A807F2422405348C27012
:101170000A8893B25A1C92B20A80DB092340037199
:101180004E4C0023E371200008F0FEFC207201F0B9
:101190006BFA534B1B78002B30D00022504B1A7047
:1011A000464A082353704F4B19887F2001409170A5
:1011B0001B88DB090340D370444B1B889BB2002B78
:1011C00002D10122414B1A8040490A88013A92B269
:1011D0000A807F200240394C22710A8893B25A1C3F
:1011E00092B20A80DB09034063710023A371E371AB
:1011F000200008F0C9FC207201F036FA3A4B1B7847
:10120000002B3BD00022384B1A702C4A0723537016
:10121000344B19887F20014091701B88DB09034003
:10122000D3702A4B1B889BB2002B02D10122274B83
:101230001A8026490B88013B9BB20B807F2213400A
:101240001E4803710B889BB25C1CA4B20C80DB09A6
:10125000134043711C4B19880A4082711B881B067E
:1012600003D5417940230B434371144C0023E371B0
:10127000200008F089FC207201F0F6F91B4B1B7866
:10128000002B35D00022194B1A700C4C24236370AC
:101290001B3BA3700C4B19887F200140E1701B8819
:1012A000DB09034023716271A271E271200008F032
:1012B0006BFC207201F0D8F9F9000020E800002052
:1012C000260100205C0000203601002030020020B2
:1012D0000C0000203F010020330100205D000020B1
:1012E000DC0100208C000020D80100203E020020FC
:1012F000E14B1B78002B1CD00023DF4A1370DF4A20
:101300001278D2B2DE4C227010226270DD49088B56
:101310006F320240A2700A8BD209D2B2E2702371FE
:101320006371A371E371200008F02EFC207201F0BC
:101330009BF9D54B1B78002B1FD0D14B24225A7020
:10134000203A9A70D04B1B78012B03D16032CC4BE2
:10135000DA7004E0CD4B1B78DBB2C94AD370C84CBD
:10136000002525716571A571E571200008F00CFC60
:101370002072C54B1D7001F077F9C54B1B78002B0F
:1013800036D02422BE4B5A70C14B1B78DBB2062BE1
:101390001DD89B00BF4AD3589F460122BC4B1A70F0
:1013A000B74B01229A703F32DA7010E00122B84B3D
:1013B0001A70B34A05239370B74B1B78013BDBB21D
:1013C000D37004E0AE4B02229A703E32DA70AC4C1D
:1013D000002323716371A371E371200008F0D4FB33
:1013E0002072AB4A1378013BDBB2137001F03CF979
:1013F000AA4B1B78002B24D02422A14B5A70A74B58
:101400001B78022B0AD1A54A1378013BDBB213707B
:101410009B4B01229A703F32DA7006E000229F4B0C
:101420001A70974B05219970DA70954C002323713F
:101430006371A371E371200008F0A6FB207201F034
:1014400013F9974B1B78002B34D00022944B1A7061
:101450008B4A03235370934B19887F20014091706E
:101460001979014011711988C9090140D1701969B0
:101470000904890E51711B881BB2002B04DA5179C3
:1014800040230B43537104E07D4A537940218B4341
:101490005371844B1A69D2087F210A40784CA2719B
:1014A0001B691B010B40E371200008F06DFB2072EB
:1014B00001F0DAF87C4B1B78002B4BD0714B1A886B
:1014C0007F2002406E498A701B88DB090340CB7085
:1014D0000022764B1A70744B1B78022B1AD10532FE
:1014E0004A7000240C714C716F4A1378013BDBB2D7
:1014F00013706E4D01232B7006F092FD2C70614B22
:101500009A7E02218A439A761B885B045B0C684AA8
:1015100013800DE05A4902234B70654A10887F24DE
:10152000204008711388DB0923404B71002313808E
:10153000534C0023A371E371200008F025FB2072B7
:10154000594A1378013BDBB213700122594B1A70D0
:1015500001F08AF8584B1B78002B1ED00022564B06
:101560001A70474C1E236370464B19887F20014038
:10157000A1701B88DB090340E370504B1B78DBB282
:1015800023714F4B1B78DBB26371A271E2712000B3
:1015900008F0FAFA207201F067F84A4B1B78002B2A
:1015A00018D00023474A1370354C1F226270354A09
:1015B00011887F200140A1701288D2090240E27098
:1015C00023716371A371E371200008F0DDFA2072CA
:1015D00001F04AF83C4B1B78002B1BD000223A4B01
:1015E0001A70274C1D236370264B19887F200140F9
:1015F000A1701B88DB090340E370304B1B78DBB222
:1016000023716271A271E271200008F0BDFA2072AC
:1016100001F02AF82D4B1B78002B25D01C22184BEB
:101620005A702A4B1B78052B09D1154B0D3A9A702D
:101630000D3ADA70013A1A7100225A7108E0104B23
:1016400000229A70DA701A715A71C832204B1A70DF
:101650000B4C0025A571E571200008F095FA207269
:101660001A4B1D7001F000F800221A4B1A7008F096
:101670009BFA00F0F9FFC046DB010020E4000020E7
:10168000E80000208C000020400200206E010020B5
:1016900032020020DCA30000D9010020DE0000207F
:1016A000B6010020000200202E0200204000002091
:1016B0003C01002044020020890000204802002054
:1016C0009E0100203E01002045020020AC010020C8
:1016D00041020020190200200022CD4B1A70CD4B90
:1016E00019000A3120321A7001339942FBD1CA4BDA
:1016F000D9780904C94A11601979106809020143AF
:1017000011605879116801431160DA78C1493032AB
:101710000A702E224A701B79DBB20224092B09D9E8
:10172000BD4B1879C0B20A2108F014FC3030B94B17
:1017300098700134A31CB84EF05CC0B2B54F0A21BA
:1017400008F08EFC30313955651C2E237B55AB1CBF
:10175000F35CDBB2092B08D9A51CE31CF05CC0B21A
:101760000A2108F0F7FB303078556C1CE4B2631C9A
:10177000A94EF05CC0B2A74F0A2108F071FC3031CD
:1017800039550023BB72A31CF35C002B04D0AC1CA6
:10179000E4B2631CF25C3A55A31C9F4AD35C002B55
:1017A00006D00134E4B2631CD35C3033994A13553C
:1017B0009A4B1A689A4B9A4203D80122994B1A7095
:1017C00002E00022974B1A7008F0EEF900F04CFF8F
:1017D000914A5379DBB294490B701379DBB2527999
:1017E000D2B29249CA540122914B1A7008F0DCF926
:1017F00000F03AFF884B5B79002B06D0864A1379BC
:10180000DBB25279D2B28949CA54834BDB79002BBF
:1018100006D0814A9379DBB2D279D2B28349CA54D5
:101820000122834B1A7008F0BFF900F01DFF7A4BBC
:101830009B78DBB27F4A137008F0B6F900F014FF12
:101840007D4B1B889B0700D5A2E173498A787F23D3
:101850001A40C9780B40DB019B18784A1278002A9D
:1018600000D1B8E0744A118802230B4313806A4BFD
:101870009B79002B03D1684B5B79002B02D00022AF
:101880006F4B1A83644803799B08032213406C4909
:101890000B7103791A408A700B79DBB2012B24D0CB
:1018A000002B02D0022B44D067E0654B0E221A7148
:1018B0009B78DBB2012B0CD0002B04D0022B0CD078
:1018C000032B0ED05EE05E4B37225A7147321A71FD
:1018D00058E02E225A4B5A7154E03122584B5A711B
:1018E00050E03422564B5A714CE0554B9B78DBB29A
:1018F000012B0CD0002B04D0022B0ED0032B12D0C6
:1019000040E04F4B37225A7147321A713AE04C4B44
:101910001B221A7114325A7134E0494B1B221A717E
:1019200017325A712EE0464B1C221A7119325A7125
:1019300028E0434B9B78DBB2012B0CD0002B04D06A
:10194000022B0ED0032B12D01CE03D4B37225A71D4
:1019500047321A7116E03A4B1B221A7115325A712E
:1019600010E0374B1B221A7118325A710AE0344BBF
:101970007E221A71483A5A7104E0314B37225A716B
:1019800047321A712E4AD3781279DBB2934203D9C7
:101990002B4A1379DBB2D370294B5B79294A5279F0
:1019A000DBB2934207D006F03BFB0022234B1A70B8
:1019B00001321F4B1A70204B1A880B2313400B2B3C
:1019C00000D0E5E000221D4B1A701E4A917E0223D2
:1019D0000B439376DCE01B4A12885204520C93426C
:1019E00000D0D5E0144A118802230B4313800A4B20
:1019F0009B79002B03D1084B5B79002B24D0064A3E
:101A000093795279DB01D3180E4A13831FE0C04645
:101A100041020020580200201C0200206C0000201F
:101A200001000200FC0100209E010020FC000020BB
:101A3000440200202F020020680000204000002007
:101A40007C0100208C0000200022CE4B1A83CE485F
:101A500003799B0803221340CA490B7103791A408A
:101A60008A70C379887E012213405A00022398436A
:101A7000030013438B768B7E9B0708D4C34D012450
:101A80002C7006F0CDFA00232B70C14B1C70BD4B9F
:101A90001B79DBB2012B24D0002B02D0022B44D0C7
:101AA00067E0B84B0E221A719B78DBB2012B0CD089
:101AB000002B04D0022B0CD0032B0ED05EE0B14BD8
:101AC00037225A7147321A7158E02E22AD4B5A71A3
:101AD00054E03122AB4B5A7150E03422A94B5A7179
:101AE0004CE0A84B9B78DBB2012B0CD0002B04D030
:101AF000022B0ED0032B12D040E0A24B37225A719A
:101B000047321A713AE09F4B1B221A7114325A71F4
:101B100034E09C4B1B221A7117325A712EE0994BFC
:101B20001C221A7119325A7128E0964B9B78DBB24D
:101B3000012B0CD0002B04D0022B0ED0032B12D083
:101B40001CE0904B37225A7147321A7116E08D4BC8
:101B50001B221A7115325A7110E08A4B1B221A711E
:101B600018325A710AE0874B7E221A71483A5A712C
:101B700004E0844B37225A7147321A71814AD37874
:101B80001279DBB2934203D97E4A1379DBB2D37068
:101B900008F00AF800F068FD7C4B1B78002B47D159
:101BA0007C4B1B885B0743D4774B9978DB78754B6C
:101BB0001B887F220A405B045B0C9A4238D1754A2D
:101BC000118804230B4313806F4A1379DBB26D49EC
:101BD000CB7053795B0606D50A00098880231B0267
:101BE0000B43138004E0674A13885B045B0C13808B
:101BF000644A9168684B0B409360634B59799068D5
:101C00008C0266492140014391609068644901401B
:101C1000916099799068C9000143916091680720AB
:101C200081439160DB7991685B065B0F0B439360A6
:101C300007F0BAFF00F018FD564B1B881B0700D5B4
:101C400091E0514883787F210B401A00C3780B4004
:101C5000DB019B184D4A1278002A43D0514A128862
:101C60005204520C93422DD14A4A118808230B4347
:101C700013804C4B98684C4901409960424908795F
:101C80009C680004204398609C6848482040986005
:101C900048799C68C005204398609C68444820406F
:101CA0009860897998688907014399601088E021D4
:101CB000C900014311800121354A11703D4A0C339E
:101CC00013CA13C3334B1A880B2313400B2B00D0BA
:101CD0007EE000222D4B1A702A4A917E02230B438C
:101CE000937675E0274A12885204520C93426FD1C2
:101CF000284A118808230B431380224B99682A4AEB
:101D00000A409A60204A1179986809040143996051
:101D1000986826490140996051799868C90501433E
:101D20009960986822490140996092799968920770
:101D30000A439A601B8B9BB2002B03D001221E4BDF
:101D40001A7045E001221D4B1A7012490888E023E1
:101D5000DB0003430B800E4B1A70164A094B0C3301
:101D600013CA13C334E00B4B1B88154A134093422C
:101D70002ED0044B1B8B9BB2002B23D001220E4B89
:101D80001A7025E08C0000201C020020400000207A
:101D90004402002068000020FF03FFFF00FCFEFF5C
:101DA00007FCFFFF7C010020FFFF80FFFFFF7FC0DB
:101DB000FFFF7F3F44CC0000DB0100203E010020FC
:101DC0000B070000CC4A1188E023DB000B43138093
:101DD00007F0EAFE00F048FCC84883787F210B40FA
:101DE0001A00C3780B40DB019B18C54A1278002A01
:101DF00007D09B049B0CC34A53820222C24B1A7029
:101E000003E09B049B0CC14A138307F0CDFE00F056
:101E10002BFCBA4883787F210B401A00C3780B4013
:101E2000DB019B18B64A1278002A00D18CE09BB2E5
:101E3000B44A138003799B087C390B40D370037933
:101E400019409170D378DBB2012B24D0002B02D043
:101E5000022B44D067E0AB4B0E22DA709B78DBB2EA
:101E6000012B0CD0002B04D0022B0CD0032B0ED056
:101E70005EE0A44B37221A714732DA7058E02E2206
:101E8000A04B1A7154E031229E4B1A7150E034225B
:101E90009C4B1A714CE09B4B9B78DBB2012B0CD016
:101EA000002B04D0022B0ED0032B12D040E0954B18
:101EB00037221A714732DA703AE0924B1B22DA70FD
:101EC00014321A7134E08F4B1B22DA7017321A71F8
:101ED0002EE08C4B1C22DA7019321A7128E0894BE3
:101EE0009B78DBB2012B0CD0002B04D0022B0ED040
:101EF000032B12D01CE0834B37221A714732DA7061
:101F000016E0804B1B22DA7015321A7110E07D4BFF
:101F10001B22DA7018321A710AE07A4B7E22DA70CC
:101F2000483A1A7104E0774B37221A714732DA7057
:101F300072494B79DBB2734A53718B79DBB293717F
:101F40000122734B1A7023E0704A12885204520C1B
:101F500093421DD1684B1B88DB0510D4664A11885B
:101F600080235B000B43138064494B79DBB2674AE3
:101F700013738B79DBB253730122654B1A705E4B7E
:101F80001B88644A1340934202D10022624B1A60BC
:101F900007F00AFE68E35A4B1B78002B14D0574A0F
:101FA0009178C9B2574BD971D178C9B219721179E8
:101FB000C9B259725179C9B299729279D2B2DA72B0
:101FC0000122534B1A702AE04B4B1B88DB0500D4CF
:101FD0004AE3494B1B889B0521D447490A88802343
:101FE0009B0013430B80454A9078C0B2474B9873CF
:101FF000D078C0B2D8731079C0B218745079C0B21A
:1020000058749279D2B29A740122414B1A700B889B
:10201000404A1340934202D100223F4B1A6007F01E
:10202000C3FD21E3364B1B78002B11D0334A917846
:10203000C9B2344B1973D178C9B259731179C9B285
:1020400099735279D2B2DA730122314B1A702AE0B5
:10205000294B1B88DB0500D406E3274B1B885B0557
:1020600021D425490A888023DB0013430B80234AAF
:102070009078C0B2254BD874D078C0B2187510795A
:10208000C0B258755279D2B29A750122204B1A709B
:102090000B88204A1340934202D100221E4B1A6043
:1020A00001221E4B1A7007F07FFDDDE2124B1B88E8
:1020B000DB0700D5B6E01422174B1A60184B1B78CB
:1020C000002B64D00D4A10797F2318401549C87041
:1020D000907803400B80D3780888DB01C3189BB24B
:1020E0000B8053795B061FD50A00098880231B02E9
:1020F0000B4313801DE0C046680000201C02002036
:102100004902002074000020420000208C000020C2
:10211000440200200F0700004C0200203E01002076
:10212000400000207C010020B74A13885B045B0C50
:102130001380B6488279D200B34B9A6042799C688A
:102140003F210A40920212199A60C2799968520698
:10215000520F0A439A601B88AD4A128892B25B0400
:102160005B0C93425ED1AB4B1B885B045B0CAA4AB1
:1021700013800022A64B1A800132A84B1A70A8497E
:102180000B8813439BB20B80A64B1A704AE09F4A00
:1021900010797F2318409F49C870907803400B80C6
:1021A000D3780888DB01C3189BB20B8053795B0698
:1021B00006D50A00098880231B020B43138004E024
:1021C000944A13885B045B0C138090488279D20098
:1021D000904B9A6042799C683F210A409202121902
:1021E0009A60C27999685206520F0A439A601B8816
:1021F000874A128892B25B045B0C934212D1854BE2
:102200001B885B045B0C844A13800022804B1A807D
:102210000132824B1A7082490B8813439BB20B80A8
:10222000804B1A7007F0C0FC1EE2784A10797F23B9
:1022300018407549C870907803400B80D37808889F
:10224000DB01C3189BB20B8053795B0606D50A00ED
:10225000098880231B020B43138004E06A4A138819
:102260005B045B0C138069488279D200664B9A60EC
:1022700042799C683F210A40920212199A60C27901
:1022800099685206520F0A439A600122654B1A70F0
:1022900007F08AFCE8E15D4B9B78DBB2152B00D997
:1022A000C2E19B00604AD3589F46604B1B78002BCD
:1022B00000D0B9E1554B1A79D2B25D490A70DA788B
:1022C000D2B25C490A70D978012001405A4A117093
:1022D000DA78920801214A40024058490A70DA78B7
:1022E00008231340564A13709EE1484AD178137967
:1022F0005279DB01920313430B439BB29AB25149CB
:102300008A4203D11022504B1A7010E000204E492F
:1023100008704E490978092909D04D4909780129E1
:1023200002D04C4B1A8002E0DBB24B4A13700123FF
:102330004A4A13704A4A1370444B1B78DBB20F2B86
:1023400042D89B00474AD3589F460123464A137000
:10235000464A137002223C4B1A7041E00122424B64
:102360001A703C490B881B024148438000230B80B4
:10237000354B1A7034E0374A11883D4B5B880B436C
:1023800013802DE00122384B1A703A4A138801332A
:102390009BB2138002222C4B1A7021E00122324B97
:1023A0001A700132284B1A701AE000222F4B1A7053
:1023B00001232D4A1370244A137011222D4B1A80C9
:1023C000013A224B1A700BE0284B1B78002B07D0E8
:1023D0000022264B1A700123234A13701A4A1370E5
:1023E0000123104A1370244A13701DE1074BDB7858
:1023F000DBB2224A13701378DBB2214A1370012238
:10240000084B1A7010E1C0467C0100201C0200201D
:102410003C0100208C000020F40100202E0100204F
:102420006800002044020020F8A300003C020020C5
:1024300041010020B80100203D02002023010020BE
:1024400030010020FFFF0000F70100205C000020A9
:1024500033010020360100205D00002079010020BA
:10246000A001002050A40000F90000202601002057
:102470000C000020300200206F0100206E010020BF
:1024800025010020794AD178C9B2794B19601179B8
:102490001868C901014319605279196892030A4307
:1024A0001A60744B1B68002B50D0734B1B78002BA9
:1024B0004CD1724B5B796E4A11689A009B1A0F33AC
:1024C00001229A4011420ED00A226B4B1A706B4BBC
:1024D0001A8964214A436A490A6000221A751A71EE
:1024E0000132684B1A70654B5B79614A11689A003A
:1024F0009B1A0E3301229A4011420ED00A225E4BE3
:102500001A705E4B5A8964214A435D490A60012270
:102510001A75002119715B4B1A70584B5B79544A3C
:1025200011689A009B1A0D3301229A4011420DD076
:102530000A22514B1A70514A938964214B435049E6
:102540000B6001214F4B1970002313714E4B1B7808
:102550000D2B69D14D4B1B78022B65D101224C4BC1
:102560001A7061E04149CA784A4B1A800A79198881
:10257000D2010A431A801A8891008A1892B21A80EE
:102580001B88DBB2444A13700122414B1A704BE0A6
:10259000364B5B79032B03D10122404B1A7006E0C6
:1025A000324B5B79012B02D100223C4B1A70012285
:1025B000374B1A7038E02D4AD178C9B2384B1960C0
:1025C00011791868C90101431960517918688903A4
:1025D0000143196091791868490501431960D2795E
:1025E000196812070A431A600122294B1A701BE06E
:1025F0001E4AD178C9B22A4B196011791868C901ED
:102600000143196051791868890301431960917970
:102610001868490501431960D279196812070A43FD
:102620001A6001221A4B1A7007F0BEFA1CE007F07C
:10263000BBFA19E0A022D20580235B0059241620A2
:102640008821D450D050D150D558002DF9D0012236
:10265000A023DB059A600122124B1A70F432FF327C
:10266000114B1A8007F0A0FAF8BDC0461C020020EA
:102670003802002060000020F3010020000200204A
:1026800028010020B6010020240100203301002091
:1026900044020020A4010020A10100202D020020FE
:1026A0006801002019020020B4010020F8B55F463F
:1026B00056464D464446F0B4A022D20580235B0026
:1026C000592516208821D550D050D150D658002EEB
:1026D000F9D0994A116804230B431360974B1100FA
:1026E000102202E0013B002B02D0C8680242F9D060
:1026F000914B07221A611A6A802149020A431A6221
:10270000196805220A431A608D4A1A628B4B8A485F
:10271000152102E0013B002B03D0C2680A40152AB4
:10272000F8D1854A1A231361864B936000235361C5
:10273000A022D20580214903D160D360824A834917
:102740000A6083490A603221824A1160824F8349BC
:102750003960834A83481060834E84483060844DDA
:10276000296084480160FF21B96040279760D760E5
:10277000B360A9600F338360A022D205F1335925DD
:1027800016207739D550D050D150D658002EF9D0D8
:10279000794B1A6801210A431A600022DA60F82096
:1027A000400258609A601961BFF36F8F1A69002A5E
:1027B000FCD1714B9A68714B1A601B685B3300D077
:1027C000EEE0F820400200216B4A002601239C46DF
:1027D0006A4D6B4FD6605060966063461361BFF3DD
:1027E0006F8F1369002BFCD193682B602B68DBB2D1
:1027F0007B54013104302529ECD15F4B0022DA6093
:10280000604959609A6001321A61BFF36F8F1A698B
:10281000002AFCD1584B9A6858490A600A6892B25B
:10282000594802800A68120CD2B282700A68120EED
:10283000C2700022DA60554959609A6001321A610B
:10284000BFF36F8F1A69002AFCD14B4B99684E4A2F
:1028500011610022DA604E4959609A6001321A61B2
:10286000BFF36F8F1A69002AFCD1434B9968434A22
:102870001160116889B2444801811268120C4281CA
:102880000022DA60434959609A6001321A61BFF34D
:102890006F8F1A69002AFCD1374B9B68374A136047
:1028A00013689BB238498B8113681B0CDBB24B71E8
:1028B0001368DB0102D501228A7102E00022324B4B
:1028C0009A712E4B1B689B0103D501222E4B1A7562
:1028D00002E000222C4B1A75032252422948264B53
:1028E00000218C460F0001318A4624498846DF606A
:1028F00058609F6051461961BFF36F8F19690029B5
:10290000FCD199684546296029688946224989454C
:1029100004D95100214D66464E5307E01749096816
:1029200089B25500A9461D4D4E46715304300132FF
:102930000A2ADCD164E0C0460002005091D00300B6
:10294000174200003C10300080F0FA020000002026
:10295000040000200800002000400050FFFF00009D
:1029600040400050FF30000080400050FD55000006
:10297000C04000500041005000C00050A80100209D
:10298000A800002094F001000002002098F001004F
:102990009CF00100A0F00100FF3F00004800002073
:1029A000944B2222DA60F82252025A6001221A6104
:1029B000BFF36F8F1A69002AFCD1F8204002002172
:1029C0008D4B98468D4E8E4D8A4A21239C46203B46
:1029D00099464346CB5C7354735C013BFF3B2B60D1
:1029E0002B686746D760506093604B461361BFF316
:1029F0006F8F1369002BFCD1013104302929E8D1F4
:102A0000804B1B889BB2002B05D07E4B1B889BB252
:102A10007D4A93420CD97B4B0021002219809A7089
:102A2000DA7019611981598199815A719A711A75EF
:102A3000704B0022DA60754959609A6001321A6160
:102A4000BFF36F8F1A69002AFCD16A4A93687049F4
:102A50000B600B689B029B0A0B60136801218B4380
:102A60001360664B9A7AD2B26A490A705A7AD2B225
:102A7000694802701B7ADBB2684A13700B78DBB2CC
:102A80005A2B01D95A220A70634B1B78DBB25A2B9E
:102A900002D95A22604B1A70604B1B78DBB25A2B5A
:102AA00002D95A225D4B1A70544B5A7BD2B25C4900
:102AB0000A701A7BD2B25B480270DB7ADBB25A4AE8
:102AC00013700B78DBB25A2B01D95A220A70554B7E
:102AD0001B78DBB25A2B02D95A22524B1A70524B36
:102AE0001B78DBB25A2B02D95A224F4B1A70434B38
:102AF0001A7CD2B24D490A70DA7BD2B24C480270CD
:102B00009B7BDBB24B4A13700B78DBB25A2B01D99B
:102B10005A220A70464B1B78DBB25A2B02D95A2232
:102B2000434B1A70434B1B78DBB25A2B02D95A2203
:102B3000404B1A70314D00222423EA5429001431ED
:102B40003D4807F0AFFA6B79DBB23C4A137013785B
:102B5000DBB2032B02D90322384B1A70274A937930
:102B6000DBB237490B70537BDBB2002B02D0012B59
:102B700005D009E096221201324B1A8007E0962216
:102B8000D201304B1A8002E02F4A2E4B1A801B4A8A
:102B9000937852781B02D3181A0409D49BB22B4A9B
:102BA000138000222A4B1A80F532FF32294B1A80FB
:102BB000124BDB78DBB2022B13D0032B54D0012B4A
:102BC00007D00D4B3433244A13600022234B1A7074
:102BD00051E0234B4033204A136001221F4B1A70EF
:102BE00049E0204B4C331C4A136002221B4B1A70E5
:102BF00041E0C04600C000501CAE0000A80000200C
:102C0000A801002000020020FF270000FC0F100098
:102C100054020020F10100209C01002064000020EB
:102C2000FF01002078010020420200206201002004
:102C3000420100209A010020C4010020610100200F
:102C40009D010020AE01002000E1FFFF3C010020BB
:102C500068000020B4010020F80100209B01002042
:102C60001CB500001CBC0000EA4B5833EA4A136054
:102C70000322EA4B1A70A022D20580235B0059255B
:102C800016208821D550D050D150D658002EF9D0DA
:102C9000E34B802252001A600132FF321A60802218
:102CA000D2001A60DF4E8022D2043260DE490A6010
:102CB000DE480260DE4D2A60DE4D356078227260AB
:102CC000C22292009E58FF27BE43370040263E4353
:102CD0009E500D609626F6004E609E58D6493140B3
:102CE000C0263602314399500560D4494160985856
:102CF000D34901408020000401439950D14B1B6807
:102D0000002B60D10122D04B1A70E021C900A02312
:102D1000DB059963CD4B9868082101439960996858
:102D200080200001014399609968802000030143DD
:102D300099601968FF208143114319601968814324
:102D4000114319601868BC490140802040000143CC
:102D5000196059680725A943033D294359605968FB
:102D60007026B1430E004021314359605E68B84976
:102D700031408026F60031435960B6490978013167
:102D80001961B54909780131D961B449097801312E
:102D90009962C821D96099615962D96F1143D96785
:102DA000DE6F02213143D967D96F0D43DD67996822
:102DB0000A439A609A68104398609A688021490291
:102DC0000A439A6028E000229F4B1A708020C000BE
:102DD000A023DB0598639D4B996880221203114361
:102DE00099601A6894491140802252001143196079
:102DF0005A6897490A4002435A60964A127801324B
:102E00009A62C8225A62D96FC43A0A43DA679A684A
:102E1000802149020A439A6005F002F9904B1A6832
:102E2000904B1A601A000F2311680B42FCD104F07A
:102E30000DFC8D4D280004F08DFB8C4804F08AFBBE
:102E4000280004F087FB462004F0D6FE884D2800B9
:102E500004F080FB874804F07DFB280004F07AFB37
:102E6000462004F0C9FE844D280004F073FB83481B
:102E700004F070FB280004F06DFB462004F0BCFE5B
:102E80007F4D280004F066FB7E4804F063FB2800B9
:102E900004F060FB462004F0AFFE7B4D280004F0F8
:102EA00059FB7A4804F056FB280004F053FB4620F7
:102EB00004F0A2FE764D280004F04CFB754804F0A7
:102EC00049FB280004F046FB462004F095FE002153
:102ED000002004F017FB704804F03CFB02210020A6
:102EE00004F010FB6D4804F035FB00236C49FF2211
:102EF000CA540133092BFBD1FF266A4B1E70A02355
:102F0000DB059846F0231B0242465363664B674A33
:102F10001A6010229A601A68802189020A431A6096
:102F20000025634A15703E4A8021C9011160C327FC
:102F3000BF00D1598C46424960460140D1511E62C2
:102F4000196801220A431A6080235B004246D5506B
:102F5000FA20400004F050FE564D2900643107204D
:102F600004F01CFB29006C31062004F017FB29003B
:102F70007431052004F012FB4A4A1378DBB2FF2BB0
:102F8000FBD00121002004F0BDFA4B4804F0E2FA26
:102F9000444B18787F231840303004F0BFFAC82023
:102FA00004F02AFE0023454A13700A21444A117096
:102FB000444A13800939444A11702A4A1360013384
:102FC000984600239B46414B1B78002B01D104F00F
:102FD000B7F93F4E3188C9B2012004F001FD3188B4
:102FE0004904490E022004F0FBFC0022374B1A7002
:102FF00004F0A6F9CA5C002A03D000E00023DCB28A
:1030000002E00133112BF5D10A2C00D08FE000F043
:1030100055FCC0461CC30000F80100209B010020A5
:1030200000E100E0000001402000014000001140EC
:103030002000114000000168FF00FFFFC0D4010024
:10304000FFFF00FF8C4200502F01002000000440D1
:10305000FFF8FFFFF10100209C0100206400002028
:10306000540200205C010020F4CA000008CB0000DC
:103070001CCB000030CB000044CB000058CB00003C
:103080006CCB000080CB000094CB0000A8CB0000EC
:10309000BCCB0000D0CB0000C4010020E4CB00007A
:1030A000E8000020E4000020000003404204040087
:1030B0002D0100201CCA0000F4CB0000DA01002022
:1030C0002401002064010020AC0100202E0100201A
:1030D0008C000020BB7A002B2BD0C34BDB7A002B5B
:1030E00027D0C24B20221A701A3A5A7004F004FA00
:1030F0000021062004F006FABD4804F02BFABD4A70
:103100001378002BFCD1A022D2050133FF335921C3
:103110008946162588204946D150D550D050D158DF
:103120000029F8D00122A023DB059A6001E0B14E0E
:10313000AD4F3378002BCDD1102C01D901F0CDFE4D
:10314000A300AD4AD3589F46AC4B1B78032B09D143
:10315000AB4B1B78002B05D10322AA4B1A702F32E0
:10316000A94B1A60A94B1B78002B00D191E0A84B0A
:103170009B78DBB2002B02D0032B2CD05AE0A54B5E
:103180001B885B040FD0A34B9A680123A340134212
:1031900004D0A0498A689A438A6075E09D498A688C
:1031A00013438B6070E09C4B1B889BB2032B6BD846
:1031B000994A13889900CB185B009BB2138013883F
:1031C0001B199BB2138013889BB21F2B5CD91F2243
:1031D000914B1A8058E08F4B1B885B040FD08D4BAE
:1031E0009A680123A340134204D08A498A689A430B
:1031F0008A6049E087498A6813438B6044E0864BC4
:103200001B889BB2854A93423ED8834A1388990013
:10321000CB185B009BB2138013881B199BB21380E1
:1032200013889BB28022120293422DD97C4A7A4B9A
:103230001A8029E0A3B2784A138013889BB2042B2A
:1032400002D90422744B1A80724B1B885B041BD07A
:10325000704B9968704B1A8892B2012393401942BF
:1032600009D06D4B198889B26A48836801228A4067
:103270009343836008E0684B198889B26548826887
:1032800001238B40134383600122664B1A7001F0C7
:1032900024FE654B1B78002B2DD0644B1B78002B34
:1032A00007D00023624A13805B4A13805F4B0022E1
:1032B0001A70594B1B889BB2CC2B17D8564A1388CF
:1032C0009900CB185B009BB2138013881B199BB22B
:1032D000138013889BB2FF22D200934201D94E4B38
:1032E0001A804D4B1B889BB2514A138001224D4BD3
:1032F0001A7001F0F2FD4F4B1B78DBB2012B1FD08F
:10330000002B03D0022B30D001F0E7FD404B1B888F
:103310005B0401D101F0E1FD3D4B9A680123A3401C
:10332000134204D03A498A689A438A6003E03849D4
:103330008A6813438B6001223A4B1A7001F0CDFD6D
:103340005B465A1CD2B29346042B01D901F0C5FD4D
:10335000394908888300C3185B001B190B800121C1
:10336000304B1970934601F0B8FD244B1B78002BAD
:1033700000D098E06300314A9B5A9BB2002B00D1E9
:1033800091E063009B5A9BB22D490B802D4B1B880B
:103390009BB2138000232C4A1380962149002B4AAC
:1033A0001180254A1380234B00221A7001221D4BE5
:1033B0001A70274B1B7800229346002B73D0254BA5
:1033C0001B78DBB2012B4FD0032B5DD1224B1A7837
:1033D0000132224B1A61224A12780132DA61214A03
:1033E000127801329A625EE0440100203801002028
:1033F000ECCA0000DB00002090A40000F2010020D5
:103400001A020020320200201C010020310100209D
:103410008C0000207C01002030020020CB0C00003A
:103420000080FFFF44020020180200203A01002023
:10343000D6010020DA0100206401002048000020AD
:103440003C010020F401002068000020B4010020AD
:103450002F010020B2010020FF01002000000440E5
:103460007801002042020020B94B1A780132B94B92
:103470001A61B94A12780132DA61B84A1278013217
:103480009A6200239B460EE0B54B1A780132B14B8D
:103490001A61B44A12780132DA61B34A1278013201
:1034A0009A6200239B46B14B1B780A3BDAB2042A8E
:1034B00001D901F012FD9300AD4AD3589F46AD4BA0
:1034C0001B78032B26D1AC4B1B78DBB2012B02D02F
:1034D000022B0CD01EE0A94B1B78002B1AD0A84A57
:1034E00011888B00CB185B001B19138012E0A34BD3
:1034F0001B78002B0ED0A34B1A690123A340134263
:1035000004D0A0490A699A430A6103E09D490A6907
:1035100013430B619C4B1C7001229C4B1A7001F0F1
:10352000DCFC9B4B1B78DBB2062B01D901F0D5FCF0
:103530009B00984AD3589F46974B1B78002B01D18C
:1035400001F0CBFC954B1B78002B04D00022944B50
:103550001A80924B1A70924B1B889BB20422FF3246
:10356000934211D88E4A13889900CB185B009BB206
:10357000138013881B199BB2138013889BB2FF2BF7
:1035800002D9FF22864B1A800122804B1A7001F06B
:10359000A4FC844B1B78002B01D101F09EFC7F4BD7
:1035A0001B78002B04D000227D4B1A807B4B1A70B5
:1035B0007B4B1B889BB27C4A934211D8784A138874
:1035C0009900CB185B009BB2138013881B199BB228
:1035D000138013889BB2754A934201D9704B1A80AD
:1035E00001226A4B1A7001F078FC714B1B78002B9A
:1035F0000AD1A3B26F4A138013889BB2082B25D936
:1036000008226C4B1A8021E0644B1B78002B04D0FD
:103610000022634B1A80614B1A70614B1B889BB26E
:103620000422FF32934211D85D4A13889900CB18C7
:103630005B009BB2138013881B199BB21380138805
:103640009BB2FF2B02D9FF22554B1A8001224F4B10
:103650001A7001F042FC564B1B78002B22D14F4BC5
:103660001B78002B04D00022524B1A804B4B1A704F
:10367000504B1B889BB2504A934264D84D4A1388E2
:103680009900CB185B009BB2138013881B199BB267
:10369000138013889BB28022D200934253D9454BAA
:1036A0001A8050E03A4B1B78012B2AD1404B1B78F3
:1036B000012B13D1394B1B78002B04D00022384B3F
:1036C0001A80364B1A70A3B2354A138013889BB206
:1036D000072B38D90722324B1A8034E02F4B1B7846
:1036E000002B04D00023354A13702C4A1370334B3F
:1036F0001C701B78DBB2012B25D901222F4B1A70CD
:1037000021E0264B1B78002B04D00022244B1A808A
:10371000224B1A70224B1B889BB20422FF32934229
:1037200011D81F4A13889900CB185B009BB21380F5
:1037300013881B199BB2138013889BB2FF2B02D9ED
:10374000FF22174B1A800122104B1A7001F0C5FBA3
:103750006201002000000440420100209A01002084
:10376000F10100209C0100206400002024010020C1
:10377000D4A40000F201002034010020B101002097
:1037800064010020000200204001002044020020CB
:1037900033010020E8A40000790100206F0100201F
:1037A00036010020A001002005040000FF270000D2
:1037B0002601002030020020E70300005D00002009
:1037C000AA4B1B78002B04D00022A94B1A80A74BD0
:1037D0001A70A74B1B889BB2A64A934212D8A44AE0
:1037E00013889900CB185B009BB2138013881B19B8
:1037F0009BB2138013889BB28022D201934201D9DD
:103800009B4B1A8001229C4B1A7001F066FB9B4B6C
:103810001B78052B01D001F060FB994B1B78002B26
:1038200001D101F05AFB974B1B78032B01D001F01B
:1038300054FB954B1B78002B01D001F04EFB934BB2
:103840001B889BB2CC2B12D8904A13889900CB18B6
:103850005B009BB2138013881B199BB213801388E3
:103860009BB2FF22D200934201D9884B1A800122D9
:10387000814B1A7001F031FB062C1AD8A300844A40
:10388000D3589F460022834B1A7012E00122814BCD
:103890001A700EE002227F4B1A700AE000227E4B63
:1038A0001A7006E001227C4B1A7002E002227A4B69
:1038B0001A700122704B1A7001F00FFB774B1B78C6
:1038C000DBB2012B00D1C3E0002B03D0022B00D1CF
:1038D00004E121E2724B1B78002B33D0714B1B8823
:1038E0009BB27F2B07D96F4B1B889BB26E4A13800C
:1038F00001226E4B1A7000226A4B1A8001325E4B15
:103900001A706B490E0032206A4D00E01A000B68F5
:10391000002B02D0012B03D00AE03060130008E036
:10392000654B20221A7000225A70624B1B7805E00A
:1039300013002F78002F01D0002AE7D100225C4B22
:103940001A60E9E15D4B1B78002B27D05C4B1B789C
:10395000032B1BD15B4B1B889BB2524A13801388ED
:103960009BB2002B12D0584B1A78002AFCD14D4A3A
:103970001388013B9BB2138013885B009BB21380BA
:103980000122524B1A7002324F4B1A7001223A4BED
:103990001A70484B1A78002AFCD1BDE10123444E2D
:1039A0003000282100E013003268012A12D0002ADA
:1039B00002D00F2A03D03CE001601A003CE0444AE8
:1039C000D27A002A37D13C4B20321A7000225A702A
:1039D00003F0BDFC2022384B1A703D4BDB7A002BE4
:1039E00022D01A3A344B5A7003F086FD002106208B
:1039F00003F088FD374803F0ADFD2E4B1A78002AFE
:103A0000FCD1A022D20580235B00592616208821F4
:103A1000D650D050D150D758002FF9D00122A02332
:103A2000DB059A6003F093FC0022234B5A7003F0ED
:103A30008EFC1A0000E01A001E4D2F78002F01D0D6
:103A4000002BB0D10023224A9372194A136063E11C
:103A50000022214B1A80114B1A700122064B1A705A
:103A6000144A1378002BFCD19B4655E16F010020CE
:103A700036010020660600004402002033010020C9
:103A800034010020F2010020DC000020A20100200F
:103A900004A500002C01002022010020DA010020F2
:103AA00031010020300200206C010020C201002002
:103AB0005C010020DB0000203801002018020020FB
:103AC000B2010020D6010020460200203A01002069
:103AD00044010020ECCA0000640100200122D44B04
:103AE0001A7000230022D3490B80D3490B80D3499D
:103AF0000A70D3490A70D34A1380D34B1B78DBB2C8
:103B0000D24A1370D24B1B78D24A13800C2100206A
:103B100003F0E8FCD04B1B789A08012353400122A4
:103B20001340CE4A1370CE4B1B78002B00D1E9E036
:103B3000CB4B1B78032B0BD1CA4B1B88002B07D018
:103B40000022C84B1A80C64A13780133DBB21370C7
:103B5000C54B1B78092B08D1C44B1B780D2B04D106
:103B60001022C349C34806F0A5FABF4B1B78022BAD
:103B700008D1BE4B1B780A2B04D10B22BC49BE488E
:103B800006F098FAB84B1B78042B00D0B4E0B74B82
:103B90001B780A2B00D0AFE0B14B1B78022B00D072
:103BA000AAE0B64B1B78002B00D1A5E0A022D205DD
:103BB00080235B00592616208821D650D050D15042
:103BC000D758002FF9D0AE4B1A6801210A431A606A
:103BD0002222DA60F82252025A601961BFF36F8F15
:103BE0001A69002AFCD1A749CB788A7809881B0674
:103BF00012049B18CB18A24A2121D160A24951601E
:103C0000936001231361BFF36F8F13001A69002AB9
:103C1000FCD19C4B1A699A4B2121D9609B49596070
:103C20009A6001221A61BFF36F8F1A69002AFCD1D2
:103C3000944B5A891B89924B2122DA60944A5A602C
:103C4000944A9A6001221A61BFF36F8F1A69002AA1
:103C5000FCD18C4B9A791A7D5A799B89884B212209
:103C6000DA608D4A5A600A229A60093A1A61BFF3F3
:103C70006F8F1A69002AFCD1F8214902874D804BC9
:103C800021270126A85C0138FF38DF605960986061
:103C90001E61BFF36F8F18690028FCD10132043117
:103CA000252AEFD17E49243A7E4D754B21270126E6
:103CB0005000405B80B2DF60596098601E61BFF3C6
:103CC0006F8F18690028FCD1013204310A2AEFD124
:103CD0006B4A136801218B4313600023802252003A
:103CE000A021C9058B50654A1370664AD378DBB2B0
:103CF000137102226C4B1A60594A1378013BDBB2F4
:103D0000137002E00022694B1A70694A1378002B85
:103D1000FCD10022674B9A72674B1B78002B01D1B4
:103D200001F0DBF8614B1B78002B01D001F0D5F8D6
:103D3000624B1B78DBB2012B10D0032B1DD1604BE3
:103D40001A7801325F4B1A615F4A12780132DA61E8
:103D50005E4A127801329A6201F0BFF85C4B1A7821
:103D60000132584B1A615B4A12780132DA615A4AC1
:103D7000127801329A6201F0B0F8584B1A78013289
:103D8000504B1A61564A12780132DA61554A12785C
:103D900001329A6201F0A1F8444B1B78002B1CD130
:103DA000514B1B78002B10D1504B1B881BB2002BA2
:103DB00005DA4E4A13885B045B0C138005E04B4A1E
:103DC000118880231B020B4313800022474BDA70BB
:103DD0000132174B1A7001F080F8344B1B78DBB2BC
:103DE000012B00D1CFE0002B04D0022B00D16BE1DE
:103DF00001F073F83E4B1B78002B00D193E00D4B84
:103E00001B889BB21F2B77D80A48018889B2374E8E
:103E1000B26801238B405340B36003889BB20F2BE1
:103E200002D90122334B1A700022024B1A8072E031
:103E300044020020300200203601002079010020D9
:103E4000A0010020A2010020250100206E01002019
:103E5000A1010020A4010020B801002023010020BE
:103E6000F201002064010020330100202401002021
:103E7000E0010020C4010020980000206A0000201A
:103E800000C000500002002094F0010098F00100F2
:103E90009CF001000A000A00A0F00100A800002028
:103EA000A4F001004800002060000020DA0100209A
:103EB000DB000020440100202F010020B20100207F
:103EC000FF01002000000440780100204202002091
:103ED00062010020420100209A010020F10100202F
:103EE0009C010020640000209D0100208C00002027
:103EF0003101002065000020D94B1B889BB27F2B2D
:103F000009D9D74B1A8880231B021343D54A138043
:103F10000122D54B1A700022D14B1A800132D34BAB
:103F20001A7000F0DAFFD24B1B78002B24D0D14B53
:103F30001B78032B1BD1D04B1B889BB2C84A138024
:103F400013889BB2002B12D0CC4B1A78002AFCD1DC
:103F5000C34A13885B009BB213801388013B9BB25A
:103F600013800122C64B1A700232C44B1A70012210
:103F7000BE4B1A7000F0B1FFC24B20221A701D3ADE
:103F80005A7000F0AAFFC04B1B88002B00D18BE0B9
:103F9000BE4A1278002A39D0BD4A12885204520C07
:103FA0009A4212D1BA4B9B7EDB0705D5B84A937E65
:103FB00001218B43937604E0B54A917E01230B43A4
:103FC00093760022B14B1A7019E0B24A128892B26D
:103FD000B1490A80B14A13800022B14B1A802D32B8
:103FE000FF32B04B1A800121002003F08BFAAE485B
:103FF00003F0B0FA04F014F80122AC4B1A7000225E
:10400000A14B1A800132994B1A7046E0A04A1288DF
:104010005204520C934226D19D4A927ED20705D576
:104020009B498A7E012082438A7604E09849887EF3
:10403000012202438A769E4A128852040CD0944987
:104040008A7E012082438A760221984A1170934A1F
:1040500013800022924B1A8000228B4B1A8001326F
:10406000824B1A7019E08B4A128892B28A490A80F0
:104070008A4A138000238A4A138096214900894A7C
:104080001180814A13802C39FF39002003F03AFA5D
:10409000854803F05FFA03F0C3FF0022854B1A70D6
:1040A00000239B4600F019FF784B1B78002B03D0B0
:1040B0000022764B1A7002E00122744B1A70012222
:1040C0006A4B1A7000F009FF7B4B1B78DBB2032BA5
:1040D00004D8794A13780133DBB21370764B1B781E
:1040E000012B23D10122754B1A700023744A1370DF
:1040F000744A1370744A1370744B1B78DB0703D532
:1041000013780133DBB21370704B1B789B0704D517
:104110006D4A13780133DBB213706C4B1B785B076D
:1041200004D5694A13780133DBB21370624B1B78F4
:10413000DBB2012B01D800F076FD654B1B780A3B02
:10414000DAB2062A01D900F06EFD9300614AD35815
:104150009F465B4B1B78DBB2062B01D900F063FD59
:104160009B005D4AD3589F4601225C4B1A70524B0C
:104170001B78022B12D15A4F5A4E3900300005F0ED
:1041800091FF3A000C3A11884904490C731F1980B9
:10419000118B89B259825279D2B21A71464B1B786F
:1041A000032B01D000F03FFD0023434A13704B4A1C
:1041B00013704D4A1370374A128892B236490A80FA
:1041C0004A4A128892B235490A803A4A1370344AF0
:1041D0001380FA225200334B1A800121002003F091
:1041E00091F9314803F0B6F903F01AFF404B1B7800
:1041F000002B01D100F017FD1E4B1B78DBB2012B09
:1042000010D0032B1DD13B4B1A7801323A4B1A6167
:104210003A4A12780132DA61394A127801329A62E6
:1042200000F001FD374B1A780132334B1A61364AE0
:1042300012780132DA61354A127801329A6200F05E
:10424000F2FC334B1A7801322B4B1A61314A127847
:104250000132DA61304A127801329A6200F0E3FCEE
:10426000300200206C010020C20100204402002026
:1042700018020020B2010020D601002046020020D2
:104280003A01002038010020640100204000002095
:104290008C000020F4010020480000203C01002098
:1042A00068000020B401002000CC00002E02002095
:1042B0007C010020DA010020F201002070010020C2
:1042C00033010020340100209F0100204101002023
:1042D0002401002020A500003CA500004902002088
:1042E0009800002079000020420000207400002087
:1042F0002F010020FF010020000004407801002071
:104300004202002062010020420100209A010020A8
:10431000F10100209C01002064000020DE4B1B788E
:10432000032B01D000F07FFC023BDC4A1370DA4A19
:104330001370DB4A138802218B43138000F073FC57
:10434000D54B1B78022B0ED1D64E0B223100D6480E
:1043500005F0B0FE0022D54B1A703378DBB2D44A98
:10436000137000F060FC0222CB4B1A70CF4A137816
:10437000DBB2591CC9B21170CD480178C9B2CD4E1B
:10438000F31819731378F3181B7BDBB203701378DF
:10439000DBB20A2B01D800F046FC1126C14B9A462D
:1043A000C14DC54F10225146280005F083FE04235D
:1043B0003B700122B84B1A700C21002003F092F8D8
:1043C000013E002EEED10022B84B1A7000F02BFCFB
:1043D000B14B1B78032B01D000F025FCB74B1B78A9
:1043E000B74A128892B25B00B6495A52A022D2054F
:1043F00080235B00592616208821D650D050D150FA
:10440000D758002FF9D0B04B1A6801210A431A601F
:10441000AA4A1278AD488446624492000020D860CF
:104420005A6098601961BFF36F8F1A69002AFCD136
:10443000A54B9A68A64B1A601E68A0480378A1494C
:104440005B005A5A03785B005B5A9BB232409A4237
:104450001AD103785B009B4A9B5A9BB29C4A13601B
:1044600003789A498C4663449B001168964A212040
:10447000D0605360916001231361BFF36F8F13000D
:104480001A69002AFCD148E0A022D20580235B00F3
:10449000592616208821D650D050D150D758002FF9
:1044A000F9D0894B1A6801210A431A602222DA6086
:1044B000F82252025A601961BFF36F8F1A69002AFD
:1044C000FCD1F8214902834D7F4B21270126A85CAE
:1044D0000138FF38DF60596098601E61BFF36F8F4D
:1044E00018690028FCD101320431292AEFD17A4918
:1044F000283A744D744B212701265000405B80B24E
:10450000DF60596098601E61BFF36F8F18690028E3
:10451000FCD1013204310A2AEFD16B490B68012228
:1045200093430B60002380214900A020C005435025
:104530006A490B706A490A70574A137073E3564B05
:104540001B78042B66D1594B1B78DBB2062B61D844
:104550009B00644AD3589F46634B1B78002B09D1BC
:10456000624A1360624A1370624A13710122624BFD
:104570001A7029E05F4B1B889BB2002B1AD14D4962
:104580000A885204520C5B4B1A800A79D2B29A7094
:104590000A795208DA7000221A610A2119815981B8
:1045A00099815A719A711A750939544B19704F4B88
:1045B0001A6002E002224D4B1A604E4AD378DBB2F9
:1045C000137101224C4B1A700222334B1A70013ABC
:1045D000434B1A701EE0444B1B78002B09D0354B1F
:1045E0001B885B045B0C434A1380454B1B78D370DC
:1045F00013713D4B1B78002B02D001223F4B1A70E8
:104600000222254B1A70013A354B1A7002E0022241
:10461000214B1A70204B1B78DBB2042B00D802E32D
:1046200004221D4B1A70FEE21B4B1B78032B00D09B
:10463000F9E2344B1B78002B03D00122324B1A7065
:1046400002E00122314B1A702E4A11784B424B4145
:10465000DBB213700122224B1A700F4A1378013B10
:10466000DBB21370DFE20C4B1B78032B00D0DAE2D5
:10467000023B274A1370084A13700022174B1A7026
:10468000D1E2244B1B78DBB2062B00D9CBE29B0096
:10469000214AD3589F46C046F20100203201002033
:1046A0006800002098000020E00100203401002074
:1046B000660000208C0000205002002040010020F5
:1046C000F40100204800002000C00050287C0000B9
:1046D000A8010020A8000020A4F00100DA010020B9
:1046E0004402002058A50000B10100206000002015
:1046F000DE00002000020020B60100206A00002039
:1047000064010020200100208900002045020020D3
:10471000700000203301002074A50000CD4B1B78F1
:10472000002B04D0CB4A1378013BDBB21370CA4B89
:104730001B78032B00D076E2C84B1B889BB2002B62
:1047400002D1C64B42461A800122C54B1A70C14B9A
:104750001B78002B04D0C24A13780133DBB21370EC
:104760000122C04B1A700132BB4B1A700022BE4BA3
:104770001A70BA4B1B889BB2984654E2BB4B1B780D
:10478000002B0BD10133B74A13700021B14A1170CD
:10479000B24A1380B24B01221A7044E20223B04A9B
:1047A0001370B34A13700122AA490A70AB490A80F8
:1047B0000021AE4A1170A84A1370AA4B01221A7048
:1047C00031E2AC4B1B78002B0ED10133A54A13709C
:1047D0000021A04A11701131A04A1180A04A137023
:1047E0001022A34B1A701EE202229D4B1A700A215E
:1047F0009F4B1970012397490B701120974908802E
:1048000000209C49087094490A70964A13700AE285
:10481000914B1B78032B00D005E20122904B1A70BC
:104820008C4B1B78002B04D08D4A13780133DBB2FC
:10483000137001238C4A13708A4A13700222864B2C
:104840001A70F0E1844B1B78032B00D0EBE10122BE
:10485000894B1A700132804B1A70E4E17E4B1B7851
:10486000032B00D0DFE10122844B1A7001327A4B16
:104870001A70D8E1784B1B78032B00D0D3E10122CA
:104880007F4B1A700132744B1A70CCE17D4B1B7850
:10489000DBB20A2B00D9C6E19B007B4AD3589F4666
:1048A0006D4B1B78032B00D0BDE1784B1978C9B252
:1048B000052003F095F80122674B1A70B3E1664BAF
:1048C0001B78032B00D0AEE1714B1978C9B20620DA
:1048D00003F086F80122604B1A70A4E15E4B1B784E
:1048E000DBB2022B02D0042B04D09CE10122694BE5
:1048F0001A7098E10223584A1370664A137092E1C5
:10490000554B1B78022B02D10122634B1A70524B7C
:104910001B78042B00D086E1604B1B78002B03D062
:1049200002225D4B1A7002E002225D4B1A700222D5
:10493000494B1A7077E1484B1B78022B00D072E18B
:104940000122584B1A706EE1434B1B78022B0FD19A
:10495000524B1B78002B05D00023534A1380534A37
:10496000138002E0524A504B1A800122514B1A70B8
:10497000394B1B78042B00D055E1484B1B78002B9A
:104980002CD04D4B1B78002B0ED04C4B1B78002BA2
:1049900003D00022494B1A7002E00122474B1A70E3
:1049A0000222444B1A7015E0404B1B889BB2002B2F
:1049B00004D13E4A138801339BB213803B4A1388CB
:1049C000013B5B009BB238490B800023138001221E
:1049D000384B1A700322204B1A7024E10223354A07
:1049E00013701D4A13701EE11B4B1B78032B00D064
:1049F00019E102222A4B1A70013A174B1A7012E180
:104A0000154B1B78032B00D00DE10222244B1A70AA
:104A1000013A114B1A7006E10F4B1B78032B00D0A3
:104A200001E1274B1B78DBB2012B0AD0002B04D00D
:104A3000022B0AD0032B47D049E00022214B1A70E9
:104A400045E001221F4B1A7041E003221D4B1A70F2
:104A50003DE0C04626010020F20100203002002087
:104A6000F7010020F90000203F010020790100201B
:104A70005C000020A0010020D8010020DC01002003
:104A80003E0200203301002090A5000061010020BB
:104A90009D0100204002002043020020340100203C
:104AA0003C020020B701002098010020A201002054
:104AB000FF3F0000DD000020DC0000202D02002070
:104AC0009F010020410100200722CF4B1A700222D3
:104AD000CE4B1A70013ACE4B1A70A4E0CC4B1B7827
:104AE000022B0DD1CB4E11223100CB4805F0E2FA5A
:104AF0000022CA4B1A703378DBB2C94A137092E0B5
:104B00000222C34B1A70C54B1A78D2B2511CC9B2DB
:104B10001970C3480178C9B2BE4EB1541A78D2B2E6
:104B2000B25CD2B202701B78DBB20F2B7BD9142699
:104B3000B84FB94B9A46B64D10223900504605F091
:104B4000B9FA3300143BF95CC9B2F0B202F048FF85
:104B500001232B700C21002002F0C4FC0136252E0D
:104B6000EAD10022AD4B1A705DE0A94B1B78032BF4
:104B700059D1AC4E3178C9B2032002F031FF3378FD
:104B8000DBB2022B0DD0032B10D0012B04D0A64B8F
:104B90003433A64A13600DE0A54B4033A34A13609B
:104BA00008E0A44B4C33A14A136003E0A24B5833F6
:104BB0009E4A13600122964B1A7034E0A022D2055F
:104BC00080235B00592416208821D450D050D15026
:104BD000D558002DF9D0994B1A6801210A431A6063
:104BE0002222DA60F92252025A601961BFF36F8FF4
:104BF0001A69002AFCD1914B2132DA60F922520263
:104C00005A608F4A9A6001221A61BFF36F8F1A6946
:104C1000002AFCD1894A116803230B431360894A97
:104C2000894B1A60FEE70122884B1A7055E1002378
:104C3000874A1360874A1380874B1B78002B03D168
:104C4000864B1B78002B07D00023834A1370834ABE
:104C500013700122824B1A70814B1B78DBB2002B40
:104C600002D0012B09D038E100227E4B1A800123AB
:104C7000764A13707A4A13702FE17B4B1B889BB2E4
:104C8000002B0CD0774B1B78774AD370D3781279EE
:104C9000DBB2934203D9744A1379DBB2D37000229A
:104CA000704B1A800132694B1A706D4B00221A70DA
:104CB00013E16B4B1B78002B18D16B4B1B889BB2FD
:104CC000002B13D00022654B1A70634B1B78002B0E
:104CD00005D00023604A1370644A138002E0012269
:104CE0005D4B1A700122594B1A70F6E05C4B1B7831
:104CF000022B00D0F1E05E4B1B780D2B00D0ECE0D6
:104D00005C4B1B78002B06D000225A4B1A700332E2
:104D1000594B1A70E1E00122564B1A700532564B7E
:104D20001A70DAE04E4B1B78002B00D0D5E0002241
:104D3000494B1A70494B1B78002B0ED04B4B1B88EC
:104D40009BB2002B05D00023484A13804B4A1380A6
:104D500006E00022414B1A7002E001223F4B1A701C
:104D600001223A4B1A70B8E00023454A1360012132
:104D7000364A1170384A1370394B1B78002B00D11A
:104D80009AE0374B1B78012B05D13E4A11784B42F4
:104D90004B41DBB213700022314B1A703A4B1B7837
:104DA000002B00D199E0394B1B78DBB2012B0FD0DF
:104DB000032B1BD1364B1A780132364B1A61364A17
:104DC00012780132DA61354A127801329A6284E04F
:104DD000334B1A7801322F4B1A61324A1278013262
:104DE000DA61314A127801329A6276E02F4B1A78F2
:104DF0000132284B1A612E4A12780132DA612D4AAB
:104E0000127801329A6268E0410100203C020020E1
:104E1000F2010020C4010020E00100203401002044
:104E2000660000209B0100201CAE0000F80100205D
:104E30001CB500001CBC00001CC3000000C00050DA
:104E40005AA55AA50400FA050CED00E04402002022
:104E50004C0200203C0100203101002018020020FB
:104E6000DA010020640100208C00002030020020C4
:104E7000240100201A02002032020020D601002066
:104E800074010020B00100202F010020B201002099
:104E9000FF010020000004407801002042020020B1
:104EA00062010020420100209A010020F10100204F
:104EB0009C01002064000020D24B1B78002B05D001
:104EC000D14B46221A61453ADA619A620222CF4BEF
:104ED0001A70013ACE4B1A70FFE70023CD49002229
:104EE000CA540133112BFBD1CB4B1B78002B01D1C2
:104EF000FEF769F80022C84B1A70C44B1B78DBB26E
:104F0000012B00D1B6E1002B04D0022B00D1D5E15A
:104F1000FEF759F8C14B1B78002B00D12AE1C04B9A
:104F20001B885B0400D025E1BE4C20884004400C67
:104F300002F01CFBBC4802F00DFBBC4B188880B291
:104F400002F014FBBA4802F005FB00210C2002F02D
:104F5000D9FAE178032002F00BFD23881BB2002B65
:104F600003DA7E2002F0DAFA02E07F2002F0D6FABD
:104F70000121002002F0C6FAAA4B9B78DBB2002B7D
:104F800003D0032B01D0042400E020240025A54FEA
:104F9000A84EBA680123AB401A422ED0A54B5B5DE8
:104FA000073BDAB2462A03D89300A34AD3589F4658
:104FB0000A21280005F054F83031C8B202F0AEFAE8
:104FC0004DE02A2002F0AAFA49E0132002F0A6FAE6
:104FD00045E0052002F0A2FA41E00C2002F09EFA22
:104FE0003DE0B22002F09AFA39E0072002F096FA8A
:104FF00035E0F52002F092FA31E0735D073BDAB25A
:10500000462A03D893008D4AD3589F460A21280088
:1050100005F026F8002903D00D2002F07FFA1EE0EB
:105020002E2002F07BFA1AE0192002F077FA16E03F
:105030002D2002F073FA12E06F2002F06FFA0EE0FA
:105040005F2002F06BFA0AE0152002F067FA06E032
:105050004B2002F063FA02E07C2002F05FFA013597
:10506000052D96D16F4B9B78012B7ED06D4B9B7895
:10507000022B7AD06B4E6F4FB2680123AB401A42BD
:105080002DD07B5D073BDAB2462A03D893006C4AE9
:10509000D3589F460A21280004F0E2FF3031C8B2FD
:1050A00002F03CFA4EE0132002F038FA4AE0052004
:1050B00002F034FA46E02A2002F030FA42E00C20F6
:1050C00002F02CFA3EE0B22002F028FA3AE0072083
:1050D00002F024FA36E0F52002F020FA32E0554BD7
:1050E0005B5D073BDAB2462A03D89300554AD35892
:1050F0009F460A21280004F0B3FF002903D00D20A9
:1051000002F00CFA1EE02E2002F008FA1AE0192034
:1051100002F004FA16E02D2002F000FA12E06F20EF
:1051200002F0FCF90EE05F2002F0F8F90AE0152029
:1051300002F0F4F906E04B2002F0F0F902E07C20E6
:1051400002F0ECF90135202D96D1384B1B889BB22B
:105150007F2B01D8FDF737FF0221002002F0D2F9A2
:10516000394802F0F7F9FDF72EFF384802F0F2F95E
:10517000FDF729FF364B1B78002B3FD002F0BCF91E
:1051800034497C31002002F009FA334E311D0120F0
:1051900002F004FA31000C31022002F0FFF9310074
:1051A0001431032002F0FAF90021002002F0AAF9DC
:1051B000002002F0B3F9294802F0CCF9284B1888F6
:1051C00080B202F0D3F90121002002F09BF92548BA
:1051D00002F0C0F9012002F0A1F9234802F0BAF967
:1051E000032002F09BF9214802F0B4F9022002F0FA
:1051F00095F91F4802F0AEF9FDF7E5FE02F04CFF0D
:10520000FDF7E1FE2F01002000000440DA0100203C
:1052100070010020440100204402002031010020E0
:105220007C0100208C00002010CC00003002002007
:1052300018CC0000FC000020BCA50000D8A600008F
:10524000F4A7000010A9000020CC000034CC00001E
:10525000180200201CCA00009CCA000050CC0000AC
:10526000D601002058CC000044CC000060CC0000E7
:1052700064CC00000021002002F044F9E44B1B78CC
:10528000002B07D0E34802F065F90021072002F067
:1052900039F906E0E04802F05DF90021052002F04E
:1052A00031F9DE4B188802F061F90121002002F08B
:1052B00029F9DB4802F04EF9FDF785FE02F01CF9F2
:1052C000D84B1B78DBB2012B00D102E1002B09D0B7
:1052D000022B01D100F012FD032B01D101F03EFDA4
:1052E000FDF771FED0491C31002002F057F9012171
:1052F000002002F007F9002002F010F9CB4B1B78D8
:105300000A3BDAB2062A01D9FDF75DFE9300C84ACE
:10531000D3589F46C74B186802F01CF9C64B1B6850
:10532000002B0BD1C34B1868C44B9C46604402F061
:1053300011F9C822C04B1A60FDF745FEBE4B1B6831
:10534000012B01D0FDF73FFEBD4802F003F9BA4A38
:105350001368013B1360FDF736FEB64B1868113039
:1053600002F0F8F8B44B1B68002B0BD1B14B186856
:10537000B24B9C46604402F0EDF8C822AE4B1A6076
:10538000FDF721FEAC4B1B68012B01D0FDF71BFE86
:10539000AB4802F0DFF8A84A1368013B1360FDF741
:1053A00012FEA44B1868223002F0D4F8A24B1B68FE
:1053B000002B0BD19F4B1868A04B9C46604402F019
:1053C000C9F8C8229C4B1A60FDF7FDFD9A4B1B687B
:1053D000012B01D0FDF7F7FD994802F0BBF8964A82
:1053E0001368013B1360FDF7EEFD924B18683330F4
:1053F00002F0B0F8904B1B68002B0BD18D4B186856
:105400008E4B9C46604402F0A5F8C8228A4B1A6075
:10541000FDF7D9FD884B1B68012B01D0FDF7D3FDAB
:10542000874802F097F8844A1368013B1360FDF740
:10543000CAFD844B1B78002B05D0834B46221A6192
:10544000453ADA619A627B4B1868443002F082F880
:10545000794B1B68002B0BD1764B1868774B9C4619
:10546000604402F077F8C822734B1A60FDF7ABFD79
:10547000714B1B68012B01D0FDF7A5FD704802F0B0
:1054800069F86D4A1368013B1360FDF79CFD00222B
:10549000694B1A600021002002F034F8002002F06D
:1054A0003DF8644B1868553002F054F8674802F034
:1054B00051F8674802F04EF8664802F04BF8FDF7E5
:1054C00082FD00225C4B1A60634802F043F8FDF74E
:1054D0007AFD564B1B780A3BDAB2062A01D9FDF752
:1054E00072FD93005D4AD3589F464F491C310020FE
:1054F00002F054F80121002002F004F8002002F02C
:105500000DF8574B1B78DBB2FF2B10D1554B1B8886
:105510009BB2002B08D0534B1B8B9BB2002B03D0AC
:1055200006224F4B1A7002E005224D4B1A704C4B6D
:105530001B78DBB2062B3DD89B004B4AD3589F46C5
:105540003C4B1868494B9C46604402F003F8FDF759
:105550003AFD384B1868CC23DB009C46604401F0D0
:10556000F9FFFDF730FD424801F0F4FFFDF72BFD98
:105570003C4B1B889BB2002B1CD03A4B1B8B9BB225
:10558000002B17D02B4B1868993001F0E3FF012155
:105590000B2001F0B7FF334B19884904490C052053
:1055A00002F0E6F97F2001F0B9FF324801F0D2FFA6
:1055B000FDF709FD00222A4B1A701E4B1868663051
:1055C00001F0C8FFFDF7FFFC1A4B1868773001F0B7
:1055D000C1FF244E31884904490C052002F0C8F966
:1055E000254801F0B7FF33889BB2002B0AD01D4B32
:1055F0005B791801C3180F4A1068C01801F0AAFFA0
:10560000FDF7E1FC1D4801F0A5FFFDF7DCFCC046FD
:105610004000002070CC000080CC0000640100201D
:1056200090CC0000F20100209CCA00002401002060
:105630002CAA0000F8010020740100202E050000B3
:10564000A4CC00002F01002000000440B8CC0000D2
:1056500058020020E4CB0000C0CC000048AA0000A3
:10566000330100208C00002064AA00003F050000E8
:10567000C8CC0000D8CC0000C0CD000064CC000035
:10568000E84B1868883001F065FF01210B2001F01C
:1056900039FFE54E31884904490C052002F068F9CC
:1056A00030000C3001F056FFFDF78DFCDF491C3156
:1056B000002001F073FF0121002001F023FF0020F2
:1056C00001F02CFFDA4B1B78DBB2FF2B02D1062254
:1056D000D74B1A70D64B1B78DBB2062B03D89B0036
:1056E000D44AD3589F460022D14B1A70CD4B18682C
:1056F000AA3001F02FFFFDF766FCCA4B1868BB30DB
:1057000001F028FFFDF75FFCC64B1868CC3001F0B4
:1057100021FFFDF758FCC34B1868DD3001F01AFF7C
:10572000FDF751FCBF4B1868EE3001F013FFFDF799
:105730004AFCBC4B1868FF3001F00CFFBA4B9B7859
:10574000032B01D1FDF73FFCB64B186888239B0063
:105750009C46604401F0FEFEFDF735FCB14B186835
:105760001130FF3001F0F6FEAF4B9B78032B01D1D7
:10577000FDF729FCAB4B186888239B009C466044CE
:1057800001F0E8FEFDF71FFCA8491C31002001F0E4
:1057900005FF0121002001F0B5FE002001F0BEFE52
:1057A000A34B1B78002B02D00022A14B1A709D4BFB
:1057B00018682230FF3001F0CDFEFDF704FC9B4954
:1057C0001C31002001F0EAFE0121002001F09AFEC8
:1057D000002001F0A3FE964B1B78DBB2FF2B02D119
:1057E0000A22934B1A70924B1B78DBB20A2B03D818
:1057F0009B00914AD3589F4600228D4B1A70894EC8
:1058000030683330FF3001F0A5FE8C4B5B792133DB
:105810001801C3183068C01801F09CFEFDF7D3FBD7
:10582000804B18684430FF3001F094FE844B1B78A5
:10583000002B08D07B4B1868824B9C46604401F0DB
:1058400089FEFDF7C0FB774B18687F4B9C46604490
:1058500001F080FEFDF7B7FB724B18685530FF3042
:1058600001F078FEFDF7AFFB6E4E30686630FF301A
:1058700001F070FE3068754B9C46604401F06AFE92
:10588000FDF7A1FB674B18687730FF3001F062FE2F
:105890006F4B198889B2062002F06AF8FDF793FB76
:1058A000604E30688830FF3001F054FE3068674B3E
:1058B0009C46604401F04EFEFDF785FB594B18688D
:1058C0009930FF3001F046FE624B1B78002B04D06C
:1058D000614801F03FFEFDF776FB604801F03AFEBB
:1058E000FDF771FB4F4B1868AA30FF3001F032FE14
:1058F0005B4B1B78002B04D05A4801F02BFEFDF7C0
:1059000062FB594801F026FEFDF75DFB454E30680D
:10591000BB30FF3001F01EFE544B1B7838331801AA
:10592000C3183068C01801F015FEFDF74CFB3D4B65
:105930001868CC30FF3001F00DFE4D4E300001F004
:1059400009FE102231004B4804F0B4FBFDF73BFB8D
:10595000494B1B78DBB2022B23D0032B31D0012B18
:105960000FD0304E3368454A94466344180001F026
:10597000F1FD3068424B9C46604401F0EBFDFDF7C1
:1059800022FB284E33683F4A94466344180001F0D6
:10599000E1FD30683C4B9C46604401F0DBFDFDF7C7
:1059A00012FB204E3368394A94466344180001F0D4
:1059B000D1FD3068364B9C46604401F0CBFDFDF7CD
:1059C00002FB184E3368BB22D20094466344180091
:1059D00001F0C0FD30682F4B9C46604401F0BAFDD9
:1059E000FDF7F1FA11492431002001F0D7FD002123
:1059F000002001F087FD002001F090FD094B1868A0
:105A0000443001F0A7FD244B1B78002B00D129E185
:105A1000224B1B78DBB2012B57D0002B40D0022B3E
:105A200068D07BE0F80100208C0000209CCA0000B8
:105A30003301002080AA00009CAA0000A8000020DA
:105A40009D01002086020000750200009702000000
:105A5000AE01002030010020E4CC0000F8CC0000B2
:105A60003D0200200CCD000020CD00009F01002051
:105A7000C4010020E00100209B010020720500000D
:105A80009405000083050000A5050000B605000090
:105A9000C7050000E90500002F01002022010020B9
:105AA0000121052001F02EFDE34801F053FDE34BF9
:105AB0001A780132E24B1A61E24A12780132DA6155
:105AC000E14A127801329A6228E00121052001F0B2
:105AD00019FDDE4801F03EFDDD4B1A780132D84B4E
:105AE0001A61DC4A12780132DA61DB4A127801323B
:105AF0009A6213E00121052001F004FDD74801F06E
:105B000029FDD74B1A780132CD4B1A61D54A12784C
:105B10000132DA61D44A127801329A6201210120FD
:105B200001F0F0FCD14B1B78DBB2012B35D0002B00
:105B300003D0022B61D0FDF746FACD4B1B78DBB2C8
:105B4000012B0ED0002B02D0022B14D01CE0BB4E38
:105B5000307801F00BFD3178C9B20A2001F040FF26
:105B600012E0BB4E307801F001FD3178C9B20D2052
:105B700001F036FF08E0BA4E307801F0F7FC3178DA
:105B8000C9B2102001F02CFF0221002001F0BAFC64
:105B9000B84801F0DFFCFDF716FAB54B1B78DBB215
:105BA000012B0ED0002B02D0022B14D01CE0A54EEE
:105BB000307801F0DBFC3178C9B2092001F010FF28
:105BC00012E0A44E307801F0D1FC3178C9B20C203B
:105BD00001F006FF08E0A34E307801F0C7FC3178F1
:105BE000C9B20F2001F0FCFE0221002001F08AFC66
:105BF000A14801F0AFFCFDF7E6F99D4B1B78DBB245
:105C0000012B13D0002B02D0022B19D021E08E4E95
:105C1000307801F0ABFC964B1B783178C9B2580054
:105C2000C0180830C0B201F0DBFE12E08A4E3078B6
:105C300001F09CFC3178C9B20B2001F0D1FE08E0E4
:105C4000894E307801F092FC3178C9B20E2001F013
:105C5000C7FE0221002001F055FC884801F07AFCC3
:105C6000FDF7B1F9864801F075FC744E307801F00B
:105C70007DFC3178C9B20A2001F0B2FEFDF7A3F92C
:105C800080492431002001F089FC0021002001F02E
:105C900039FC7D4801F05EFC7C4B1868553001F002
:105CA00059FC7B4801F056FC7A4B186880B201F031
:105CB0005DFCFDF788F9734E31002431002001F0BE
:105CC0006DFC31001431042001F068FC002100203B
:105CD00001F018FC002001F021FC6F4801F03AFCB3
:105CE000674801F037FC042001F018FC6B4801F014
:105CF00031FC6B4801F02EFCFDF765F9694B1B7810
:105D00000A3BDAB2052A01D9FDF75DF99300664A2C
:105D1000D3589F465B492431002001F03FFC00210D
:105D2000002001F0EFFB002001F0F8FB5F4B1B7837
:105D3000DBB2FF2B02D103225C4B1A705B4B1B784A
:105D4000DBB2062B03D89B00594AD3589F4600224A
:105D5000564B1A704D4B1868663001F0FBFB002162
:105D60000B2001F0CFFB534B1B889BB2002B01D1C2
:105D7000FDF729F94F4E31884904490C052001F0FF
:105D8000F7FD4D4801F0E6FB701D01F0E3FB022139
:105D9000002001F0B7FB494801F0DCFB3379180122
:105DA000C3183A4A1068C01801F0D4FBFDF70BF98C
:105DB000364B1868773001F0CDFB414E31884904ED
:105DC000490C052001F0D4FD3E4801F0C3FB3388A7
:105DD0009BB2002B0AD03A4B5B791801C3182B4AAF
:105DE0001068C01801F0B6FBFDF7EDF8364801F079
:105DF000B1FBFDF7E8F8254B1868883001F0AAFBE5
:105E000000210B2001F07EFB2D4E31884904490C06
:105E1000052001F0ADFD0E21002001F063FB3000F4
:105E20000C3001F097FB294B1878C0B2012101F02A
:105E300069FBFDF7C8F8C04634CD0000F101002031
:105E4000000004409C0100206400002040CD0000C0
:105E5000FF01002078010020420200204CCD00000C
:105E600062010020420100209A0100202C01002044
:105E70002201002058CD000064CD000070CD00004C
:105E80004CCC00009CCA00006CCC0000F801002043
:105E90007CCD00005402002088CD000098CD000089
:105EA000A8CD000024010020C8AA00003301002072
:105EB000E0AA000074000020BCCD0000C4CD0000AA
:105EC0008C000020C0CD000064CC00003401002014
:105ED000DA4B1868DA4B9C46604401F03BFB00212A
:105EE0000A2001F00FFBD74801F034FBD64B1B789A
:105EF000002B04D1D44A13780133DBB21370D24B98
:105F0000187801F033FB0121002001F0FBFACB4EA1
:105F10003368AA22D20094466344180001F01AFBA9
:105F20003068CA4B9C46604401F014FBFDF74BF807
:105F3000C24B1868CC23DB009C46604401F00AFB8E
:105F4000C34B1B78DBB2062B03D89B00C14AD35846
:105F50009F460022BE4B1A70B84B1868BE4B9C4639
:105F6000604401F0F7FABD4801F0F4FABC4B1B782D
:105F7000002B08D0B14B1868BA4B9C46604401F026
:105F8000E9FAFDF720F8AD4B1868B74B9C46604422
:105F900001F0E0FAFDF717F8A84B1868B34B9C46E0
:105FA000604401F0D7FAB24BDB78B24E3380AB4895
:105FB00001F0D0FA308801F0D9FAFDF704F89F4BD0
:105FC0001868AD4B9C46604401F0C4FA02210020E1
:105FD00001F098FA0026A64B994601274B461A690C
:105FE0003B00B3401A4203D02A2001F097FA02E0A6
:105FF0000D2001F093FA01360A2EEFD1FCF7E3FFF2
:106000008E4B18689D4B9C46604401F0A3FA022118
:10601000002001F077FA964B5B79DBB2042B02D9B2
:106020000422934B5A71924B5E79F6B2944801F078
:1060300091FA7300F6180136300001F097FA914892
:1060400001F088FAB01C80B201F090FAFCF7BBFFB7
:106050007A4B18688C4B9C46604401F07BFA7C4E6E
:1060600030782D30C0B201F059FA0221002001F041
:1060700049FA834801F06EFA33785B007C4A9B5AF8
:106080009BB2002B07D1724B1A7879495200535AB0
:1060900001339BB253526E4B1B785B00744A985A83
:1060A00080B201F063FA794801F054FAFCF78BFFF3
:1060B000774801F04FFA774801F04CFA764B9B781D
:1060C000012B14D0744B9B78022B10D0734B1B7890
:1060D000DBB2802B02D91C22704B1A706F4B1B78DD
:1060E000DBB21C2B13D900226C4B1A700FE06B4BE8
:1060F0001B78DBB2802B02D90422684B1A70674BE5
:106100001B78DBB2042B02D90022644B1A70634B5C
:10611000187801F02BFA4B4801F01CFA01210620F7
:1061200001F0F0F95E4B1B78DBB2802B02D909221B
:106130005B4B1A705A4B1B78DBB24D2B03D89B007C
:10614000584AD3589F460022554B1A700D2001F033
:10615000E5F91AE06F2001F0E1F916E0192001F0ED
:10616000DDF912E02D2001F0D9F90EE0152001F043
:10617000D5F90AE05F2001F0D1F906E04B2001F0EB
:10618000CDF902E07C2001F0C9F90E21002001F0D8
:10619000A9F9454B1B78002B05D00121062001F001
:1061A000B1F9FCF710FF0121022001F0ABF9FCF777
:1061B0000AFF224B1868993001F0CCF9364B1B8846
:1061C0009BB2002B01D1FCF7FEFE01210B2001F058
:1061D00099F9314B19884904490C052001F0C8FB95
:1061E0000121002001F08EF930492431012001F015
:1061F000D5F9012001F092F92D4801F0ABF9FCF737
:10620000E2FE2A492431002001F0C8F900210020D3
:1062100001F078F9002001F081F9264B1B78DBB200
:10622000FF2B02D10622234B1A70224B1B78DBB2C4
:10623000062B43D89B00204AD3589F46F8010020E4
:106240003F05000054CC0000400100206105000023
:1062500034010020FCAA00007106000068CC000098
:10626000B1010020C6060000D7060000820600002B
:10627000000200206401002093060000A406000034
:106280004CCC0000CCCD0000B5060000D0CD000005
:10629000C8CC0000D8CD00008C00002048020020AF
:1062A0009E01002018AB0000200100209CCA0000C5
:1062B000D8CC00003301002050AC00000022D34BAA
:1062C0001A70D34B1868AA3001F044F9D14B1B88DF
:1062D0009BB2002B04D10121042001F049FB05E011
:1062E000CC4B198889B2042001F042FBCA4801F066
:1062F00031F9CA4B1B889BB2FF2B06D8C74B1988B4
:1063000089B2032001F034FB03E00021032001F0F7
:106310002FFBC34B1B78DBB2012B0AD0002B04D020
:10632000022B0ED0102B14D01AE0BE4801F012F947
:1063300016E0B74B1868BC4B9C46604401F00AF964
:106340000EE0B34B1868B94B9C46604401F002F96B
:1063500006E0AF4B1868B64B9C46604401F0FAF873
:106360000221002001F0CEF8AA4B1B889BB21D2B06
:106370002CD89B00AF4AD3589F46A54B1868FF23E3
:106380009B009C46604401F0E5F81FE0A14B1B8890
:106390003B331801C3189E4A1068C01801F0DAF8A0
:1063A00014E09C4B1B8833331801C318984A1068BB
:1063B000C01801F0CFF809E0964B1B882B33180169
:1063C000C318934A1068C01801F0C4F80E210020C9
:1063D00001F088F8984B1B78002B05D10121032090
:1063E00001F090F8FCF7EFFD0121072001F08AF899
:1063F000FCF7E9FD864B1868BB3001F0ABF88F481D
:1064000001F0A8F8834B1B889BB2002B04D101211B
:10641000042001F0ADFA05E07E4B198889B2042012
:1064200001F0A6FA864801F095F87C4B1B889BB2D8
:10643000072B05D8794B188880B201F097F802E055
:10644000002001F093F83D2001F068F87D4B1878AA
:1064500001F08CF80221012001F054F8704B1B78F8
:10646000DBB2012B0AD0002B04D0022B0ED0102B54
:1064700014D01AE06B4801F06DF816E0644B186810
:10648000694B9C46604401F065F80EE0604B18686B
:10649000664B9C46604401F05DF806E05C4B186872
:1064A000634B9C46604401F055F80E21002001F03A
:1064B00019F8614B1B78002B05D10121062001F052
:1064C00021F8FCF780FD5C4B1B78012B05D10121E5
:1064D0000C2001F017F8FCF776FD01210E2001F0E9
:1064E00011F8FCF770FD4A4B1868CC3001F032F817
:1064F000554801F02FF8494B1B889BB2FF2B06D85B
:10650000464B198889B2032001F032FA03E00021DA
:10651000032001F02DFA0221032000F0F3FF404B8D
:106520001B78DBB2012B0CD0002B05D0022B11D035
:10653000102B18D0FCF747FD3A4801F00BF8FCF798
:1065400042FD334B1868384B9C46604401F002F81A
:10655000FCF739FD2E4B1868344B9C46604400F024
:10656000F9FFFCF730FD2A4B1868314B9C4660441C
:1065700000F0F0FFFCF727FD254B1868DD3000F038
:10658000E9FF314800F0E6FF244B19888904890CA3
:106590002E4B19802E4B994203D8052001F0E8F9C3
:1065A00003E00021052001F0E3F90221032000F0BF
:1065B000A9FF1B4B1B78DBB2012B0CD0002B05D0A5
:1065C000022B11D0102B18D0FCF7FDFC154800F061
:1065D000C1FFFCF7F8FC0E4B1868134B9C46604457
:1065E00000F0B8FFFCF7EFFC094B18680F4B9C4616
:1065F000604400F0AFFFFCF7E6FC054B18680C4B5D
:106600009C46604400F0A6FFFCF7DDFC330100204F
:10661000F801002030020020C0CD0000360100202B
:10662000F7010020DCCD0000D9040000FB040000CD
:10663000EA0400006CAC000026010020E4CD00005C
:10664000E8CD00005D000020F0CD000064010020D6
:10665000FF270000DE4B1868EE3000F07BFFDD4BBB
:106660009B78032B09D0DA4B186888239B009C4643
:10667000604400F06FFFFCF7A6FCD74800F06AFF0B
:10668000D64B1B889BB2002B05D0D44B188880B208
:1066900000F06CFF02E0012000F068FFD04800F03D
:1066A00059FFD04B198889B2032001F061F90E21FE
:1066B000002000F017FFCC4B1B78002B05D10121E7
:1066C000042000F01FFFFCF77EFC0121092000F0F0
:1066D00019FFFCF778FCC54B1B78032B04D0C44B87
:1066E00020221A701D3A5A70B94B1868FF3000F01A
:1066F00031FFB84B9B78032B09D0B54B1868882322
:106700009B009C46604400F025FFFCF75CFCB94808
:1067100000F020FFB14B1B889BB2002B06D0AF4B83
:10672000198889B2042001F023F903E00121042033
:1067300001F01EF9AA4800F00DFFAA4B198889B292
:10674000032001F015F90221002000F0DBFEA34B2D
:106750001B889BB21D2B2CD89B00A74AD3589F4661
:106760009B4B1868FF239B009C46604400F0F2FEA0
:106770001FE09A4B1B883B331801C318944A1068DA
:10678000C01800F0E7FE14E0944B1B883333180167
:10679000C3188F4A1068C01800F0DCFE09E08F4B68
:1067A0001B882B331801C318894A1068C01800F0E1
:1067B000D1FE0E21002000F095FE8B4B1B78002BA4
:1067C00005D10121062000F09DFEFCF7FCFB012114
:1067D0000B2000F097FEFCF7F6FB844B1B78032B95
:1067E00004D0834B20221A701D3A5A70784B1868D7
:1067F0001130FF3000F0AEFE764B9B78032B09D0B2
:10680000734B186888239B009C46604400F0A2FEEE
:10681000FCF7D9FB794800F09DFE704B1B889BB2BA
:10682000002B05D06D4B188880B200F09FFE02E06F
:10683000012000F09BFE0221002000F063FE674B68
:106840001B889BB21D2B01D9FCF7BDFB9B006C4A3A
:10685000D3589F465E4B1868FF239B009C466044BC
:1068600000F078FEFCF7AFFB5C4B1B883B33180154
:10687000C318574A1068C01800F06CFEFCF7A3FB61
:10688000564B1B8833331801C318514A1068C0187F
:1068900000F060FEFCF797FB504B1B882B33180170
:1068A000C3184B4A1068C01800F054FEFCF78BFB6D
:1068B00054492431002000F071FE0021002000F036
:1068C00021FE002000F02AFE4F4B1B78002B02D047
:1068D00000224D4B1A703E4B18682230FF3000F0FA
:1068E00039FE404B198889B2052001F041F8022198
:1068F000012000F007FE454800F02CFE444B1868CC
:1069000000F040FEFCF75FFB3E4E31001C310020E2
:1069100000F044FE31002431012000F03FFE310040
:106920002C31022000F03AFE0121002000F0EAFDA7
:10693000354B1B78DBB2FF2B02D10A22324B1A7087
:10694000314B1B78DBB20A2B03D89B00314AD3585A
:106950009F4600222C4B1A700021002000F0D2FD2F
:10696000012000F0DBFD1A4E30683330FF3000F0BC
:10697000F1FD294B1B7821331801C3183068C0186A
:1069800000F0E8FDFCF71FFB0021002000F0BAFD3D
:10699000012000F0C3FD0E4B18684430FF3000F0BA
:1069A000D9FD1E4B1B78002B08D0094B18681C4BD7
:1069B0009C46604400F0CEFDFCF705FB044B1868D4
:1069C000184B9C46604400F0C5FDFCF7FCFAC0463D
:1069D000F80100208C000020F8CD000030020020DB
:1069E00054CC00003601002026010020B201002016
:1069F0003801002000CE0000E4AC000004CE00000E
:106A00005CAD00009CCA0000330100200CCE0000E9
:106A100068010020D4AD0000610100209D0100202C
:106A20008602000075020000002000F077FDEC4BAC
:106A30001B78002B08D0EB4B1868EB4B9C4660444E
:106A400000F088FDFCF7BFFAE64B1868AA239B000C
:106A50009C46604400F07EFDE44B1978032000F072
:106A600087FFFCF7B0FA002000F058FDDC4B1B78E4
:106A7000002B1ED0DB4B1868DD4B9C46604400F0B9
:106A800069FD0221002000F03DFDDA4B1B889BB21E
:106A9000002B09D0D74B188880B200F067FDD6488C
:106AA00000F058FDFCF78FFAD44800F053FDFCF7D6
:106AB0008AFACC4B1868D24B9C46604400F04AFDE1
:106AC0000221002000F01EFDCE4B1B78002B08D0C9
:106AD000C44B1868CC4B9C46604400F03BFDFCF76F
:106AE00072FAC04B1868C94B9C46604400F032FDF6
:106AF000FCF769FA0021002000F004FD012000F0FD
:106B00000DFDB84B18687730FF3000F023FDC04B07
:106B1000198889B2062000F02BFFFCF754FA0020F8
:106B200000F0FCFCAE4B1B78002B2CD0AD4B186852
:106B3000B84B9C46604400F00DFD0221002000F09F
:106B4000E1FCB54B1E88F608B60001363100042082
:106B500000F00EFF2D2000F0E1FCF11C89B20420B2
:106B600000F006FFAD4800F0F5FCAD4B1B78002BA4
:106B700004D0AC4800F0EEFCFCF725FAAA4800F07F
:106B8000E9FCFCF720FA974B1868BB239B009C4656
:106B9000604400F0DFFCFCF716FA0021002000F052
:106BA000B1FC012000F0BAFC8E4B18689930FF3020
:106BB00000F0D0FC9D4B1B78002B04D09C4800F0CB
:106BC000C9FCFCF700FA9B4800F0C4FCFCF7FBF999
:106BD0000021002000F096FC012000F09FFC814B7A
:106BE0001868AA30FF3000F0B5FC934B1B78002BDF
:106BF00004D0924800F0AEFCFCF7E5F9904800F0B4
:106C0000A9FCFCF7E0F90021002000F07BFC01204A
:106C100000F084FC734E3068BB30FF3000F09AFC0B
:106C2000884B1B7838331801C3183068C01800F03F
:106C300091FCFCF7C8F90021002000F063FC012062
:106C400000F06CFC674B1868CC30FF3000F082FC21
:106C50000121002000F056FC7B4800F07BFC0E2157
:106C6000002000F03FFC5E4B1878C0B2012100F01C
:106C700049FCFCF7A8F90021002000F043FC0120AA
:106C800000F04CFC714B1B78DBB2022B2BD0032B9A
:106C90003DD0012B13D0534E33686D4A9446634464
:106CA000180000F057FC0121002000F02BFC306898
:106CB000684B9C46604400F04DFCFCF784F9494E5B
:106CC0003368654A94466344180000F043FC012190
:106CD000002000F017FC3068604B9C46604400F0D8
:106CE00039FCFCF770F93F4E33685D4A94466344C3
:106CF000180000F02FFC0121002000F003FC306898
:106D0000584B9C46604400F025FCFCF75CF9354E7E
:106D10003368BB22D20094466344180000F01AFC8A
:106D20000121002000F0EEFB30684F4B9C46604490
:106D300000F010FCFCF747F94C4A1378013BDBB23A
:106D4000137001224A4B1A70FCF73DF90022474BA1
:106D50001A700132464B1A70FCF735F9454B1B7817
:106D6000DBB20A2B04D00D2B00D12EE1FCF72BF95E
:106D7000414B1B78042B01D0FCF725F9002000F0D3
:106D8000CDFB174B1B78DBB2062B03D89B003B4A8D
:106D9000D3589F460022124B1A70124B1868384B7A
:106DA0009C46604400F0D6FB364B1B78002B07D086
:106DB0000C4B1868344B9C46604400F0CBFB06E05B
:106DC000084B1868314B9C46604400F0C3FB02211D
:106DD000002000F097FB2E4800F0BCFBFCF7F3F816
:106DE00034010020F8010020B90200006E010020EB
:106DF000DB020000A401002014CE000018CE000029
:106E0000CA020000230100201D0500000C0500003F
:106E1000AE010020FD0200009801002054CC0000CB
:106E20002D0200201CCE000024CE000030010020E6
:106E3000E4CC0000F8CC00003D0200200CCD0000A6
:106E400020CD00009F010020C40100209B010020F4
:106E5000720500009405000083050000A5050000F0
:106E6000B6050000C7050000E9050000F20100209A
:106E700044020020240100203301002000AE000065
:106E800071060000B1010020C6060000D706000010
:106E9000A8CC0000D24B1868D24B9C46604400F04E
:106EA00059FBD14B9B78D14A12889A4203D9CE4BD9
:106EB0009A78CE4B1A80CD4B188800F057FBFCF720
:106EC00082F8C74B1868CA4B9C46604400F042FBEE
:106ED0000026C54B994601274B461A693B00B34033
:106EE0001A4203D02A2000F019FB02E00D2000F026
:106EF00015FB01360A2EEFD10221002000F002FB23
:106F0000B74B1868DD23DB009C46604400F022FB91
:106F1000B84800F01FFBFCF756F8B14B1868B64BA9
:106F20009C46604400F016FBAF4B5B79DBB2042B50
:106F300002D90422AC4B5A71AB4B5E79F6B2AF4822
:106F400000F008FB7300F6180136300000F00EFB6D
:106F5000AB4800F0FFFAB01C80B200F007FB022142
:106F6000002000F0CFFAA74800F0F4FAFCF72BF865
:106F70009B4B1868A44B9C46604400F0EBFAA34E70
:106F800030782D30C0B200F0C9FA0121032000F0A2
:106F9000B9FA33785B00944A9B5A9BB2002B07D115
:106FA0009A4B1A7890495200535A01339BB253526C
:106FB000964B1B785B008C4A985A80B200F0D6FA48
:106FC000934800F0C7FAFBF7FEFF92492C310220EC
:106FD00000F0E4FA0021002000F094FA012000F013
:106FE0009DFA8D4B1B78DBB2032B00D18BE0052B78
:106FF00000D1C8E0022B01D0FBF7E5FF834B1B78E3
:10700000002B6DD0854B1B68002B02D11422834BC3
:107010001A60734B1868824B9C46604400F09AFAE1
:107020000121002000F06EFA7E4800F093FA7E4BBA
:107030001B78002B02D101227B4B1A707A4B1978F6
:10704000032000F095FC202000F068FA0F26774B13
:10705000994601274B461A683B00B3401A4203D0B9
:10706000022000F05BFA02E0DB2000F057FA013E5C
:10707000072EEFD10221002000F044FA462000F054
:107080004DFA7E2000F04AFA694B1B78002B03D0A2
:10709000684800F05FFA02E0674800F05BFA634B73
:1070A000994601274B461A683B00B3401A4203D069
:1070B000022000F033FA02E0DB2000F02FFA013E5C
:1070C000002EEFD1594B1B68DB0704D5022000F0DE
:1070D00025FAFBF778FFDB2000F020FAFBF773FFBF
:1070E0003F4B1868AA239B009C46604400F032FA8C
:1070F0000121002000F006FA504B1978032000F01F
:1071000037FCFBF760FF414B1B78002B1AD0344B48
:1071100018684B4B9C46604400F01CFA494B1B8896
:107120009BB2002B09D0474B188880B200F01EFAA2
:10713000454800F00FFAFBF746FF444800F00AFA12
:10714000FBF741FF264B1868414B9C46604400F01A
:1071500001FA0121002000F0D5F93E4B1B78002BED
:1071600008D01F4B18683C4B9C46604400F0F2F975
:10717000FBF729FF1A4B1868384B9C46604400F017
:10718000E9F9FBF720FF214B1B78002B00D1B3E07E
:10719000134B1868324B9C46604400F0DBF9012128
:1071A000002000F0AFF92F4B1E88F608B60001361C
:1071B0003100042000F0DCFB2D2000F0AFF9F11CC1
:1071C00089B2042000F0D4FB274800F0C3F9274B14
:1071D0001B78002B4ED0264800F0BCF94DE0C0468D
:1071E000F801002082060000000200206401002057
:1071F0009306000028CE0000A40600004CCC00003E
:10720000CCCD000044CC0000B506000034010020C5
:10721000D0CD00009CCA0000330100201C010020DA
:10722000B902000030CE0000D90100203802002051
:107230001A02002038CE000040CE00006E0100206F
:10724000DB020000A401002014CE000018CE0000D4
:10725000CA020000230100201D0500000C050000EB
:10726000FD0200009801002054CC00002D020020F7
:107270001CCE0000384800F06DF90221002000F01B
:1072800041F9364B198889B2002900D1013189B200
:10729000042000F06DFB314B1B88013BDA170326FD
:1072A0001640F618B610B6002D4800F053F9013616
:1072B000B6B23100042000F05BFB2D2000F02EF967
:1072C000F11C89B2042000F053FB292000F026F9BC
:1072D0000E21002000F006F9224B1B78002B05D070
:1072E00001210C2000F00EF9FBF76DFE01210320B7
:1072F00000F008F9FBF767FE1B4B1868BB239B00E7
:107300009C46604400F026F90121002000F0FAF8C4
:10731000164B1B78002B04D0154800F01BF9FBF727
:1073200052FE144800F016F9FBF74DFE124B1B7885
:10733000002B01D0FBF762FE01330F49FBF75AFE29
:107340000E4B1B78002B01D1FDF7CEFDEEE70B4B6A
:107350001B78FCF777FBC04624CE0000A20100207A
:1073600048CE0000DC000020F80100202D020020A3
:107370001CCE00004CCE000044010020DB000020A9
:1073800010B500210F4B19600F4A14690F23984361
:1073900023401843906001220C4B1A600C4B1A6872
:1073A000D3009A1A0B4B5A60996005221A60190093
:1073B000802252020B681342FCD00022034B1A6059
:1073C00010BDC04694420050804000509042005092
:1073D0000800002010E000E0F0B55F4656464D463C
:1073E0004446F0B4FD222D4B1A60FC3A2C4B1A6037
:1073F00000222C4B1A602C4B98462C4B0020052564
:10740000802252022A4C01218B46C4464746642101
:10741000464636687143596098601D60196811428C
:10742000FCD05946216061460968C9006646366845
:10743000891B596098601D6019681142FCD017497A
:1074400009697F26B143C9B2894620603968C900FD
:107450003E68891B596098601D6019681142FCD014
:1074600059462160104909688A46C9005646891B59
:10747000596098601D6019681142FCD0206049462F
:107480000029C4D10022064B1A600A4A034B1A6035
:107490003CBC90469946A246AB46F0BD80400050A9
:1074A000944200504C4200500800002010E000E0E0
:1074B00090420050FD55000010B50C00002803D08C
:1074C0000122074B1A6002E00022054B1A602000DF
:1074D000FFF756FF2401E0B2FFF752FF10BDC04690
:1074E0004C42005070B504000D00FFF775FF2900F5
:1074F0002000FFF7E1FF70BD10B501210020FFF76C
:10750000F1FF10BD10B50901401880214942014327
:10751000C9B20020FFF7E6FF10BDC04610B501005C
:1075200003003C33DAB2382A0ED89300084AD35805
:107530009F46812108E0842106E0942104E09A21FD
:1075400002E08E2100E099210120FFF7CBFF10BD62
:1075500058CE000010B504000078002805D0013492
:10756000FFF7DCFF20780028F9D110BD00B585B009
:107570000A2201A902F092FD01A8FFF7EBFF05B076
:1075800000BDC04600B585B0102201A902F086FDFD
:1075900001A8FFF7DFFF05B000BDC04670B50400CD
:1075A0000D00072816D828210020FFF79BFFE400D4
:1075B00040210C43E1B20020FFF794FF2C00083576
:1075C0002078FFF7ABFF0134AC42F9D180210020D5
:1075D000FFF788FF70BDC04610B501280AD000280B
:1075E00004D002280AD003280CD00FE00948FFF786
:1075F000B1FF0EE00848FFF7ADFF0AE00748FFF7CC
:10760000A9FF06E00648FFF7A5FF02E00548FFF7DF
:10761000A1FF10BD3CCF000044CF00004CCF0000C4
:1076200054CF00005CCF000010B5002808D0262100
:107630000020FFF757FF18210020FFF753FF03E05A
:1076400029210020FFF74EFF10BDC04610B53220A3
:1076500000F0D2FA3020FFF793FE022000F0CCFABF
:107660003020FFF78DFE012000F0C6FA3020FFF732
:1076700087FEBD4B1B685A00D318DA009B18BB4A23
:10768000536000239360053313601100802252027F
:107690000B681342FCD02020FFF772FEB24B1B6830
:1076A0005A00D318DA009B18B04A53600023936045
:1076B000053313601100802252020B681342FCD084
:1076C0002020FFF75DFEA84B1B685A00D318DA0094
:1076D0009B18A64A53600023936005331360110082
:1076E000802252020B681342FCD09020FFF748FE24
:1076F0009D4B1B685A00D318DA009B189B4A5360B5
:1077000000239360053313601100802252020B683E
:107710001342FCD01020FFF733FE934B1B685A0036
:10772000D318DA009B18914A536000239360053305
:1077300013601100802252020B681342FCD0D0204B
:10774000FFF71EFE884B1B685A00D318DA009B18FF
:10775000864A536000239360053313601100802232
:1077600052020B681342FCD07020FFF709FE7E4BDB
:107770001B685A00D318DA009B187C4A5360002318
:107780009360053313601100802252020B6813428C
:10779000FCD06020FFF7F4FD734B1B685A00D31830
:1077A000DA009B18714A536000239360053313601D
:1077B0001100802252020B681342FCD05020FFF7C8
:1077C000DFFD694B1B685A00D318DA009B18674A23
:1077D000536000239360053313601100802252022E
:1077E0000B681342FCD00020FFF7CAFD5E4B1B68FC
:1077F0005A00D318DA009B185C4A53600023936048
:10780000053313601100802252020B681342FCD032
:107810006020FFF7B5FD544B1B685A00D318DA00FF
:107820009B18524A53600023936005331360110084
:10783000802252020B681342FCD0C020FFF7A0FD4B
:10784000494B1B685A00D318DA009B18474A53600B
:1078500000239360053313601100802252020B68ED
:107860001342FCD00020FFF78BFD3F4B1B685A00F2
:10787000D318DA009B183D4A536000239360053308
:1078800013601100802252020B681342FCD0C0200A
:10789000FFF776FD344B1B685A00D318DA009B18AB
:1078A000324A536000239360053313601100802235
:1078B00052020B681342FCD00020FFF761FD2A4BF7
:1078C0001B685A00D318DA009B18284A536000231B
:1078D0009360053313601100802252020B6813423B
:1078E000FCD01020FFF74CFD1F4B1B685A00D3182B
:1078F000DA009B181D4A5360002393600533136020
:107900001100802252020B681342FCD00020FFF7C6
:1079100037FD154B1B685A00D318DA009B18134A21
:1079200053600023936005331360110080225202DC
:107930000B681342FCD06020FFF722FD0A4B1B6846
:107940005A00D318DA009B18084A5360002393604A
:10795000053313601100802252020B681342FCD0E1
:10796000FFF73AFD10BDC0460800002010E000E01F
:10797000F0B5474680B40E0001280AD9012401223F
:10798000A300E4186400A4B20132D2B29042F7D14D
:1079900000E0012400281FD0A64212D2431EDBB211
:1079A00098460025471E02E00135A64209D2BD4295
:1079B00003D10020FFF7DAFD07E02020FFF7AEFD3E
:1079C00003E03000FFF7D2FD06E00A21200002F0BC
:1079D000C1FA84B24545E7D104BC9046F0BDC0462B
:1079E000F0B5474680B48846332800D9EAE0774BA3
:1079F0001B5CDBB28B4200D1E4E0A022D2058023E5
:107A00005B00592716268825D750D650D550D45814
:107A1000002CF9D08024A40180236D4AD4506D4BF2
:107A20001A6801252A431A60F822D2018418A4009A
:107A30000022DA605C609A601D61BFF36F8F1A00EC
:107A40001369002BFCD1634B9B6842461340984559
:107A50000FD1013AFF3A5F4B2125DD605C609A60EF
:107A600001221A61BFF36F8F1A001369002BFCD13A
:107A70009AE0A022D20580235B005927162688258C
:107A8000D750D650D550D458002CF9D0514B1A6845
:107A9000012422431A602222DA60F82252025A603C
:107AA0001C61BFF36F8F1A001369002BFCD1474B89
:107AB00042461A54F8256D0200241900454A212730
:107AC00001260B5D013BFF3BD7605560936016615B
:107AD000BFF36F8F1369002BFCD101340435252CC3
:107AE000EFD13D4CE378A27824881B0612049B1842
:107AF000E318384A2124D460384C54609360012341
:107B00001361BFF36F8F1369002BFCD1324B1A69DD
:107B1000304B2124DC60324C5C609A6001221A6197
:107B2000BFF36F8F1A001369002BFCD12A4B5A89BF
:107B30001B89284B2122DA602A4A5A602A4A9A6015
:107B400001221A61BFF36F8F1A001369002BFCD159
:107B5000214B9A791A7D5A799B891E4B2122DA6032
:107B6000224A5A600A229A60093A1A61BFF36F8F5B
:107B70001A001369002BFCD11D4D01241D4B9C469E
:107B8000144A21270126630061465B5A9BB2D760E5
:107B9000556093601661BFF36F8F1369002BFCD1A2
:107BA000013404350A2CEED10A4A13680124A34398
:107BB0001360002480235B00A022D205D450034B25
:107BC00042461A5404BC9046F0BDC046A8000020AE
:107BD00000E100E000C000500002002094F001002D
:107BE00098F001009CF001000A000A00A0F00100DA
:107BF000A4F00100480000200022054B1A60830019
:107C000018184000024A13689842FCD87047C046D2
:107C10003402002010B50122094B9A60094B1B6801
:107C2000002B03D0074A1368013B1360064B1B78F7
:107C3000002B04D00022044B1A70F8F77DFA10BD17
:107C400000000140E0000020F8000020F8B501220B
:107C50007E4B9A607E4B1B68002B0CD07C4B1A68C5
:107C6000013A1A601B68002B05D10022794B1A706B
:107C70000132794B1A70794B1B78DBB2452B04D853
:107C8000764A13780133DBB21370754B1B78002BE7
:107C90000AD0734A1378013BDBB213701378002BC0
:107CA00002D101226F4B1A706F4B1B78002B0CD046
:107CB0006D4A1378013BDBB213701378002B04D1AB
:107CC0000133644A1370644A1370684B1B68002BBD
:107CD0003FD0664B1A68013A1A601B68002B38D1F6
:107CE0000122634B1A70634BDA78D2B21A711B7D92
:107CF000002B06D15F4A118880231B020B4313809F
:107D000004E05C4A13885B045B0C1380594B5B797D
:107D1000594A11689A009B1A0D3307229A40114262
:107D200007D0524A13680A3313601422534B1A7057
:107D30000FE0524B1B78002B0BD0504A1378013BBD
:107D4000DBB213701378002B03D0484A13680A3350
:107D500013604B4B1B68002B0CD0494B1A68013A3F
:107D60001A601B68012B05D10222464B1A700332A0
:107D7000434B1A60444B1B68002B03D0424A1368E4
:107D8000013B1360414B1B68002B09D03F4B1A6825
:107D9000013A1A601B68002B02D104223C4B1A7076
:107DA0003C4B1B68012B09D93A4B1A68013A1A60FF
:107DB0001B68012B02D10122274B1A70364B1B780E
:107DC000012B11D1354B1B68002B04D15022334BB2
:107DD0001A60FFF791FB314A1368591E1160282B76
:107DE00002D101221C4B1A702D4B1B889BB2002B19
:107DF00004D02B4A1388013B9BB21380294B1B688C
:107E0000002B60D0274B1A68013A1A601B68002BC0
:107E100059D1254B1B88254A1340934250D0224A02
:107E2000138809218B431380214B1B78002B06D12B
:107E3000204B1B885B045B0C1F4A138043E01F4BE5
:107E40001B885B045B0C1C4A13803CE00000114063
:107E500068020020FC01002044020020FD010020F7
:107E6000FE010020460200204102002028010020DF
:107E7000B60100200002002038020020F30100209B
:107E800060000020DE0000205C0100201C010020BA
:107E90003202002074010020B201002010000020F6
:107EA000C00100204C020020680000200B070000E9
:107EB000400000208C0000203C0100207C010020BC
:107EC0000022514B1A800023504AFF218C46012783
:107ED0004F4EF0256146916091683800984081438B
:107EE000916011699C002940301D21500133042B01
:107EF000F0D1474B04225A61FF21444A916000218E
:107F0000444A11701B691A0604D4012242494A707E
:107F100040490A705A0604D401223F498A703D49FB
:107F20000A709A0604D401223B49CA7039490A7082
:107F3000DB0604D40123384A1373364A1370344BDA
:107F4000DB681A0604D4012233490A7131490A70E8
:107F50005A0604D4012230494A712E490A709A0601
:107F600004D401222C498A712A490A70DB0604D400
:107F70000123294A5373274A1370254B9B681A061D
:107F800004D401222449CA7122490A705A0604D431
:107F9000012221490A721F490A709A0604D401225B
:107FA0001D494A721B490A70DB0604D401231A4A90
:107FB0009373184A1370164B5B681A0604D4012297
:107FC00015498A7213490A705A0604D401221249CB
:107FD0000A7010490A709A0604D401220E49CA7226
:107FE0000C490A70DB0604D401230B4AD373094AF7
:107FF00013700A4B1B68002B04D10133064A13741B
:10800000044A1370F8BDC0463C01002000400050F7
:1080100010000020DB000020440100207C420050C2
:1080200030B5194B1B78002B12D0184B18491A0089
:108030000C3231C931C20021002219809960DA70F6
:10804000FF31997019710139FF3919835A7119E09B
:10805000104B0F491A000C3231C931C200210022E5
:1080600019809960DA70FF31997019710139FF39FF
:1080700019835A719A7E03318A439A769A7E01391E
:108080008A439A7630BDC046400000207C01002023
:1080900044CC00008C000020F0B585B0FFF72CFA2E
:1080A000C74B1B78002B03D00120FFF7BDFA02E07D
:1080B0000020FFF7B9FAC34B1B889BB2002B06D0F8
:1080C000C04B18884004400CFFF750FA02E0BE484D
:1080D000FFF740FABD4B1B885B0400D1E2E0BC49CE
:1080E0000020FFF75BFA00210420FFF70BFA0020C5
:1080F000FFF714FAB74B1B78DBB2062B03D89B00B3
:10810000B54AD3589F460022B44B1A600132B44B93
:108110001A60B448FFF71EFA2AE00022AF4B1A603B
:108120000132AF4B1A60B048FFF714FA20E000228A
:10813000AA4B1A600132AA4B1A60AC48FFF70AFA40
:1081400016E00122A54B1A600022A54B1A60A84830
:10815000FFF700FA00210820FFF7D4F908E0002219
:108160009E4B1A6001329E4B1A60A248FFF7F2F94B
:10817000964B18884004400CFFF7F8F900210C20BA
:10818000FFF7C0F98F4CE1780320FFF7F1FB23885C
:108190001BB2002B03DA7E20FFF7C0F902E07F203C
:1081A000FFF7BCF901210020FFF7ACF92020FFF711
:1081B000B5F90024834E0125E0B2B2682B00A3403C
:1081C0001A4207D00A2101F04BFF3031C8B2FFF745
:1081D000A5F902E00D20FFF7A1F90134052CEBD140
:1081E000854B1B78002B03D08448FFF7B3F902E0DE
:1081F0008348FFF7AFF90024744E0125E0B2B2685E
:108200002B00A3401A4207D00A2101F029FF303188
:10821000C8B2FFF783F902E00D20FFF77FF90134C0
:10822000052CEBD102210020FFF76CF92020FFF78D
:1082300075F92500634F0126E8B2BA683300AB40F8
:108240001A4207D00A2101F00BFF3031C8B2FFF704
:1082500065F902E00D20FFF761F901350A2DEBD138
:10826000654B1B78002B03D06448FFF773F902E0DD
:108270006348FFF76FF9554E0125E0B2B2682B0055
:10828000A3401A4207D00A2101F0EAFE3031C8B2F9
:10829000FFF744F902E00D20FFF740F901340A2C02
:1082A000EBD1AEE1474B9B7EDB0703D4454B9B7E76
:1082B0009B070BD546490020FFF770F900210520E8
:1082C000FFF720F90020FFF729F906E0002105203B
:1082D000FFF718F92020FFF721F93E4B1B78DBB29E
:1082E000062B03D89B00474AD3589F4600223B4B9E
:1082F0001A6001323A4B1A604348FFF72BF93BE012
:108300000022364B1A600132354B1A603F48FFF7A6
:1083100021F931E00022314B1A600132304B1A60F2
:108320003B48FFF717F927E001222C4B1A60002287
:108330002B4B1A60234B1B889BB2002B03D1354873
:10834000FFF708F918E01F4B9878C0B2FFF744F91F
:1083500012E00022214B1A600132214B1A602E4894
:10836000FFF7F8F808E000221C4B1A6001321C4BA2
:108370001A602A48FFF7EEF8124CE1780320FFF765
:10838000F7FA23881BB2002B03DA7E20FFF7C6F82A
:1083900002E07F20FFF7C2F800230A4CE218107BAE
:1083A00001A9C854127B002A3AD10A2B38D82021BF
:1083B00001AAD1540133DBB20B2BF9D134E0C04612
:1083C000B00100208C00002004D500007C010020BA
:1083D000E4CA0000B201002064CF00002C4200502B
:1083E0002842005008D500000CD5000010D5000030
:1083F00014D5000018D50000310100201CD5000064
:1084000020D5000080CF000024D500002CD500002E
:1084100034D5000018CC00003CD5000044D5000045
:108420000133DBB20A2BB9D901A80023C372FFF7CD
:1084300091F87E4B1B885B0400D1E2E000247B4F67
:108440007B4D7C4EE0B2BA680123A3401A422DD086
:10845000774B1B5D073BDAB2462A03D89300764A76
:10846000D3589F460A2101F0FBFD3031C8B2FFF717
:1084700055F84CE02A20FFF751F848E01320FFF7A9
:108480004DF844E00520FFF749F840E00C20FFF7E5
:1084900045F83CE0B220FFF741F838E00720FFF74D
:1084A0003DF834E0F520FFF739F830E02B5D073B6D
:1084B000DAB2462A02D89300F3589F460A2101F007
:1084C000CFFDC9B2002903D00D20FFF727F81EE029
:1084D0002E20FFF723F81AE01920FFF71FF816E007
:1084E0002D20FFF71BF812E06F20FFF717F80EE0C2
:1084F0005F20FFF713F80AE01520FFF70FF806E0FA
:108500004B20FFF70BF802E07C20FFF707F801345F
:10851000052C97D1454B9B78012B6FD0434B9B7813
:10852000022B6BD0414D424E444FE0B2AA6801236A
:10853000A3401A422BD0335D073BDAB2462A02D859
:108540009300FB589F460A2101F08AFD3031C8B2E2
:10855000FEF7E4FF4EE02A20FEF7E0FF4AE013209A
:10856000FEF7DCFF46E00520FEF7D8FF42E00C20D6
:10857000FEF7D4FF3EE0B220FEF7D0FF3AE007203E
:10858000FEF7CCFF36E0F520FEF7C8FF32E0284BBF
:108590001B5D073BDAB2462A03D89300284AD3581A
:1085A0009F460A2101F05CFDC9B2002903D00D20CD
:1085B000FEF7B4FF1EE02E20FEF7B0FF1AE01920F0
:1085C000FEF7ACFF16E02D20FEF7A8FF12E06F20AB
:1085D000FEF7A4FF0EE01520FEF7A0FF0AE05F20E3
:1085E000FEF79CFF06E04B20FEF798FF02E07C20A0
:1085F000FEF794FF0134152C97D102E01148FEF7E5
:10860000A9FF114B1B78002B0ED0FA2252000F4B02
:108610001A6002210020FEF775FF0D4B18680D4B04
:108620009C466044FEF796FF05B0F0BD8C0000202C
:10863000FC000020B8D000009CCF0000D4D1000086
:10864000F0D20000A4CC0000FC0100206802002051
:10865000F8010020F90600004000C0B2002901D056
:108660000123184303230340013B012B06D8C30613
:1086700002D50E23184301E00E2398437047C046ED
:1086800070B50122CA4B9A60CA4A1368013313605D
:10869000C94B1B78002B04D0C74A1378013BDBB2CF
:1086A0001370C64CA3690133A361C54B1968C9B2E5
:1086B000207FFFF7D1FF05002077C24B1968C9B2B0
:1086C000607FFFF7C9FF60773F239D439843802D6C
:1086D00009D1002801D101F0E7F9C02801D001F04B
:1086E000FFF901F0EFF9402D01D001F0F9F9C028B0
:1086F00001D101F0D9F9002801D101F0E3F901F02D
:10870000EFF9B14B1B78002B0DD0B04BDB78002B71
:1087100009D1AF4B1B78DBB2132B04D80022AC4B32
:108720001A7001F0DDF9AB4A13780133DBB2137034
:10873000A94B1B78032B00D0FBE0A44B1B889BB2FA
:10874000002B00D1EAE0A04B1B78002B08D09E4BF9
:108750001B78002B70D09D4B1B881BB2002B6BDA53
:108760009A4B1B79DBB2642B56D99C4B1B78DBB23E
:10877000012B06D0002B09D0022B0DD0032B2FD0BC
:108780004FE0924AD3780133DBB2D3708F4AD3786B
:108790000133DBB2D37044E08C4BDB78DBB2132BBC
:1087A00005D88A4AD3780133DBB2D3700FE0874B08
:1087B000DB78DBB23D2B05D8844AD3780233DBB2B9
:1087C000D37004E0814AD3780433DBB2D3707F4B9B
:1087D000DB78DBB27E2B24D97E227C4BDA7020E062
:1087E0007A4BDB78DBB2092B05D8784AD378013392
:1087F000DBB2D37015E0754BDB78DBB2152B05D8F7
:10880000724AD3780233DBB2D3700AE06F4AD3786E
:108810000433DBB2D37004E06C4AD3780133DBB2AB
:10882000D3706A4AD3781279DBB293426FD9674A20
:108830001379DBB2D3706AE0644B1B79DBB2642B33
:108840004ED9664B1B78DBB2012B06D0002B09D02A
:10885000022B0DD0032B27D047E05C4AD378013B95
:10886000DBB2D370594AD378013BDBB2D3703CE022
:10887000564BDB78DBB23E2B05D9544AD378043B08
:10888000DBB2D37031E0514BDB78DBB2142B05D96E
:108890004E4AD378023BDBB2D37026E04B4AD37802
:1088A000013BDBB2D37020E0484BDB78DBB2162B08
:1088B00005D9464AD378043BDBB2D37015E0434B6D
:1088C000DB78DBB20A2B05D9404AD378023BDBB216
:1088D000D3700AE03D4AD378013BDBB2D37004E0A9
:1088E0003A4AD378013BDBB2D370384BDB78DBB24A
:1088F000C82B0CD90022354BDA70334B1B78002B78
:1089000005D0324A118880231B020B4313802F4B62
:10891000DB78002B02D100222D4B1A702B4B1B88C9
:108920005B0401D001F0DCF80022284BDA7001F082
:10893000D7F8254B1B78002B01D101F0D1F8234B40
:108940001B881BB2002B01DA01F0CAF81F4BDB7841
:10895000002B01D101F0C4F81C4AD378013BDBB2F3
:10896000D37001F0BDF81E4B1B78DBB2012B3BD05E
:10897000002B07D0022B00D127E1032B00D118E3F5
:1089800001F0AEF8134A13780133DBB21370154AC5
:1089900013780133DBB213701378DBB2102B01D8DC
:1089A00001F09EF80A220F4B1A7001F099F8C046A8
:1089B000200001403402002064020020100000204A
:1089C000684200506C4200509D0100208C00002045
:1089D000FD01002033010020B201002061010020D0
:1089E000F201002024010020CC4A13780133DBB2CD
:1089F0001370CB4B1B780D2B06D11378042B03D1AE
:108A000013780133DBB21370C54B1B780E2B01D0EA
:108A100001F066F8C34B1B78002B00D1C4E0C24BB9
:108A20001B78DBB2012B43D0002B03D0022B7DD06F
:108A300001F056F8BD4B1B78DBB2012B16D0002B92
:108A400003D0022B23D001F04BF8B94B1B78DBB2DB
:108A50005F2B04D8B64A13780533DBB21370B44BDE
:108A60001B780133B34A936201F03AF8B24B1B789A
:108A7000DBB25F2B04D8B04A13780533DBB2137036
:108A8000AD4B1B780133AB4AD36101F029F8AB4BF6
:108A90001B78DBB25F2B04D8A84A13780533DBB20E
:108AA0001370A64B1B780133A24A136101F018F82A
:108AB0009E4B1B78DBB2012B16D0002B03D0022B70
:108AC00023D001F00DF89E4B1B78DBB25F2B04D84E
:108AD0009B4A13780533DBB21370994B1B78013333
:108AE000944A936200F0FCFF964B1B78DBB25F2B3D
:108AF00004D8944A13780533DBB21370914B1B787A
:108B000001338C4AD36100F0EBFF8F4B1B78DBB253
:108B10005F2B04D88C4A13780533DBB213708A4B71
:108B20001B780133834A136100F0DAFF7F4B1B7817
:108B3000DBB2012B16D0002B03D0022B23D000F088
:108B4000CFFF824B1B78DBB25F2B04D87F4A1378B0
:108B50000533DBB213707D4B1B780133754A93628A
:108B600000F0BEFF7A4B1B78DBB25F2B04D8784A4B
:108B700013780533DBB21370754B1B7801336D4AE4
:108B8000D36100F0ADFF734B1B78DBB25F2B04D8D1
:108B9000704A13780533DBB213706E4B1B780133C8
:108BA000644A136100F09CFF614B1B78DBB25F2BC2
:108BB00004D85F4A13780533DBB213705C4B1B7823
:108BC00001335C4A936200F08BFF554B1B78DBB29C
:108BD0000B2B00D121E10D2B00D153E10A2B01D049
:108BE00000F07EFF4D4B1B78DBB2052B01D900F066
:108BF00077FF9B00584AD3589F46584B1B78002B51
:108C000001D100F06DFF0122554B1A7000F068FF92
:108C1000544A53790133DBB253715379DBB2372BAA
:108C200002D92E224F4B5A714E4B1B885B045B0CB2
:108C3000FF2B07DD4B4B5B79DBB2332B02D83422A1
:108C4000484B5A71474B1B885B045B0C464A934266
:108C500001DC00F045FF3722424B5A7100F040FF23
:108C6000424B1878C0B20121FEF74CFC404A137801
:108C70000133DBB213701378DBB21F2B02D8202232
:108C80003B4B1A703A4B1B785BB2002B02DA202266
:108C9000374B1A70354B1B78354A1278D2B23149AE
:108CA000CB181A7300F01CFF324B1B78022B01D03B
:108CB00000F016FF2D4A13780133DBB213701378DE
:108CC000DBB2062B01D800F00BFF0022274B1A70F5
:108CD00000F006FF284B1B78002B00D193E0274BB8
:108CE0001B78DBB20F2B00D179E00DD8092B64D0B3
:108CF00004D8062B57D0072B5AD047E00B2B66D051
:108D000060D30C2B68D041E03C2B74D038D8112BA9
:108D10006BD067D3222B6BD038E0C04633010020E4
:108D2000240100202F010020220100202C0100201E
:108D3000F1010020000004409C010020640000209C
:108D4000FF01002078010020420200206201002083
:108D5000420100209A0100200CD4000049020020AA
:108D6000420000208C000020FF270000340100207A
:108D700066000020F2010020200100209E0100205A
:108D80004C2B08D04D2B0BD0402B37D04C22E34B33
:108D90001A7000F0A5FE4D22E04B1A7000F0A0FE04
:108DA0000622DE4B1A700722DC4B1A7000F098FE88
:108DB0000922DA4B1A7000F093FE0A22D74B1A7080
:108DC00000F08EFE0B22D54B1A7000F089FE0C22AB
:108DD000D24B1A7000F084FE0F22D04B1A70102272
:108DE000CE4B1A701122CD4B1A702222CB4B1A7027
:108DF0003C22CA4B1A704022C84B1A700022C74B43
:108E00001A7000F06DFEC64A13780133DBB213709E
:108E10000122C44B1A7000F063FEC34B1B78DBB217
:108E2000062B01D900F05CFE9B00C04AD3589F4638
:108E30000123BF4A1370BF4A137000F051FEBC4AB1
:108E400013780133DBB213701378DBB2022B02D933
:108E50000222B74B1A700122B64B1A7000F040FE86
:108E6000B54A138801339BB2138013889BB28022CA
:108E7000D200934201D800F033FE0122AE4B1A809B
:108E800000F02EFEA84B1B78DBB20A2B01D900F0B4
:108E900027FE9B00A94AD3589F46A94A137801335D
:108EA000DBB213701378DBB2032B01D800F018FE8D
:108EB0000022A34B1A7000F013FEA24A11784B4215
:108EC0004B41DBB2137000F00BFE00229E4B1A8068
:108ED00001329E4B1A7001229D4B1A7000F000FE69
:108EE0009C4B1B889BB296221201934204D19A4A52
:108EF000984B1A8000F0F4FD964B1B889BB2964A63
:108F0000934201D000F0ECFD944A924B1A8000F09D
:108F1000E7FD934A11784B424B41DBB2137000F0EE
:108F2000DFFD904A11784B424B41DBB2137000F0E9
:108F3000D7FD8D4B1A780132D2B21A7019780322FC
:108F40000A401A701878383011234343874A106852
:108F5000C018FEF7FFFA00F0C3FD7D4B1878C0B2D1
:108F60000121FEF7CFFA824A13780133DBB2137086
:108F700013785BB2002B02DA20227D4B1A70744BFF
:108F80001B78DBB27A4A1278D2B27A49CA5400F01E
:108F9000A7FD794A13780133DBB213701378DBB283
:108FA000032B01D800F09CFD0022734B1A7000F0D7
:108FB00097FD724B1B78DBB20A2B62D00D2B01D0D0
:108FC00000F08EFD584B1B78DBB2032B27D0052B0E
:108FD00043D0022B01D000F083FD5D4B1B78002BAA
:108FE0000FD0674B1B78674A1278DBB2934201D3EC
:108FF00000F076FD624A13780133DBB2137000F0A3
:109000006FFD604B1B78DBB2332B01D900F068FD9C
:109010005C4A13780133DBB2137000F061FD4C4BF6
:109020001B78002B11D0584A138805339BB213804C
:1090300013889BB2FA229200934201D800F050FDAF
:109040000022514B1A8000F04BFD504A11784B42E0
:109050004B41DBB2137000F043FD3D4B1B78002BFE
:1090600007D04B4A11784B424B41DBB2137000F0F2
:1090700037FD484A11784B424B41DBB2137000F088
:109080002FFD334B1B78DBB2062B01D900F028FDF6
:109090009B00414AD3589F46404A11784B424B416E
:1090A000DBB2137000F01CFD3D4B9A783D4B1B88E2
:1090B0009BB29A4201D800F013FD3A4A138801335B
:1090C0009BB2138000F00CFD354B5B79DBB2032BB8
:1090D00001D900F005FD324A53790133DBB25371F7
:1090E00000F0FEFC1A4B1A782D495200535A0133F6
:1090F0009BB2535200F0F4FC124B1B78002B57D05C
:10910000294BDB78002B53D1284B1B78DBB2132B78
:109110004ED80022254B1A7000F0E2FC9E01002080
:1091200048020020450200203301002024D4000022
:10913000260100206F0100203002002040D40000F2
:10914000610100209D01002098010020DD00002029
:1091500034010020AE010020904C000000E1FFFF30
:10916000300100203D0200209F010020F801002076
:1091700066000020C40100209B0100202401002083
:10918000D90100206E010020A4010020230100204D
:10919000DC0000202D0200206CD40000B101002072
:1091A00000020020640100208C000020FD0100204E
:1091B000BF4B1B78002B04D0BD4A1378013BDBB2B8
:1091C0001370BC4B1B78002B08D0BA4B1B78002BBC
:1091D0006FD0B94B1B881BB2002B6ADAB64B1B79D8
:1091E000DBB2642B4ED9B54B1B78DBB2012B06D01A
:1091F000002B09D0022B0DD0032B27D047E0AE4A1D
:10920000D378013BDBB2D370AB4AD378013BDBB2FE
:10921000D3703CE0A84BDB78DBB23E2B05D9A64AE5
:10922000D378043BDBB2D37031E0A34BDB78DBB205
:10923000142B05D9A04AD378023BDBB2D37026E0C9
:109240009D4AD378013BDBB2D37020E09A4BDB78A8
:10925000DBB2162B05D9984AD378043BDBB2D37026
:1092600015E0954BDB78DBB20A2B05D9924AD3780F
:10927000023BDBB2D3700AE08F4AD378013BDBB20A
:10928000D37004E08C4AD378013BDBB2D3708A4BB5
:10929000DB78DBB2C82B7BD90022874BDA70854B99
:1092A0001B78002B74D0844A13885B045B0C1380FA
:1092B0006EE0834B1B78032B60D17F4B1B79DBB2B5
:1092C000642B56D97D4B1B78DBB2012B06D0002BCB
:1092D00009D0022B0DD0032B2FD04FE0764AD37844
:1092E0000133DBB2D370744AD3780133DBB2D3706D
:1092F00044E0714BDB78DBB2132B05D86E4AD37890
:109300000133DBB2D3700FE06B4BDB78DBB23D2B6C
:1093100005D8694AD3780233DBB2D37004E0664AD9
:10932000D3780433DBB2D370634BDB78DBB27E2BB4
:1093300024D97E22604BDA7020E05F4BDB78DBB211
:10934000092B05D85C4AD3780133DBB2D37015E022
:10935000594BDB78DBB2152B05D8574AD37802334B
:10936000DBB2D3700AE0544AD3780433DBB2D37053
:1093700004E0514AD3780133DBB2D3704E4AD3783C
:109380001279DBB2934203D94B4A1379DBB2D37023
:10939000494BDB78002B02D100224A4B1A70464B16
:1093A0001B885B0400D09BE30022434BDA7097E3F9
:1093B000454B1B78DBB2012B1BD0002B06D0022BB8
:1093C00000D117E1032B00D1E5E289E3384A137895
:1093D000013BDBB213703D4A1378013BDBB21370E3
:1093E0001378DBB2092B00D97AE31022374B1A70BD
:1093F00076E32F4A1378013BDBB21370334B1B78B3
:109400000D2B06D11378042B03D11378013BDBB26B
:1094100013702E4B1B780E2B00D061E32C4B1B7866
:10942000002B00D1D6E02B4B1B78DBB2012B5DD09B
:10943000002B03D0022B00D192E051E3264B1B7886
:10944000DBB2012B14D0002B02D0022B20D047E33B
:10945000224B1B78DBB2042B04D9204A1378053B3E
:10946000DBB213701D4B1B7801331D4A936237E347
:109470001C4B1B78DBB2042B04D91A4A1378053B2A
:10948000DBB21370174B1B780133154AD36127E306
:10949000154B1B78DBB2042B04D9134A1378053B18
:1094A000DBB21370104B1B7801330D4A136117E3C5
:1094B000330100209D0100208C000020610100206C
:1094C000B2010020FD010020F20100202401002053
:1094D0002F010020220100202C010020F10100209A
:1094E000000004409C01002064000020C04B1B7859
:1094F000DBB2012B14D0002B02D0022B20D0EFE2E4
:10950000BC4B1B78DBB2042B04D9BA4A1378053B59
:10951000DBB21370B74B1B780133B74A9362DFE2BB
:10952000B64B1B78DBB2042B04D9B44A1378053B45
:10953000DBB21370B14B1B780133AF4AD361CFE27A
:10954000AF4B1B78DBB2042B04D9AD4A1378053B33
:10955000DBB21370AA4B1B780133A74A1361BFE239
:10956000A34B1B78DBB2012B14D0002B02D0022BB3
:1095700020D0B5E2A34B1B78DBB2042B04D9A14A5F
:109580001378053BDBB213709E4B1B7801339A4A6C
:109590009362A5E29C4B1B78DBB2042B04D99A4A58
:1095A0001378053BDBB21370974B1B780133924A5B
:1095B000D36195E2954B1B78DBB2042B04D9934A17
:1095C0001378053BDBB21370904B1B7801338A4A4A
:1095D000136185E28E4B1B78DBB2042B04D98C4AD5
:1095E0001378053BDBB21370894B1B780133824A39
:1095F000936275E2874B1B78DBB20B2B00D1D9E06D
:109600000D2B00D13DE10A2B00D069E2824B1B7883
:10961000DBB2052B00D963E29B00804AD3589F46FA
:109620007F4B1B78002B00D15AE203227D4B1A702E
:1096300056E27D4A5379013BDBB253715379DBB279
:109640002D2B02D83722784B5A71774B1B885B043D
:109650005B0CFF2B07DD744B5B79DBB2332B02D83D
:109660003722714B5A71704B1B885B045B0C6F4A3D
:10967000934200DC34E237226B4B5A7130E26C4B80
:109680001878C0B20121FDF73DFF6A4A1378013B0B
:10969000DBB213701378DBB21F2B02D87F22654B2D
:1096A0001A70644B1B78DBB21F2B02D82022614B4F
:1096B0001A705F4B1B785F4A1278D2B25A49CB18A6
:1096C0001A730DE25C4B1B78022B00D008E2584A5B
:1096D0001378013BDBB213701378DBB20A2B00D88E
:1096E000FEE10622524B1A70FAE1544B1B78002B14
:1096F00057D0534B1B78DBB20F2B2FD00DD8092B33
:109700003CD004D8062B40D0072B3BD014E00B2BC9
:109710002CD02FD30C2B25D00EE03C2B12D005D80B
:10972000112B15D017D3222B0FD005E04C2B34D0A2
:109730004D2B2ED0402B02D04022414B1A703C22A0
:109740003F4B1A7022223E4B1A7011223C4B1A706A
:1097500010223B4B1A700F22394B1A700C22384BD7
:109760001A70BDE10B22364B1A70B9E10A22344B54
:109770001A70B5E10922324B1A70B1E10722304B61
:109780001A70ADE106222E4B1A704D222C4B1A7026
:10979000A6E14C222A4B1A70A2E10022284B1A7033
:1097A0009EE1284A1378013BDBB213700122264B5D
:1097B0001A7095E1184B1B78DBB2062B00D98FE1AC
:1097C0009B00224AD3589F460022214B1A70013237
:1097D000204B1A7084E11E4B1B78002B04D01C4ACE
:1097E0001378013BDBB2137001221A4B1A7077E138
:1097F0002C010020FF01002000000440780100201F
:109800004202002062010020420100209A01002053
:10981000F1010020240100203301002088D4000041
:1098200049020020420000208C000020FF27000099
:109830003401002066000020F201002020010020F9
:109840009E0100204802002045020020A0D4000014
:10985000260100206F010020A24B1B889BB2002B29
:1098600004D0A04A1388013B9BB213809D4B1B88F8
:109870009BB2002B00D033E18022D200994B1A809A
:109880002EE1994B1B78DBB20A2B00D928E19B0013
:10989000964AD3589F46964A1378013BDBB2137021
:1098A0001378DBB2032B00D81AE10322904B1A7015
:1098B00016E1904A11784B424B41DBB213700FE135
:1098C0008D4A8E4B1A8001228D4B1A7000228D4BCF
:1098D0001A7005E18C4B1B889BB2E1221202934265
:1098E00003D18A4A884B1A80FAE0874B1B889BB2C7
:1098F000864A934200D0F3E096221201824B1A80EE
:10990000EEE0834A11784B424B41DBB21370E7E043
:10991000804A11784B424B41DBB21370E0E07E4B42
:109920001A78013AD2B21A70197803220A401A70D2
:109930001878383011234343784A1068C018FDF76F
:1099400009FECDE06F4B1878C0B20121FDF7DAFDBA
:10995000734A1378013BDBB213701378DBB21F2B11
:1099600002D87F226E4B1A70664B1B78DBB26C4AB2
:109970001278D2B26B49CA54B2E06B4A1378013BF9
:10998000DBB213701378DBB2052B00D8A8E00222FB
:10999000654B1A70A4E0654B1B78DBB20A2B55D0DF
:1099A0000D2B00D09CE0504B1B78DBB2032B1FD05B
:1099B000052B36D0022B00D092E0524B1B78002BA7
:1099C0000BD05B4B1B78DBB2012B00D888E0584AE8
:1099D0001378013BDBB2137082E0564B1B78002BEF
:1099E00000D17DE0534A1378013BDBB2137077E07E
:1099F000444B1B78002B0DD04F4A1388053B9BB27C
:109A0000138013889BB2FA229200934268D94A4B82
:109A10001A8065E0494A11784B424B41DBB2137022
:109A20005EE0384B1B78002B09D0454A11784B4239
:109A30004B41DBB213700022424B1A8050E0424A85
:109A400011784B424B41DBB2137049E02D4B1B7830
:109A5000DBB2062B44D89B003C4AD3589F463C4A75
:109A600011784B424B41DBB2137039E0394B1B8804
:109A70009BB2002B34D0374A1388013B9BB2138032
:109A80002EE0354B5B79002B2AD0334A5379013BCA
:109A9000DBB2537124E01B4B1A782F495200535A02
:109AA000013B9BB253521BE001222C4B1A702C4BF2
:109AB0001B78DBB2002B01D1FFF71EFB022B00D17C
:109AC00076E40DE00122254B1A70254B1B78DBB2A2
:109AD000002B01D1FEF715FE022B01D1FEF743FF4B
:109AE00070BDC0463002002033010020BCD400000D
:109AF000610100209D010020FF3F0000980100202F
:109B0000DD00002034010020AE010020904C000058
:109B1000300100203D0200209F010020F8010020BC
:109B200066000020C40100209B01002024010020C9
:109B3000D90100206E010020A40100202301002093
:109B4000DC000020A20100202D020020E8D400004B
:109B5000B101002064010020000200204402002026
:109B6000DA01002048400823072142B2002A03DA24
:109B700040004840C0B201E04000C0B2013BDBB24F
:109B8000002BF2D17047C04670B5040005000835BF
:109B900000202178FFF7E6FF0134AC42F9D103063B
:109BA00001D5C043C0B270BD10B50322324B5A700C
:109BB000324B1B78002B2CD0314B1B885B0428D0F8
:109BC0002F4A10887F2420402B4988701388DB0996
:109BD0002340CB7093681B049B0E4B7113881BB200
:109BE000002B05DA0A00497940230B43537104E046
:109BF000214A537940218B435371214B9A68D208F3
:109C00007F2002401C498A719B681B010340CB7175
:109C100027E01C4A10887F24204017498870138849
:109C2000DB092340CB7093681B049B0E4B71138898
:109C30001BB2002B05DA0A00497940230B4353710C
:109C400004E00D4A537940218B4353710D4B9A68C0
:109C5000D2087F20024008498A719B681B0103409B
:109C6000CB71084BDA787F231340034C237120001B
:109C7000FFF78AFF207210BDE800002031010020AC
:109C80007C0100208C00002010B57B4B1B787B4AA8
:109C900010697B49CB182021585480235B02536400
:109CA00078490B78DBB25A1CD2B20A70072B0ED956
:109CB000754A764B1A60A022D205516B744B0B404B
:109CC00053630022734B1A600132734B1A606A4B64
:109CD0001B78012B47D1714B1B78DBB2FF2B23D1B3
:109CE0006F4B1B78002B3ED06E4B5B78403B032BB9
:109CF00039D86D4B1B78002B35D06C4A634B1A60FA
:109D00000122654B1A60A021C9054B6B8020C00160
:109D100003434B635F4B1A600023654A1370594A33
:109D20001370614A13701EE05E4B1B785B4A127819
:109D3000DBB2934217D1534B1B78DBB2082B0FD900
:109D40005A4A524B1A60A022D205536B8021C90196
:109D50000B43536301224F4B1A600022544B1A707D
:109D60000022484B1A70524B1B78DBB24D4AD25C32
:109D7000D2B2424B1A62196801220A431A603E4B62
:109D80001B783F4AD31820229B5C7F2B09D93A4A83
:109D900013783B482021C3185B5C435401231370A4
:109DA00069E0354B1B78DBB20E2B04D8324A1378AE
:109DB0000133DBB213703E4B1B78DBB20E2B04D8A1
:109DC0003B4A13780133DBB213702B4B1B78082B03
:109DD0001AD100232A483749020020329A5CCA541B
:109DE0000133082BF8D12D4B1B78DBB2FF2B0BD1A5
:109DF000304B5B78403B032B03D80122284B1A7071
:109E000002E00022264B1A701B4B1B78092B32D123
:109E1000FF22244B1A701A4B20331B7A254C2372D5
:109E20002000FFF7B1FE237ADBB298420FD0164A2A
:109E3000164B1A60A022D205516B154B0B40536391
:109E40000022144B1A600132134B1A6013E0194BB5
:109E50001B785BB2002B0EDA164B1B780F4A127878
:109E6000DBB2934204D10D4B1B78DBB20D4A137069
:109E70000122114B1A7010BD2D010020000003407B
:109E80001000002041000020FF2000004040005052
:109E9000FFBFFFFF2C42005038420050E40000207A
:109EA0002C020020E8000020F6010020FF10000036
:109EB0006B0000201C020020F800002030B50022BA
:109EC0001E4B1A601E4B1B69073213400DD11D4AF1
:109ED0001B4B1A621C4B1A48042102E0013B002B69
:109EE00023D0C2681142F9D01FE0072B25D1174AB1
:109EF000134B1A62164B1248042102E0013B002B5F
:109F000013D0C2681142F9D00FE0D550D450D050D0
:109F1000D1580029F9D00222094B1A61002180236F
:109F20005B00A022D205D15007E0A022D2058023F9
:109F30005B00592516248820E7E730BD000000208B
:109F40000002005017420000E12E000039560800C0
:109F500067560000002243088B4274D303098B42EA
:109F60005FD3030A8B4244D3030B8B4228D3030CE9
:109F70008B420DD3FF22090212BA030C8B4202D38B
:109F80001212090265D0030B8B4219D300E0090AB3
:109F9000C30B8B4201D3CB03C01A5241830B8B42BC
:109FA00001D38B03C01A5241430B8B4201D34B03A5
:109FB000C01A5241030B8B4201D30B03C01A52410A
:109FC000C30A8B4201D3CB02C01A5241830A8B428F
:109FD00001D38B02C01A5241430A8B4201D34B0278
:109FE000C01A5241030A8B4201D30B02C01A5241DC
:109FF000CDD2C3098B4201D3CB01C01A5241830990
:10A000008B4201D38B01C01A524143098B4201D3C9
:10A010004B01C01A524103098B4201D30B01C01AF4
:10A020005241C3088B4201D3CB00C01A524183086E
:10A030008B4201D38B00C01A524143088B4201D39B
:10A040004B00C01A5241411A00D2014652411046FB
:10A050007047FFE701B5002000F006F802BDC046DA
:10A060000029F7D076E770477047C046931E10B5B9
:10A070000C00222B0ED80A2A05D00021611800F00E
:10A0800053F8200010BD0028F7DA2D2340420B7052
:10A090000121F3E7002300200B70F3E710B5FFF771
:10A0A000E5FF10BD031C0A7801311A700133002A44
:10A0B000F9D170470B00034370B505009B0701D130
:10A0C000032A15D8002A12D04C1C0978013A6B1CBF
:10A0D000297000291BD0210007E00C7801335D1E98
:10A0E000013A2C700131002C11D0002AF5D170BD3D
:10A0F0000B4E0C680B4BE318A3433342E4D10435F9
:10A100002B1F043A04311C60032AF2D8DAE79C18AA
:10A110000021002AEBD019700133A342FBD1E6E7FE
:10A1200080808080FFFEFEFEF0B5574645464E46D5
:10A13000E0B48AB090466A461D4B0D00060013CB72
:10A1400013C213CB13C213CB13C21B78EA4613708E
:10A150004346023B2F000024222B01D924E04C4629
:10A16000631C300041469946FFF77AFF53465B5C1B
:10A1700030003B704146FFF7EDFE0137061EEED181
:10A180004B46E8540023002C07D0EA5C295DE954D3
:10A190002A550133013CA342F7DB28000AB01CBC5E
:10A1A00090469946A246F0BD2C700020F6E7C046C6
:10A1B0004CD50000AA030000AC070000BA0600005E
:10A1C000AC070000AC070000AC070000AC070000C3
:10A1D00036070000AC070000AC070000AC07000029
:10A1E000AC070000AC070000AC070000AC070000A3
:10A1F000AC070000AC070000AC070000AC07000093
:10A20000AC070000AC070000AC070000AC07000082
:10A21000AC070000AC0700008A030000AC07000098
:10A22000AC070000AC070000AC070000AC07000062
:10A23000AC07000020070000AC070000AC070000DE
:10A24000AC070000AC070000AC070000AC07000042
:10A25000AC070000AC070000AC070000AC07000032
:10A26000AC070000AC070000AC070000AC07000022
:10A27000AC070000AC070000AC070000AC07000012
:10A28000AC070000AC070000AC070000AC07000002
:10A29000AC070000AC070000AC070000AC070000F2
:10A2A000AC070000AC07000094030000940300001A
:10A2B000940300009403000036050000FE05000032
:10A2C000360500009A050000280500004204000041
:10A2D000C804000064260000642600004C0800004A
:10A2E0006426000064260000642600005626000054
:10A2F000AC2000002A220000401800006426000064
:10A300006426000064260000381C0000981B000032
:10A3100064260000D81D0000121E0000961F0000D9
:10A32000242000006426000064260000642600004B
:10A3300064260000642600006426000064260000F5
:10A3400064260000D816000064260000D017000024
:10A35000F4170000342600002E26000064260000BA
:10A3600064260000962200002E1800004A09000012
:10A370004A0900004A090000520900005209000081
:10A38000520900005A0900005A0900005A09000049
:10A39000420900008A0900007409000080090000D9
:10A3A0008A09000074090000800900008A09000081
:10A3B00074090000380A0000380A0000380A00005A
:10A3C000400A0000400A0000400A0000480A00005D
:10A3D000480A0000480A0000300A0000CE130000BE
:10A3E000C4130000B2130000A0130000AC1300005F
:10A3F000CE1300009A130000AA22000028260000B5
:10A400002826000064250000EC23000084240000BE
:10A41000282600009025000028260000B625000010
:10A42000F02500002826000028260000282600002D
:10A4300028260000282600002826000028260000E4
:10A44000282600002826000028260000EA22000016
:10A45000C82300004A230000C8230000C8230000CE
:10A46000C8230000C8230000C8230000AA2300005E
:10A470009C23000084230000C8230000C8230000A0
:10A48000C8230000C8230000762300005C230000DE
:10A490004831000064310000643100006431000084
:10A4A0006431000064310000643100006431000058
:10A4B0006431000064310000BC380000DA3D000067
:10A4C0002E4C0000B24C0000244D0000684D0000EE
:10A4D000983D0000BE34000022350000C037000067
:10A4E0000E3800007838000056360000563600005E
:10A4F0003835000092350000EA350000563600007D
:10A5000056360000B2380000843800008C38000055
:10A51000943800009C380000A4380000AC380000DB
:10A520005241000082460000744800008C48000040
:10A53000264C0000264C0000BC4B00006841000087
:10A540001C43000040430000D04300003E45000093
:10A55000284600006646000058450000D645000029
:10A560000E460000F2450000F2450000F2450000F2
:10A57000F24500002E4700001C4700007C47000009
:10A58000C247000010480000444800005C4800003A
:10A59000A0480000BE480000DC4800000049000060
:10A5A0003649000048490000E8490000004A000020
:10A5B000184A0000DC4A00006A4B0000EA4F000025
:10A5C000B04F0000F24F0000DA4F0000E24F0000F1
:10A5D000CA4F0000B04F0000B04F0000B04F000065
:10A5E000B04F0000B04F0000B04F0000B04F00006F
:10A5F000B04F0000B04F0000B04F0000B04F00005F
:10A60000B04F0000B04F0000B04F0000B04F00004E
:10A61000B04F0000B04F0000B04F0000B04F00003E
:10A62000B04F0000B04F0000B04F0000B04F00002E
:10A63000B04F0000B04F0000B04F0000B04F00001E
:10A64000B04F0000B04F0000B04F0000B04F00000E
:10A65000B04F0000B04F0000B04F0000B04F0000FE
:10A66000B04F0000B04F0000B04F0000B04F0000EE
:10A67000B04F0000B04F0000B04F0000B04F0000DE
:10A68000B04F0000B04F0000B04F0000B04F0000CE
:10A69000B04F0000B04F0000B04F0000B04F0000BE
:10A6A000B04F0000B04F0000B04F0000B04F0000AE
:10A6B000B04F0000B04F0000B04F0000B04F00009E
:10A6C000B04F0000B04F0000B04F0000B04F00008E
:10A6D000C24F0000D24F0000505000000C5000004C
:10A6E0005850000048500000405000002850000022
:10A6F0000C5000000C5000000C5000000C500000EA
:10A700000C5000000C5000000C5000000C500000D9
:10A710000C5000000C5000000C5000000C500000C9
:10A720000C5000000C5000000C5000000C500000B9
:10A730000C5000000C5000000C5000000C500000A9
:10A740000C5000000C5000000C5000000C50000099
:10A750000C5000000C5000000C5000000C50000089
:10A760000C5000000C5000000C5000000C50000079
:10A770000C5000000C5000000C5000000C50000069
:10A780000C5000000C5000000C5000000C50000059
:10A790000C5000000C5000000C5000000C50000049
:10A7A0000C5000000C5000000C5000000C50000039
:10A7B0000C5000000C5000000C5000000C50000029
:10A7C0000C5000000C5000000C5000000C50000019
:10A7D0000C5000000C5000000C5000000C50000009
:10A7E0000C5000000C5000000C50000038500000CD
:10A7F00030500000CE50000094500000D6500000B1
:10A80000BE500000C6500000A6500000945000004A
:10A8100094500000945000009450000094500000A8
:10A820009450000094500000945000009450000098
:10A830009450000094500000945000009450000088
:10A840009450000094500000945000009450000078
:10A850009450000094500000945000009450000068
:10A860009450000094500000945000009450000058
:10A870009450000094500000945000009450000048
:10A880009450000094500000945000009450000038
:10A890009450000094500000945000009450000028
:10A8A0009450000094500000945000009450000018
:10A8B0009450000094500000945000009450000008
:10A8C00094500000945000009450000094500000F8
:10A8D00094500000945000009450000094500000E8
:10A8E00094500000945000009450000094500000D8
:10A8F00094500000945000009450000094500000C8
:10A900009450000094500000B6500000AE5000007B
:10A9100036510000F25000003E5100002E51000060
:10A92000265100000E510000F2500000F2500000CD
:10A93000F2500000F2500000F2500000F25000000F
:10A94000F2500000F2500000F2500000F2500000FF
:10A95000F2500000F2500000F2500000F2500000EF
:10A96000F2500000F2500000F2500000F2500000DF
:10A97000F2500000F2500000F2500000F2500000CF
:10A98000F2500000F2500000F2500000F2500000BF
:10A99000F2500000F2500000F2500000F2500000AF
:10A9A000F2500000F2500000F2500000F25000009F
:10A9B000F2500000F2500000F2500000F25000008F
:10A9C000F2500000F2500000F2500000F25000007F
:10A9D000F2500000F2500000F2500000F25000006F
:10A9E000F2500000F2500000F2500000F25000005F
:10A9F000F2500000F2500000F2500000F25000004F
:10AA0000F2500000F2500000F2500000F25000003E
:10AA1000F2500000F2500000F2500000F25000002E
:10AA2000F25000001E5100001651000014530000A7
:10AA30005A530000A2530000EA53000032540000B1
:10AA40008E540000C2540000EA540000AC560000CE
:10AA500088570000BE570000E4590000805C0000E9
:10AA6000B65C0000BA550000C855000080560000D2
:10AA7000405500005255000066550000705500001A
:10AA8000EC560000FA560000085700001657000068
:10AA900024570000325700005C570000FE570000AA
:10AAA00020580000585800006858000084580000E2
:10AAB000A0580000BC580000E45800000C590000E9
:10AAC0002E59000050590000145D00000262000081
:10AAD000B068000008690000386D00004C6D00008F
:10AAE000545D0000B05D0000F65D0000D05E000027
:10AAF000305F0000B0600000B2610000585F0000ED
:10AB0000985F0000BE5F0000006000005060000021
:10AB100050600000506000004C6100004661000081
:10AB20004661000046610000466100004661000089
:10AB3000466100007C610000466100008461000005
:10AB40006C610000746100005C61000046610000FF
:10AB50004661000046610000466100004661000059
:10AB60004661000046610000466100004661000049
:10AB70004661000046610000466100004661000039
:10AB80004661000046610000466100004661000029
:10AB90004661000046610000466100004661000019
:10ABA0004661000046610000466100004661000009
:10ABB00046610000466100004661000046610000F9
:10ABC00046610000466100004661000046610000E9
:10ABD00046610000466100004661000046610000D9
:10ABE00046610000466100004661000046610000C9
:10ABF00046610000466100004661000046610000B9
:10AC000046610000466100004661000046610000A8
:10AC10004661000046610000466100004661000098
:10AC20004661000046610000466100004661000088
:10AC30004661000046610000466100004661000078
:10AC4000466100004661000054610000646100003C
:10AC5000C2620000F4630000E66400007865000052
:10AC600054660000D6660000DA6700007A630000D0
:10AC70008C6300008C6300008C6300008C63000018
:10AC80008C6300008C6300008C6300008C63000008
:10AC9000CC630000CC630000CC630000CC630000F8
:10ACA000CC630000CC630000CC630000CC630000E8
:10ACB000A2630000A2630000A2630000CC63000056
:10ACC000CC630000CC630000CC630000CC630000C8
:10ACD000CC630000CC630000CC630000B8630000CC
:10ACE000B8630000606700007267000072670000D0
:10ACF00072670000726700007267000072670000F0
:10AD00007267000072670000B2670000B26700005F
:10AD1000B2670000B2670000B2670000B2670000CF
:10AD2000B2670000B2670000886700008867000013
:10AD300088670000B2670000B2670000B2670000D9
:10AD4000B2670000B2670000B2670000B26700009F
:10AD5000B26700009E6700009E6700005468000014
:10AD600068680000686800006868000068680000A3
:10AD70006868000068680000686800006868000093
:10AD8000C62F0000C62F0000C62F0000C62F0000EF
:10AD9000C62F0000C62F0000C62F0000C62F0000DF
:10ADA000806800008068000080680000C62F0000F6
:10ADB000C62F0000C62F0000C62F0000C62F0000BF
:10ADC000C62F0000C62F0000C62F000098680000A4
:10ADD000986800005869000088690000286A00002F
:10ADE000666A0000F46A00001E6B00009A6B0000A7
:10ADF000D06B0000066C0000366C0000766C000022
:10AE00009A6D0000946E0000C26E00001A6F000080
:10AE1000706F0000706F0000706F0000A5FFFFFFF3
:10AE2000FF0000FF0F0F0F0000FFFFFF0000830E69
:10AE300020202055736572206E616D6520202020D2
:10AE400000FFFFFFFFFFFFFFFFFFFFFFFFFF0F0000
:10AE50004C6F6B204D656EFC2020202020202000B0
:10AE6000004443432D50726F6772616D6D672E20F1
:10AE700000006D332D50726F6772616D6D672E200B
:10AE800020000045696E7374656C6C756E67656E45
:10AE9000202000004C43442042656C657563687453
:10AEA000756E67000048616E64436F6E74726F6CFC
:10AEB00020563220000041757377E4686C656E207F
:10AEC00020202020200000446174656E666F726D42
:10AED00061742020202000004E616D65202020201C
:10AEE00020202020202020000045696E74726167B8
:10AEF0002020202020202020000043562028627996
:10AF0000746529202020202020000043562028623C
:10AF100069742920202020202020000042617369CC
:10AF2000732D41647265737365202000006C616E3F
:10AF30006765204164726573736520200000526567
:10AF4000676973746572202020202020200000484B
:10AF500061757074676C6569732020202020000083
:10AF60005261696C436F6D204356202020202000E1
:10AF7000006D332D4164726573736520202020209D
:10AF800000003132384653204D6F64652020202068
:10AF90002000005265676C65726D6F6475732020C8
:10AFA000202000007338382D45696E7374656C6C11
:10AFB000756E670000426F6F7374657220202020E9
:10AFC000202020200000496E746572666163652050
:10AFD000426175642000005765696368656E2020D2
:10AFE00020202020202000004C6F6B666F726D6166
:10AFF0007420202020202000004D4D2D5369676EC5
:10B00000616C20506175736500005261696C436F1B
:10B010006D20537570706F727400005573657220E7
:10B020004E616D6520202020202000004B75727A33
:10B030007363686C2E2D506F6C2E2000004B757260
:10B040007A7363686C2E2D456D70662E0000616CFE
:10B050006C65205765696368656E20202000005785
:10B0600065696368656E666F726D617420200000AB
:10B070006E75722066FC722044434321202020001C
:10B08000004E617469762028313A31292020202031
:10B0900000004C696E6561722028323A3129202007
:10B0A00020000050726F67726573736976203120DB
:10B0B0002020000050726F677265737369762032CA
:10B0C00020202000004143204D6F64757320202014
:10B0D0002020202000004443204D6F647573202001
:10B0E000202020202000004B6F6E6669677572611A
:10B0F00074696F6E202000007338382D4D6F6475B1
:10B100006C653A0000000000007338382D4D6F6404
:10B11000756C74657374202000004B75727A7363CC
:10B12000686C2E2D506F6C2E2000004B75727A7358
:10B1300063686C2E2D456D70662E0000616C6C6529
:10B14000205765696368656E202020000057656997
:10B150006368656E666F726D617420200000204D1B
:10B160004D2031202031342000000000000000205C
:10B170004D4D2031202032376100000000000000DA
:10B18000204D4D20312020323762000000000000A9
:10B1900000204D4D203220203134200000000000DE
:10B1A0000000204D4D203220203237610000000089
:10B1B000000000204D4D2032202032376200000078
:10B1C00000000000204443432020203134200000B0
:10B1D000000000000020444343202020323820009B
:10B1E000000000000000204443432020313238207A
:10B1F00000000000000000206D3320202031323894
:10B200002000000000000000303A2061757320200B
:10B21000202020202020000000313A205461696C59
:10B2200062697473202020000000323A202B2049EC
:10B23000644E6F7469667920000000333A202B2039
:10B240004163636573736F727900000041647265D6
:10B2500073736520286B75727A29000000416E6651
:10B260006168722D4765736368772E000000416E38
:10B27000666168722D5665727A2E000000000042E9
:10B2800072656D732D5665727A2E00000000000005
:10B2900048F6636873742D4765736368772E000002
:10B2A000004D697474656E2D4765736368772E0071
:10B2B000000056657273696F6E00000000000000A8
:10B2C0000000004865727374656C6C65722D4944AA
:10B2D000000000004164722E20286C616E672D48CA
:10B2E00029000000004164722E20286C616E672DD9
:10B2F0004C2900000000436F6E736973742D416424
:10B30000726573736500005261696C436F6D000074
:10B3100000000000000000004B6F6E6669677572E8
:10B320006174696F6E00000000206C657365000039
:10B3300000000000000000000000204665686C6509
:10B340007200000000000000000000736368726576
:10B350006962650000000000000000006E65676122
:10B3600074697620284443432900000000706F73FD
:10B370006974697620284D4D2900000000005A6943
:10B38000666665723D4B75727A7761686C20004B1A
:10B3900075727A7761686C202020202020200000C0
:10B3A000616B746976656E204465636F64657220B5
:10B3B0000073706569636865726E2020202020200C
:10B3C00000005370726163686520202020202020D7
:10B3D0002000004C616E6775616765202020202089
:10B3E00020200000446575747363682020202020AD
:10B3F0002020200000456E676C69736820202020A3
:10B400002020202000005461616C2020202020207A
:10B41000202020202000004E656465726C616E64FF
:10B4200073202020202000004C616E67756520206D
:10B430002020202020202000004672616E63616978
:10B440007320202020202020000053707261636848
:10B4500065202020202020202000004974616C6994
:10B46000656E69736368202020200000537072614C
:10B470006368652020202020202020000053706178
:10B480006E69736368202020202020200000537004
:10B490007261636865202020202020202000005356
:10B4A0007072616368652020202020202020000029
:10B4B00050656E64656C6175746F6D6174696B0065
:10B4C00000416B746976696572656E2020202020CA
:10B4D0000000476573636877696E6469676B6569C7
:10B4E00074000046756E6B74696F6E656E20202067
:10B4F000202000004B6F6E74616B7465202020204B
:10B50000202020000048616C74652D5A6569742004
:10B51000000000000000616B74697620202020206C
:10B5200000000000000000696E616B7469762020E5
:10B5300020000000000000005461737465200000CA
:10B540000000000000000000005A656E7472616C1B
:10B5500065207570646174656E0000004C6F636FE8
:10B560006D6F74697665206D656E750000444343A8
:10B570002070726F6772616D6D696E6700006D3368
:10B580002070726F6772616D6D696E672000005385
:10B59000657474696E6773202020202020200000CD
:10B5A0004C4344206261636B6C69676874202000BF
:10B5B0000048616E64436F6E74726F6C2056322067
:10B5C000000053656C65637420202020202020201B
:10B5D0002000004461746120666F726D61742020E8
:10B5E000202000004E616D6520202020202020209A
:10B5F0002020200000456E74727920202020202019
:10B6000020202020000043562028627974652920DC
:10B610002020202020000043562028626974292021
:10B6200020202020202000005072696D6172792056
:10B63000616464726573730000457874656E642E8E
:10B640002061646472657373000052656769737486
:10B6500065722020202020202000004D61696E208E
:10B66000747261636B202020202000005261696C9D
:10B67000436F6D204356202020202000006D332092
:10B6800061646472657373202020202000003132D1
:10B69000384653204D6F6465202020202000004A4A
:10B6A0006F67206469616C206D6F64652020000005
:10B6B0007338382073657474696E677320202000B6
:10B6C00000426F6F7374657220202020202020209C
:10B6D0000000496E7465726661636520426175643D
:10B6E000200000506F696E747320202020202020DD
:10B6F000202000004C6F636F20666F726D617420B4
:10B7000020202000004D4D205369676E616C207031
:10B710006175736500005261696C436F6D205375EC
:10B7200070706F7274000055736572206E616D6584
:10B73000202020202020000053686F727420632E88
:10B7400020706F6C2E2000000053686F72742063AD
:10B750002E2073656E7365000000416C6C20706F65
:10B76000696E747320202020200000506F696E7471
:10B770007320666F726D6174202000006F6E6C79AB
:10B7800020666F722044434321202000004E6174E4
:10B7900069762028313A31292020202000004C6988
:10B7A0006E6561722028323A312920202000005035
:10B7B000726F6772657373697620312020200000F4
:10B7C00050726F6772657373697620322020200093
:10B7D000004143206D6F6465202020202020202020
:10B7E00000004443206D6F6465202020202020202D
:10B7F000200000636F6E66696775726174696F6EB1
:10B8000020200000733838206D6F64756C65733AC2
:10B810002020200000733838206D6F64756C65201F
:10B8200074657374000053686F727420632E207007
:10B830006F6C2E2020000053686F727420632E20DE
:10B8400073656E7365000000416C6C20706F696EEB
:10B85000747320202020200000506F696E747320C4
:10B86000666F726D617420200000204D4D203120E4
:10B870002031342000000000000000204D4D203118
:10B88000202032376100000000000000204D4D20D4
:10B8900031202032376200000000000000204D4DB2
:10B8A0002032202031342000000000000000204D14
:10B8B0004D203220203237610000000000000020BF
:10B8C0004D4D203220203237620000000000000081
:10B8D0002044434320202031342000000000000099
:10B8E0000020444343202020323820000000000084
:10B8F0000000204443432020313238200000000063
:10B90000000000206D33202020313238200000005C
:10B9100000000000303A206F6666202020202020A2
:10B920002020000000313A205461696C6269747310
:10B93000202020000000323A202B2049644E6F74F2
:10B9400069667920000000333A202B20416363654B
:10B9500073736F72790000004164647265737320C1
:10B960002873686F7274290000416E666168722DD9
:10B970004765736368772E000000416E66616872E8
:10B980002D5665727A2E00000000004272656D73BC
:10B990002D5665727A2E00000000000048F663689C
:10B9A00073742D4765736368772E0000004D6974CA
:10B9B00074656E2D4765736368772E0000005665C9
:10B9C0007273696F6E000000000000000000004804
:10B9D00065727374656C6C65722D494400000000DB
:10B9E000416464722E20286C6F6E672D4829000018
:10B9F00000416464722E20286C6F6E672D4C290004
:10BA00000000436F6E7369737420616464726573C0
:10BA10007300005261696C436F6D0000000000000C
:10BA200000000000436F6E66696775726174696F2C
:10BA30006E000000002072656164000000000000DC
:10BA4000000000000000204572726F7200000000CC
:10BA500000000000000000777269746500000000BB
:10BA600000000000000000006E65676174697620C8
:10BA7000284443432900000000706F73697469769D
:10BA800020284D4D2900000000005A696666657245
:10BA90003D4B75727A7761686C20004B75727A77CE
:10BAA00061686C20202020202020000061637469E0
:10BAB0007665206465636F6465722000007361764B
:10BAC00065202020202020202020202000005370EE
:10BAD0007261636865202020202020202000004C17
:10BAE000616E67756167652020202020202000009E
:10BAF0004465757473636820202020202020200076
:10BB000000456E676C69736820202020202020206B
:10BB100000005461616C2020202020202020202063
:10BB20002000004E656465726C616E647320202095
:10BB3000202000004C616E677565202020202020A9
:10BB400020202000004672616E636169732020200E
:10BB5000202020200000537072616368652020203F
:10BB6000202020202000004974616C69656E697393
:10BB70006368202020200000537072616368652094
:10BB80002020202020202000005370616E69736304
:10BB900068202020202020200000537072616368FC
:10BBA0006520202020202020200000537072616337
:10BBB00068652020202020202020000050656E6431
:10BBC000656C6175746F6D6174696B0000416B74B5
:10BBD0006976696572656E20202020200000476527
:10BBE00073636877696E6469676B656974000046A2
:10BBF000756E6B74696F6E656E20202020200000CA
:10BC00004B6F6E74616B7465202020202020200013
:10BC10000048616C74652D5A6569742020202020CD
:10BC20000000616B74697620202020200000000055
:10BC3000000000696E616B746976202020000000AE
:10BC4000000000006B65792000000000000000008B
:10BC500000000000007570646174652063656E7497
:10BC6000722E73742E0000004C6F636D656E75202C
:10BC70002020202020202000004443432D70726F9C
:10BC80006772616D6D672E2000006D332D70726FCD
:10BC90006772616D6D672E20200000496E737465B8
:10BCA0006C6C696E67656E20202000004C43442058
:10BCB0007665726C69636874696E67000048616ECE
:10BCC00064436F6E74726F6C2056322000004B69B3
:10BCD000657A656E2020202020202020200000444E
:10BCE000617461666F726D617420202020200000F5
:10BCF0004E61616D20202020202020202020200067
:10BD000000496E766F6572202020202020202020A0
:10BD100000004356202862797465292020202020C5
:10BD2000200000435620286269742920202020200A
:10BD30002020000042617369736164726573202082
:10BD400020202000006C616E6720616472657320A2
:10BD500020202020000052656769737465722020DE
:10BD600020202020200000486F6F666473706F6F82
:10BD700072202020202000005261696C436F6D20EA
:10BD80004356202020202000006D3320616472651E
:10BD900073202020202020200000313238465320FC
:10BDA0004D6F6465202020202000004A6F67646981
:10BDB000616C206D6F646520202000007338382D81
:10BDC000496E7374656C6C696E67200000426F6F1A
:10BDD0007374657220202020202020200000496EEE
:10BDE0007465726661636520426175642000005766
:10BDF000697373656C202020202020202020000003
:10BE00004C6F63666F726D617420202020202000CB
:10BE1000004D4D2D5369676E61616C7061757A6577
:10BE200000005261696C436F6D20537570706F72C2
:10BE300074000055736572204E616D6520202020CE
:10BE4000202000004B6F7274736C2E20706F6C2E6C
:10BE500020202000004B6F7274736C2E2067657673
:10BE60002E2020200000616C6C652057697373657B
:10BE70006C73202020000057697373656C666F72C5
:10BE80006D61742020200000416C6C65656E20445B
:10BE90004343212020202000004E61746976202831
:10BEA000313A31292020202000004C696E656172F2
:10BEB0002028323A3129202020000050726F67720A
:10BEC00065737369762031202020000050726F67FF
:10BED0007265737369762032202020000041432070
:10BEE0004D6F646520202020202020200000444346
:10BEF000204D6F646520202020202020200000435A
:10BF00006F6E6669672020202020202020200000FE
:10BF10007338382D6D6F64756C653A000000000051
:10BF2000007338382D6D6F64756C6574657374209B
:10BF300000004B6F7274736C2E20706F6C2E20207B
:10BF40002000004B6F7274736C2E206765762E2074
:10BF500020200000616C6C652057697373656C73F9
:10BF6000202020000057697373656C666F726D61E5
:10BF7000742020200000204D4D203120203134201D
:10BF800000000000000000204D4D203120203237FD
:10BF90006100000000000000204D4D2031202032C3
:10BFA000376200000000000000204D4D20322020AC
:10BFB00031342000000000000000204D4D203220D0
:10BFC0002032376100000000000000204D4D20327B
:10BFD000202032376200000000000000204443436C
:10BFE00020202031342000000000000000204443C5
:10BFF00043202020323820000000000000002044B0
:10C00000434320203132382000000000000000208F
:10C010006D33202020313238200000000000000065
:10C02000303A206F6666202020202020202000004B
:10C0300000313A205461696C6269747320202000D9
:10C040000000323A202B2049644E6F7469667920D3
:10C05000000000333A202B204163636573736F72D5
:10C06000790000004164726573736520286B7572F6
:10C070007A29000000416E666168722D476573631E
:10C0800068772E000000416E666168722D566572F9
:10C090007A2E00000000004272656D732D566572A5
:10C0A0007A2E00000000000048F6636873742D4784
:10C0B00065736368772E0000004D697474656E2D9A
:10C0C0004765736368772E00000056657273696F69
:10C0D0006E000000000000000000004865727374EC
:10C0E000656C6C65722D4944000000004164722E3D
:10C0F00020286C616E672D482900000000416472A1
:10C100002E20286C616E672D4C2900000000436FC3
:10C110006E736973742D41647265737365000052A8
:10C1200061696C436F6D00000000000000000000BA
:10C130004B6F6E66696775726174696F6E0000009F
:10C1400000206C657A65000000000000000000001F
:10C15000000020466F7574202000000000000000E1
:10C1600000000073636872696A76656E0000000003
:10C17000000000006E6567617469762028444343BF
:10C180002900000000706F736974697620284D4D96
:10C190002900000000005A69666665723D4B7572A1
:10C1A0007A7761686C20004B75727A7761686C20D1
:10C1B0002020202020200000616B746976656E20AD
:10C1C0004465636F646572200073706569636865B8
:10C1D000726E20202020202000005370726163685E
:10C1E00065202020202020202000004C616E6775F3
:10C1F00061676520202020202020000044657574A0
:10C2000073636820202020202020200000456E67D6
:10C210006C697368202020202020202000005461B9
:10C22000616C202020202020202020202000004E93
:10C23000656465726C616E647320202020200000AC
:10C240004C616E6775652020202020202020200072
:10C25000004672616E6361697320202020202020D7
:10C260000000537072616368652020202020202028
:10C270002000004974616C69656E697363682020F1
:10C280002020000053707261636865202020202008
:10C2900020202000005370616E69736368202020A5
:10C2A00020202020000053707261636865202020E8
:10C2B00020202020200000537072616368652020D8
:10C2C000202020202020000050656E64656C617580
:10C2D000746F6D6174696B0000416B746976696598
:10C2E00072656E2020202020000047657363687708
:10C2F000696E6469676B656974000046756E6B747E
:10C30000696F6E656E202020202000004B6F6E74D8
:10C31000616B746520202020202020000048616C83
:10C3200074652D5A65697420202020200000616BFF
:10C3300074697620202020200000000000000069A1
:10C340006E616B7469762020200000000000000000
:10C3500054617374652000000000000000000000BC
:10C36000005A656E7472616C6520757064617465E5
:10C370006E0000004D656E75204C6F636F202020AD
:10C38000202020000050726F6772616D2E204443A0
:10C390004320202000006D332050726F6772616D62
:10C3A0006D672E202000005265676C616765732001
:10C3B00020202020202000004C756D696E6F73696D
:10C3C00074652020202020000048616E64436F6E59
:10C3D00074726F6C20563220000053656C65637474
:10C3E000696F6E2020202020200000466F726D6152
:10C3F0007420646F6E6E6565732000004E6F6D2053
:10C4000020202020202020202020200000536169AF
:10C410007369652020202020202020200000435622
:10C4200020286279746529202020202020000043E4
:10C430005620286269742920202020202020000016
:10C440004164726573736520646520626173650081
:10C450000041647265737365206C6F6E677565204B
:10C4600000005265676973746572202020202020C7
:10C47000200000566F6965207072696E6369706193
:10C480006C6500005261696C436F6D20435620203B
:10C49000202020000041647265737365206D332095
:10C4A0002020202000003132384653204D6F646533
:10C4B000202020202000004A6F676469616C204DB5
:10C4C0006F646520202000005265676C61676520FD
:10C4D000733838202020200000426F6F737465721B
:10C4E00020202020202020200000496E74657266E4
:10C4F0006163652042617564200000436F6E662EA3
:10C500002041696775696C6C612E0000466F726D21
:10C510006174206C6F636F202020200000506175D3
:10C520007365207369676E616C204D4D0000526128
:10C53000696C436F6D20537570706F727400005595
:10C54000736572204E616D65202020202020000040
:10C55000506F6C2E6372742D636972637569740019
:10C560000053656E732E206372742D636972637459
:10C570000000746F75732061696775696C6C612E5A
:10C58000200000466F726D61742061696775696C87
:10C590006C2E00006E75722066FC722044434321AD
:10C5A00020202000004E617469762028313A31291C
:10C5B0002020202000004C696E6561722028323AEC
:10C5C0003129202020000050726F677265737369F3
:10C5D000762031202020000050726F6772657373DF
:10C5E0006976203220202000004143204D6F647581
:10C5F000732020202020202000004443204D6F6421
:10C6000075732020202020202000004B6F6E66696B
:10C610006775726174696F6E202000004D6F6475DC
:10C620006C65732073383800000000000054657397
:10C6300074206D6F64756C65207338380000506F1E
:10C640006C2E6372742D6369726375697400005394
:10C65000656E732E206372742D63697263740000BB
:10C66000746F75732061696775696C6C612E200049
:10C6700000466F726D61742061696775696C6C2E1C
:10C680000000204D4D2031202031342000000000DA
:10C69000000000204D4D2031202032376100000085
:10C6A00000000000204D4D20312020323762000074
:10C6B0000000000000204D4D2032202031342000A9
:10C6C000000000000000204D4D2032202032376154
:10C6D00000000000000000204D4D203220203237A5
:10C6E000620000000000000020444343202020316D
:10C6F000342000000000000000204443432020209C
:10C700003238200000000000000020444343202075
:10C710003132382000000000000000206D3320205E
:10C72000203132382000000000000000303A206143
:10C7300075732020202020202020000000313A2086
:10C740005461696C62697473202020000000323AE1
:10C75000202B2049644E6F746966792000000033F5
:10C760003A202B204163636573736F727900000078
:10C770004164726573736520286B75727A290000B5
:10C7800000416E666168722D4765736368772E009D
:10C790000000416E666168722D5665727A2E000047
:10C7A0000000004272656D732D5665727A2E00008E
:10C7B0000000000048F6636873742D476573636872
:10C7C000772E0000004D697474656E2D47657363A4
:10C7D00068772E00000056657273696F6E00000066
:10C7E000000000000000004865727374656C6C65A1
:10C7F000722D4944000000004164722E20286C61B3
:10C800006E672D4829000000004164722E20286CBC
:10C81000616E672D4C2900000000436F6E736973D1
:10C82000742D4164726573736500005261696C43D5
:10C830006F6D000000000000000000004B6F6E668E
:10C84000696775726174696F6E00000000204C6545
:10C8500063742E000000000000000000000020456E
:10C860007272657572000000000000000000002078
:10C870004563726974202000000000000000000081
:10C880006E6567617469762028444343290000007F
:10C8900000706F736974697620284D4D290000007F
:10C8A00000005A69666665723D4B75727A776168F9
:10C8B0006C20004B75727A7761686C2020202020F4
:10C8C00020200000616B746976656E204465636F9B
:10C8D0006465722000456372697420202020202046
:10C8E00020202020000053707261636865202020A2
:10C8F000202020202000004C616E67756167652054
:10C900002020202020200000446575747363682077
:10C91000202020202020200000456E676C6973686D
:10C92000202020202020202000005461616C202045
:10C9300020202020202020202000004E65646572E9
:10C940006C616E6473202020202000004C616E67B3
:10C9500075652020202020202020200000467261C4
:10C960006E63616973202020202020200000537016
:10C97000726163686520202020202020200000496B
:10C9800074616C69656E6973636820202020000003
:10C9900053707261636865202020202020202000D1
:10C9A000005370616E69736368202020202020206E
:10C9B00000005370726163686520202020202020D1
:10C9C00020000053707261636865202020202020C1
:10C9D0002020000050656E64656C6175746F6D6138
:10C9E00074696B0000416B746976696572656E20CD
:10C9F000202020200000476573636877696E6469B2
:10CA0000676B656974000046756E6B74696F6E655F
:10CA10006E202020202000004B6F6E74616B7465C7
:10CA200020202020202020000048616C74652D5AB1
:10CA300065697420202020200000616B74697620D5
:10CA40002020202000000000000000696E616B744F
:10CA500069762020200000000000000054617374FB
:10CA6000652000000000000000000000005A656E14
:10CA70007472616C65207570646174656E0000008D
:10CA800002061E1A1A1E06020E0E041F1F1F1F1F6B
:10CA900002040F0204181800101112161C181810A6
:10CAA00018191A1A1C1C1818101013171F1E1C18FE
:10CAB0000000040F110F0400040E1F04041F0E04D5
:10CAC000010101050D1F0C04001F1F1F1F1F1F0068
:10CAD0005F7369636865725F48432D322F736963C2
:10CAE0006865725F0E11111F1B1B1F0E52455345C7
:10CAF00054000000202020202020203C3E20202028
:10CB0000202020200000000020202020203C48433E
:10CB10002D323E2020202020000000002020202058
:10CB200020203C20203E202020202020000000004B
:10CB3000202020203C2048432D32203E2020202051
:10CB40000000000020202020203C202020203E202B
:10CB500020202020000000002020203C20204843EE
:10CB60002D3220203E202020000000002020202008
:10CB70003C2020202020203E2020202000000000FB
:10CB800020203C20202048432D322020203E202001
:10CB90000000000020203C202020202020202020F9
:10CBA000203E2020000000003C2020202020484380
:10CBB0002D3220202020203E000000003C2020209C
:10CBC00020202020202020202020203E00000000C7
:10CBD00020202020202048432D32202020202020EB
:10CBE000000000002048573D31352053573D312E7D
:10CBF000302E30002020416472657373653A200046
:10CC0000202077616974696E672E2E2E2E00000039
:10CC100020463A2000000000202020202020000094
:10CC20007265743D206F6E20206573633D6F66668C
:10CC30000000000020202020202020202020202074
:10CC40002020202020202020202020202020200004
:10CC5000204E722E3A200000457363203D200000D4
:10CC6000203D200020202020202020202000000027
:10CC7000232D4144523A2020202020200000000093
:10CC80004144523A20202020202020200000000093
:10CC9000455343203D204162627275636820202025
:10CCA0000000000020202020202020202020202004
:10CCB00020202020000000004543203D2056000099
:10CCC00055706461746500004678203C2D3E204913
:10CCD000636F6E20202020003D4CF6736368656E04
:10CCE000000000004443432020202020202020205A
:10CCF00020202020000000004D6F746F726F6C6167
:10CD00002020202020202020000000004C616E67A1
:10CD10003A20342E303235206D7320200000000080
:10CD20004B75727A3A20312E35206D7320202020E9
:10CD300000000000343D5320353D6720363D6B0038
:10CD4000343D7320353D4720363D6B00343D732024
:10CD5000353D6720363D4B00313D4220323D672056
:10CD6000333D7200313D6220323D4720333D720039
:10CD7000313D6220323D6720333D52005365722EB3
:10CD80002D4E722E3A20000055706461746520208B
:10CD90002020202020202000203D20557064617438
:10CDA000652020200000000020457363203D2063A3
:10CDB000616E63656C202020000000004E616D658F
:10CDC0003A000000466D743A00000000202D20005B
:10CDD000207365630000000020460000204F4B20B8
:10CDE0002020200043563A00204269743A00000097
:10CDF0004164722E3A200000526567200000000056
:10CE00004356200043563A20000000005549443A5A
:10CE100020307800206D7300415553002044434377
:10CE200000000000204D4D00302E2E2E3900000055
:10CE30004E722E3A00000000737461742E200000C0
:10CE4000636F6E742E20000020280000204D6F7448
:10CE50006F726F6C61000000427500004875000041
:10CE600048750000487500004875000048750000CE
:10CE700048750000487500004875000048750000BE
:10CE800048750000487500004875000048750000AE
:10CE9000487500004875000048750000487500009E
:10CEA0004675000048750000487500004875000090
:10CEB00048750000487500003E7500004875000088
:10CEC000487500004875000048750000487500006E
:10CED0004875000048750000367500004875000070
:10CEE000487500004875000048750000487500004E
:10CEF000487500004875000048750000487500003E
:10CF0000487500004875000048750000487500002D
:10CF1000487500004875000048750000487500001D
:10CF20003A7500004875000048750000487500001B
:10CF30004875000048750000327500006D332020F0
:10CF4000202000004D4D3120202000004D4D32208A
:10CF5000202000004443432020200000464F524D33
:10CF600041540000068100001A8100002E8100005B
:10CF700042810000068100005E8100005E810000A9
:10CF8000EC8200000083000014830000288300006E
:10CF90005283000066830000668300009C840000CA
:10CFA00064840000A48400008C8400009484000049
:10CFB0007C840000648400006484000064840000B9
:10CFC00064840000648400006484000064840000C1
:10CFD00064840000648400006484000064840000B1
:10CFE00064840000648400006484000064840000A1
:10CFF0006484000064840000648400006484000091
:10D000006484000064840000648400006484000080
:10D010006484000064840000648400006484000070
:10D020006484000064840000648400006484000060
:10D030006484000064840000648400006484000050
:10D040006484000064840000648400006484000040
:10D050006484000064840000648400006484000030
:10D060006484000064840000648400006484000020
:10D070006484000064840000648400006484000010
:10D080006484000064840000648400006484000000
:10D0900064840000648400006484000064840000F0
:10D0A00064840000648400006484000064840000E0
:10D0B000748400008484000000850000BC840000AB
:10D0C00008850000F8840000F0840000D884000087
:10D0D000BC840000BC840000BC840000BC84000050
:10D0E000BC840000BC840000BC840000BC84000040
:10D0F000BC840000BC840000BC840000BC84000030
:10D10000BC840000BC840000BC840000BC8400001F
:10D11000BC840000BC840000BC840000BC8400000F
:10D12000BC840000BC840000BC840000BC840000FF
:10D13000BC840000BC840000BC840000BC840000EF
:10D14000BC840000BC840000BC840000BC840000DF
:10D15000BC840000BC840000BC840000BC840000CF
:10D16000BC840000BC840000BC840000BC840000BF
:10D17000BC840000BC840000BC840000BC840000AF
:10D18000BC840000BC840000BC840000BC8400009F
:10D19000BC840000BC840000BC840000BC8400008F
:10D1A000BC840000BC840000BC840000BC8400007F
:10D1B000BC840000BC840000BC840000BC8400006F
:10D1C000BC840000BC840000BC840000E884000033
:10D1D000E08400007E850000468500008685000012
:10D1E0006E850000768500005E85000046850000A3
:10D1F0004685000046850000468500004685000003
:10D2000046850000468500004685000046850000F2
:10D2100046850000468500004685000046850000E2
:10D2200046850000468500004685000046850000D2
:10D2300046850000468500004685000046850000C2
:10D2400046850000468500004685000046850000B2
:10D2500046850000468500004685000046850000A2
:10D260004685000046850000468500004685000092
:10D270004685000046850000468500004685000082
:10D280004685000046850000468500004685000072
:10D290004685000046850000468500004685000062
:10D2A0004685000046850000468500004685000052
:10D2B0004685000046850000468500004685000042
:10D2C0004685000046850000468500004685000032
:10D2D0004685000046850000468500004685000022
:10D2E00046850000468500005685000066850000E2
:10D2F000E6850000A2850000EE850000D6850000CE
:10D30000DE850000BE850000A2850000A285000029
:10D31000A2850000A2850000A2850000A285000071
:10D32000A2850000A2850000A2850000A285000061
:10D33000A2850000A2850000A2850000A285000051
:10D34000A2850000A2850000A2850000A285000041
:10D35000A2850000A2850000A2850000A285000031
:10D36000A2850000A2850000A2850000A285000021
:10D37000A2850000A2850000A2850000A285000011
:10D38000A2850000A2850000A2850000A285000001
:10D39000A2850000A2850000A2850000A2850000F1
:10D3A000A2850000A2850000A2850000A2850000E1
:10D3B000A2850000A2850000A2850000A2850000D1
:10D3C000A2850000A2850000A2850000A2850000C1
:10D3D000A2850000A2850000A2850000A2850000B1
:10D3E000A2850000A2850000A2850000A2850000A1
:10D3F000A2850000A2850000A2850000A285000091
:10D40000A2850000CE850000C6850000FA8B0000D2
:10D41000108C0000608C0000E09A0000A88C0000D6
:10D42000D48C0000308E00003E8E0000E09A000098
:10D43000E09A0000308E0000308E0000608E000008
:10D440009A8E0000BA8E0000D68E0000D68E0000A4
:10D45000E08E0000CA8E0000128F0000228F0000B4
:10D46000328F00005A8F0000928F000098900000C9
:10D47000A8900000E09A0000C8900000E49000002E
:10D48000E4900000E4900000209600003296000036
:10D490007E960000E09A0000C4960000EA96000024
:10D4A000C8970000D6970000E09A0000E09A0000BC
:10D4B000C8970000C8970000589800009698000090
:10D4C000B2980000CC980000CC980000D4980000DE
:10D4D000C098000002990000109900001E990000F9
:10D4E000449900007A9900005E9A00006C9A00004E
:10D4F000E09A0000829A0000969A0000969A000036
:10D50000969A00002D2D2D00535450005352540074
:10D51000484C5400474F20005253540020203E00F6
:10D520003C20200053544F502020000053484F52BD
:10D530005421000048414C542020000050524F47D5
:10D54000522E0000524553455420000030313233F2
:10D550003435363738396162636465666768696A8D
:10D560006B6C6D6E6F707172737475767778797A93
:04D5700000000000B7
:0CD5740080F0FA0280F0FA0232000000A1
:00000001FF
